:020000040800F2
:10000000F8FF012061B80908E1B809086D4A08083D
:10001000E1B80908E1B80908E1B8090800000000E2
:10002000000000000000000000000000E1B8090826
:10003000E1B8090800000000E1B80908211008082B
:10004000E1B80908E1B80908E1B80908E1B8090808
:10005000E1B80908E1B80908C155080801570808BE
:10006000C15608088156080841560808BD600908AD
:10007000AD6009089D6009088D600908796009086C
:100080006560090851600908E1B80908E1B8090884
:10009000E1B80908E1B80908E1B8090801560808FB
:1000A000E1B809089D6F0908E1B809088D6F0908D2
:1000B0007D6F09086D6F09085D6F0908F15E090819
:1000C000155F0908355E0908595E0908F1600908DD
:1000D000E5600908D9100808CD100808C110080803
:1000E00081550808E1B8090800000000056F0908FB
:1000F000156F0908F56E09083D6F09083D6009088C
:10010000E1B809088D3509084D6F0908D96009085B
:10011000B5100808E1B80908E1B80908B580040875
:10012000296009081560090801600908ED5F0908E0
:10013000D95F0908E1B80908E1B80908E1B8090878
:1001400000000000000000000000000000000000AF
:10015000C55F0908B15F09089D5F0908A910080873
:10016000E1B80908E1B80908E1B80908E1B80908E7
:10017000E1B80908E1B80908E1B809080000000081
:10018000E1B80908E1B809089D10080891100808AD
:10019000CD600908E1B80908E1B80908E1B8090823
:1001A000E1B80908E1B80908E1B80908E1B80908A7
:1001B000E1B80908E1B80908E1B80908E1B8090897
:1001C000E1B80908E1B80908E1B80908E1B8090887
:1001D000E1B809083D830408E1B80908E1B8090855
:1001E000E1B80908E1B80908E1B80908E1B8090867
:1001F000E1B80908E1B80908E1B80908E1B8090857
:10020000E1B80908E1B80908E1B80908E1B8090846
:10021000E56E0908D56E0908C56E0908E1B8090838
:10022000E1B80908E1B80908E1B8090800000000D0
:10023000C1370908E1B8090800000000E1B8090861
:10024000E1B80908E1B80908E1B80908E1B8090806
:10025000E1B80908E1B80908E1B80908E1B80908F6
:10026000E1B80908E1B80908E1B80908E1B80908E6
:10027000E1B80908E1B80908E1B809080000000080
:10028000E1B8090800000000E1B80908000000001A
:0802900000000000E1B80908BC
:08029800E4B2090001000000BE
:1002A00000C20100000008000A0600020000004031
:1002B0000100000009026400030100C032090400CB
:1002C000000103000000092111010001223600078E
:1002D00005830308000A080B010202020100090459
:1002E00001000102020100052400100105240100A3
:1002F0000204240202052406010207058203080005
:10030000FF09040200020A00000007050102400084
:100310000007058102400000CDD40408B59E040802
:1003200049D20408000000002594040859D00408AC
:1003300051940408000000000000000000000000CC
:100340000594040815940408F5930408E59304083B
:100350001A03000000000000000000000000000080
:100360000000000000000000000000000403090479
:1003700012010002EF020140830456320002010222
:1003800003010000120100020200004083044057F4
:1003900000020102030108000090D00300000240A7
:1003A00010000240000000000000000000000B00F0
:1003B00000000000000000000000000000000240FB
:1003C00028000240010000000000000006000C00B0
:1003D00000000000000000000000000000000240DB
:1003E00040000240020000000000000010000D006C
:1003F00000000000000000000000000000000240BB
:1004000058000240030000000000000016000E002B
:10041000000000000000000000000000000002409A
:1004200070000240040000000000000020000F00E7
:10043000000000000000000000000000000002407A
:1004400088000240050000000000000026001000A7
:10045000000000000000000000000000000002405A
:10046000A000024006000000000000003000110063
:10047000000000000000000000000000000002403A
:10048000B8000240070000000000000036002F0006
:100490000000000000000000000000000004024016
:1004A00010040240000000000000000000003800BE
:1004B00000000000000000000000000000040240F6
:1004C000280402400100000000000000060039007E
:1004D00000000000000000000000000000040240D6
:1004E00040040240020000000000000010003A003A
:1004F00000000000000000000000000000040240B6
:1005000058040240030000000000000016003B00F9
:100510000000000000000000000000000004024095
:1005200070040240040000000000000020003C00B5
:100530000000000000000000000000000004024075
:10054000880402400500000000000000260044006E
:100550000000000000000000000000000004024055
:10056000A00402400600000000000000300045002A
:100570000000000000000000000000000004024035
:10058000B8040240070000000000000036004600EA
:100590000000000000000000000000007D000000DE
:1005A000010000000000803F0A0600020000004039
:1005B0000100000009022200010100E032090400EC
:1005C0000001030102000921110100012236000788
:1005D00005830308000A000009022200010100E06F
:1005E0003209040000010301020009211101000188
:1005F00022360007058303080007000009022200D5
:10060000010100E032090400000103010200092198
:10061000110100012236000705830308000A0000CB
:100620000A06000200000040010000000907430024
:10063000020104C032090400000102020100052485
:100640000010010524010001042402020524060013
:10065000010705820308001009040100020A0000D6
:10066000000705010240000007058102400000006C
:1006700009024300020100C0320904000001020225
:1006800001000524001001052401000104240202D8
:100690000524060001070582030800100904010073
:1006A000020A00000007050102000200070581029E
:1006B0000002000009024300020100C032090400E8
:1006C00000010202010005240010010524010001BF
:1006D0000424020205240600010705820308001015
:1006E00009040100020A00000007050102400000A1
:1006F000070581024000000005010905A101A100D4
:10070000050109300931093209330935093409363F
:1007100009371581257F750895088102050919019A
:10072000290815002501950875018102C0C0000047
:100730000921110100012236000000001000000014
:1007400000FF0000000000000000AA5507010000A3
:1007500001AA5505010000007EFF080064D30908C6
:10076000FF1FFF1F2D202D2D202D2D2D2D202D2D58
:100770002D2D00000000000000000000000000001F
:10078000000000AA550B010000AA5505010000AAAF
:10079000550902000000AA5503009F000100000057
:1007A000C0120000648F0024000000003C8F002471
:1007B00000000000F8450A0874450A08000000001F
:1007C0002D830708A086010004000000000000003F
:1007D0000000000000000000000000000000000019
:1007E0000000000000000000000000000000000009
:1007F00000000000F8450A0800460A080000000052
:10080000EDF40708E8030000040000000000000009
:1008100000000000000000000000000000000000D8
:1008200000000000000000000000000000000000C8
:100830000000000008460A08000000000000000058
:10084000B90F00007D000000FF0000000000000064
:100850000000000000000000000000000000000098
:100860000000000000000000000000000000000088
:10087000000000004CC40A08000000000000000056
:10088000ED0500007D000000FF00000000000000FA
:100890000000000000000000000000000000000058
:1008A0000000000000000000000000000000000048
:1008B00000000000FC590A080000000000000000D1
:1008C000351100007D000000FF0000000000000066
:1008D0000000000000000000000000000000000018
:1008E0000000000000000000000000000000000008
:1008F0000000000010460A08000000000000000090
:1009000011EC0708E80300000300000000000000ED
:1009100000000000000000000000000000000000D7
:1009200000000000000000000000000000000000C7
:100930000000000014460A0800000000000000004B
:1009400039EB06081027000003000000000000003B
:100950000000000000000000000000000000000097
:100960000000000000000000000000000000000087
:100970000000000054C00A0800000000AD0D060889
:10098000D14A08085F760000050000000000000062
:100990000000000000000000000000000000000057
:1009A0000000000000000000000000000000000047
:1009B00000000000F0C30A08000000000000000072
:1009C000216408081027000001000000000000005A
:1009D0000000000000000000000000000000000017
:1009E0000000000000000000000000000000000007
:1009F0000000000020460A0800000000000000007F
:100A0000A5E40708E803000005000000000000005E
:100A100000000000000000000000000000000000D6
:100A200000000000000000000000000000000000C6
:100A3000000000002C460A08000000000000000032
:100A40000D860708204E0000030000000000000093
:100A50000000000000000000000000000000000096
:100A60000000000000000000000000000000000086
:100A7000000000003C460A080000000000000000E2
:100A8000DD830708204E0000030000000000000086
:100A90000000000000000000000000000000000056
:100AA0000000000000000000000000000000000046
:100AB000000000004C460A08000000000000000092
:100AC00051F10708400D0300030000000000000082
:100AD0000000000000000000000000000000000016
:100AE0000000000000000000000000000000000006
:100AF000000000005C460A08000000000000000042
:100B000029B20708102700000100000000000000C3
:100B100000000000000000000000000000000000D5
:100B200000000000000000000000000000000000C5
:100B300000000000A0450A080000000000000000BE
:100B4000A593050810270000030000000000000026
:100B50000000000000000000000000000000000095
:100B60000000000000000000000000000000000085
:100B70000000000064460A080000000000000000B9
:100B8000ED510608A08601000100000000000000F1
:100B90000000000000000000000000000000000055
:100BA0000000000000000000000000000000000045
:100BB000000000006C460A08000000000000000071
:100BC00091EA070850C30000010000000000000087
:100BD0000000000000000000000000000000000015
:100BE0000000000000000000000000000000000005
:100BF0000000000074460A08000000000000000029
:100C000081E60708A8610000010000000000000064
:100C100000000000000000000000000000000000D4
:100C200000000000000000000000000000000000C4
:100C30000000000080460A080000000000000000DC
:100C400065F30508A0860100010000000000000017
:100C50000000000000000000000000000000000094
:100C60000000000000000000000000000000000084
:100C7000000000008C460A08000000000000000090
:100C800071150808A00F000001000000000000001E
:100C90000000000000000000000000000000000054
:100CA0000000000000000000000000000000000044
:100CB0000000000098460A08000000000000000044
:100CC000B9D2050810270000010000000000000054
:100CD0000000000000000000000000000000000014
:100CE0000000000000000000000000000000000004
:100CF00000000000A4460A080000000000000000F8
:100D0000E1CA05081A4100000100000000000000CF
:100D100000000000000000000000000000000000D3
:100D200000000000000000000000000000000000C3
:100D300000000000A8460A080000000000000000B3
:100D40008D090508102700000100000000000000C8
:100D50000000000000000000000000000000000093
:100D60000000000000000000000000000000000083
:100D70000000000088450A08000000000000000094
:100D80004939060850C300000100000000000000BF
:100D90000000000000000000000000000000000053
:100DA0000000000000000000000000000000000043
:100DB00000000000B4460A08000000000000000027
:100DC0006D110508400D0300000000000000000048
:100DD0000000000000000000000000000000000013
:100DE0000000000000000000000000000000000003
:100DF00000000000BC460A080000000000000000DF
:100E000069830708400D0300000000000000000097
:100E100000000000000000000000000000000000D2
:100E200000000000000000000000000000000000C2
:100E300000000000C4460A08000000000000000096
:100E40000DDE050850C30000030000000000000094
:100E50000000000000000000000000000000000092
:100E60000000000000000000000000000000000082
:100E700000000000D0460A0800000000000000004A
:100E8000B190070840420F00000000000000000081
:100E90000000000000000000000000000000000052
:100EA0000000000000000000000000000000000042
:100EB00000000000DC460A080000000000000000FE
:100EC000398A070850C3000000000000000000003D
:100ED0000000000000000000000000000000000012
:100EE0000000000000000000000000000000000002
:100EF000000000000100000000000100E00101000E
:100F0000AD780508000000000000000088D5090841
:100F1000FFFFFFFF0801FF010101FF00FFFFFFFFCF
:100F200049EC05080000000000000000D0DD0908C1
:100F300071EF0508000000000000000088DD0908CE
:100F40002D202D2D202D2D2D2D202D2D2D0000007F
:100F50000000000000000000000000000000000091
:100F600000000000000000000000000044DD09084F
:100F70008C8900249CFF2C0100000000309C002480
:100F8000E0150C1700000000089900240200000082
:100F90007CDD09086C94002488136F1701000000A1
:100FA0006E94002488136F17000000002E61002447
:100FB00000000000000000002C6100240000000080
:100FC000000000002A610024000000000000000072
:100FD00028610024000000000000000026610024B9
:100FE0000000000000000000246100240000000058
:100FF00000000000000500240000000000000000C8
:10100000F4930024030000006CDE090864940024BB
:1010100088136F1701000000D689002488136F170A
:1010200000000000757905080000000000000000C5
:101030007CDE09080999002401000000D0DE0908BF
:10104000D889002401000000DCDE0908CE890024D4
:1010500002000000E4DE09080000000000000000BB
:1010600000000000F0DE09085D79050800000000BE
:10107000000000008CDF09080000000000000000F4
:1010800000000000E0DF0908000000000000000090
:101090000000000050E009087094002402000000E5
:1010A00088E00908D2890024E0150C170000000030
:1010B00028A400247CA400240100000000000000FB
:1010C00000000000A91206088CA700240000000000
:1010D000000000000000000048F6090800000000C1
:1010E000000000000000000000F7090800000000F8
:1010F0000000000000000000ACF609089D1806087A
:101100000000000000000000D8F50908D601FF002B
:10111000FFFFFFFF01000000FA00000001000000D7
:1011200001000000010000000001010100000000BA
:101130007AA200240000F4010100000078A200243B
:101140000000F4010100000076A200240000F40178
:101150000100000074A200240000F401010000005E
:1011600072A200240000F4010100000070A200241B
:101170000000F401010000006EA200240000F40150
:1011800001000000C5FC050889FC050800000000FE
:101190009CE209085EA20024053201006CA2002432
:1011A0006400F401010000006AA200246400C40984
:1011B000010000005CA20024E803D0070100000049
:1011C0005AA20024E803D0070100000058A200241E
:1011D000E803D0070100000056A200241E00B80B4F
:1011E0000100000064A2002405000F0001000000BF
:1011F00066A2002403000A000100000054A200249B
:101200001E00F4010100000068A20024020000009A
:1012100028E3090852A20024140064000100000021
:1012200060A200243200E8030100000050A2002464
:101230000000C8000100000029A2002400C801002D
:1012400028A200240050010027A20024005A010017
:1012500025A200240200000034E3090854510A08C2
:101260005C510A08EA6000240100C4090000000083
:10127000E86000240100C40900000000E6600024CA
:101280000100C40900000000E46000240100C4095A
:1012900000000000E06000240100C409000000001C
:1012A000E26000240100C40900000000DE600024A8
:1012B0000100C40900000000DC6000240100C40932
:1012C00000000000AF94002400C80100AE94002488
:1012D00000C80100AC9400240000FFFF0A000000D9
:1012E000AA9400240100C80001000000A894002472
:1012F0003200307532000000A69400247EFF1400F6
:1013000005000000A494002405002C010500000045
:10131000A3940024055A0500A094002400FF0100B6
:10132000A294002402000000BC0F00249E9400241C
:10133000030000006CDA09089F94002400FF0100FC
:10134000A194002402000000BC0F00249D940024FE
:10135000030000006CDA090819FC0508A9FB050860
:101360000000000040E3090890A20024EE02CA0831
:10137000010000008EA2002400C8010064000000EB
:101380008DA2002400C80100640000008CA200248B
:10139000020000004CE409088A9400240000803E0A
:1013A000050000008894002480C1803E05000000F4
:1013B000829400240083007D0500000080940024B6
:1013C00080C1803E050000007B94002400FF0100E6
:1013D000749400246400F40101000000729400245D
:1013E0000400000058E40908719400240200000081
:1013F0006CE4090857A000240D00000078E40908F7
:1014000054A000240064010052A0002432001027E0
:101410000A00000050A000240D00000078E4090834
:101420004FA000240D00000078E409084EA000241D
:1014300002000000B0E4090896A200243E0000006B
:10144000BCE4090894A200240100FF7F0100000011
:1014500093A2002402000000B8E5090859A0002466
:1014600003000000C8E5090858A00024030000009C
:10147000C8E5090816A20024000A010014A20024ED
:101480000000E8030100000012A200240000E803AD
:101490000100000010A200240000E8030100000089
:1014A0000EA200240000E8030100000006A20024B0
:1014B0000000E803010000000CA200240000E80383
:1014C000010000000AA200240000E803010000005F
:1014D00008A200240014010024A20024020000003D
:1014E000D8E5090822A200240000F4010100000050
:1014F00020A200240000F401010000001EA200242C
:101500000000F401010000001CA200240000F4010E
:10151000010000001AA200240000A00F010000003A
:1015200018A200240000A00F010000003DA200242A
:10153000196401003CA2002402000000E4E509084F
:101540003AA20024E803D0070A00000038A20024D1
:10155000006401000A0000002DA2002400640100C4
:101560002CA200240064010034A2002400640100C5
:101570000A00000033A20024006401000A000000F9
:1015800032A20024006401000A00000037A20024F7
:1015900000FF01000A00000036A2002400FF010045
:1015A0000A00000035A2002400FF01000A0000002C
:1015B00031A2002401FF01000A00000030A2002433
:1015C00001FF01000A0000002FA2002401FF01001A
:1015D0000A00000062A000240000F40101000000E5
:1015E00060A000240000A00F010000005EA0002405
:1015F0000000A00F010000005CA000240000A00F6C
:10160000010000005AA000240000A00F010000000B
:10161000F5A6002400C80100F4A60024006401001F
:10162000F3A6002400640100F2A600240064010077
:10163000F1A6002400640100F0A60024FF080100C8
:10164000EFA600240164010011FB0508D5FA050886
:1016500000000000F0E50908F8A6002401320100AE
:10166000F7A600240100000060E60908F6A60024A1
:101670000400000068E60908EEA6002400640100EA
:10168000ECA600241400E80301000000EAA60024F0
:10169000E80330750A000000E8A6002400C8010035
:1016A000E7A6002400C80100E6A6002400C8010047
:1016B000E5A6002400320100FAA60024004B010038
:1016C000F9A60024040000007CE60908E4A6002432
:1016D000006401000A00000008A700240000D007F1
:1016E0000100000003A7002400C8010002A7002495
:1016F00000C8010001A7002400C8010006A70024BB
:101700000000D0070100000000A7002400C801006D
:10171000FFA6002400C80100FEA6002400C80100A6
:1017200004A700240000D00701000000FDA600244B
:1017300000C80100FCA6002400C80100FBA600248C
:1017400000C80100FDF80508E5F8050800000000E4
:1017500090E609084BA00024005A01004AA000248A
:1017600000C8010048A00024E803D00701000000E1
:101770000000000000000000E91206082CE709083C
:101780004D4154454B483734335F34323658580056
:101790009C940024000301009B940024000301009A
:1017A000D17B0508857B05080000000080E709085B
:1017B000457B0508FD7A0508000000001CE80908C3
:1017C0007DF805086DD20508000000009CE80908B6
:1017D0008C94002401030100A1FD050875FD050896
:1017E00000000000F4EB0908817A0508357A050845
:1017F0000000000064EC09080DF90508B51306089F
:101800000000000000ED0908BD150608CDFD050823
:1018100000000000A8ED09084DF9050800000000CF
:101820000000000028EE090805FA0508ADF90508D2
:10183000000000008CEE090899FA05085DFA050819
:101840000000000034EF0908197A06084DFB05086E
:1018500000000000C0EF09084FA2002401060100AB
:1018600085F905085DF9050800000000BCF00908CD
:101870005179060865140608000000002CF10908DB
:10188000617A060829150608000000007CF20908A4
:101890004EA2002401030100BDF8050895F80508D3
:1018A0000000000050F30908B97A060800000000A3
:1018B00000000000B4F30908CD7A050899C90508AD
:1018C0000000000034F409080000000000000000DF
:1018D00000000000C0F4090881FB0508A1150608F6
:1018E0000000000030F50908FFFFFFFF0000803F07
:1018F00000000000000000000000000000000000E8
:1019000000000000000000000000000000000000D7
:10191000000000000000803F000000000000000008
:10192000000000000000803F0000000000000000F8
:10193000000000000000803F0000000000000000E8
:1019400000000000010000000000FA430000FA431C
:101950000000803F39B407080000000000000000CC
:1019600000000000FFFFFFFFFF000000000000007C
:10197000B4C300240800000000000000A4C3002439
:10198000080000002D08040811080408CD07040809
:1019900000000000C1070408AD0704089907040807
:1019A0000000000000000000000000000000000037
:1019B0008907040800000000790704082D090408BD
:1019C00021090408E9080408FD080408A10804081E
:1019D0008D08040879080408A10D04087507040897
:1019E000F1060408150D0408685E0C0002000000F2
:1019F0000010000010000240000000000011000074
:101A000028000240000000000012000040000240D8
:101A10000000000000130000580002400000000019
:101A200000140000700002400000000000150000DB
:101A3000880002400000000000160000A0000240E4
:101A40000000000000170000B80002400000000085
:101A500000200000100402400000000000210000EF
:101A60002804024000000000002200004004024060
:101A700000000000002300005804024000000000A5
:101A80000024000070040240000000000025000057
:101A9000880402400000000000260000A00402406C
:101AA0000000000000270000B80402400000000011
:101AB00001000000A00F0000B80B00000102FFFFB2
:101AC00001000000FFFF000048C00A0800000802F3
:101AD000050306000000000050C00A0801000802CB
:101AE0000504060000000000786D0A080200FE01EF
:101AF0000110030000000000AC540A0803001402A7
:101B0000000300000000000058C00A0804001F0283
:101B1000020008000000000060C00A0805001F0263
:101B2000020108000000000068C00A080600250243
:101B300001001100FE810300FFFFFFFFFFFF010016
:101B4000F40100002A0000000000000075B4040841
:101B500005D80408559E040895D9040819B5040849
:101B60008593040871930408699304087C400A086B
:101B7000E0010400E0010208050000000000000090
:101B800090010400900102080500000000C0000060
:101B900000000000000000000F060000000100002F
:101BA00000000030F42200300003000101000000BA
:101BB00040D2002440E8002400030000010000009F
:101BC000FF000000281900240000000000000000B1
:101BD0000000000000000000000000000000000005
:101BE00000000000000000000000000000000000F5
:101BF00000000000000000000000000000000000E5
:101C000000000000000000000000000000000000D4
:101C100000000000000000000000000000000000C4
:081C20000000000000000000BC
:101C280001000000010000001C1B00200000000053
:041C38002000000088
:020000040804EE
:100000002DE9F04F022389468A462DED108B99B0D9
:10001000DFEDCABA14930346169004331592179372
:100020004FEADA06169DDDF85CC04FEACA0305EB1D
:1000300046111396F0004FF0000B01EB0614370148
:100040000390A6EB86020194049706EB460E04EBA0
:10005000C202041D381D06EB86072C44C6EBC608F9
:1000600002972844029D02EB46174FEAC808ED00AC
:1000700001EBC60602954FEA0E1505954FEACE052F
:100080000695139D4FEA451E019D95ED007AD344D8
:1000900092ED005AD7ED004AD945D1ED006A50EDF6
:1000A000013A35EE241AD6ED002A1CED016A73EEF2
:1000B000875A54ED017A33EEC73A36EE264A77EE88
:1000C000A21A36EE666A77EEE27A74EE256A71EE6F
:1000D000812A77EE633A37EEC57A36EEA22A77EEBA
:1000E000E47A76EEE26A0CED012A37EE247A77EEB6
:1000F000857AD1ED018AC1ED006A74EE655A96EDFC
:10010000015AB0EE460A94ED004AA7EE2B6AD2EDF2
:10011000010AE7EEAB3A74EE456AD7ED012AA7EE85
:100120006B0A9CED007AD5ED014A34EE054A37EEB4
:10013000689A90ED005A36EEE02A76EEE26A30EEEA
:10014000A28A32EE222A76EEA06AF0EE492A75EEF5
:10015000640A37EE287A75EE249AE2EE6B2A74EE82
:10016000C54AF0EE608AB0EE40AAE6EEAB4AE6EE93
:10017000AB8AA6EEEBAAF0EE496AB0EE629A37EED1
:10018000695AE2EE2B6AB0EE432A74EE08AAA7EE93
:10019000EB9AA7EEAB2A77EE297A35EE617A75EE07
:1001A000C89A35EE415A75EEC45A37EEAABA77EEC0
:1001B000EA7A37EE011A8CED00BA36EE287AC1EDF4
:1001C000017A39EE844A76EEC27A194475EE885A7D
:1001D0009C4435EE215A00ED014A70EE8A0A70EE19
:1001E000244AC5ED005A36EE686A80ED001A72EEB8
:1001F000A33A85ED015A33EE093A04ED017A72EE25
:10020000266A87ED006A1D44C6ED000A1844C2ED57
:10021000004AC4ED007A1C44C7ED016A1F44C6EDD4
:10022000013A1E4482ED013A1A443FF62EAF139A6A
:10023000072A40F2C681039A0EF1080E169F08F1B4
:1002400008000832029E059D4FF0000894463A4689
:10025000083608357244069C0499D346109207EB81
:100260000C0208340C310F92BA190E927A190D92C1
:100270003A190C923A180B927A18099207F10C026B
:100280000A9201220892149ADDF824C09044159A2B
:100290000A9F02EBC8020B9EA8EB880E0C9D02EB96
:1002A000C80192ED00BA0D9C01EBC802D1ED00AA85
:1002B0000E9802EBC80192ED00AA01EBC802D1ED45
:1002C000009A02EBC80192ED009A01EBC802D1ED51
:1002D000008A0F9902EB0E1E92ED008A109A0EEB27
:1002E000C80ADEED017A1192CDED047A0AEBC8025C
:1002F000DAED017A02EBC80A1291CDED057AD2ED62
:10030000017A0AEBC802DDF820E0CDED017ADAEDE2
:10031000017A02EBC80ACDED067AD2ED017A0AEB3A
:10032000C802CDED027ADAED017ACDED077AD2ED91
:10033000017ADDE91121CDED037A01E0F304353FC7
:1003400017ED017ADE44D2ED007A94ED005AF145C2
:10035000D5ED006A37EE274AD0ED004A77EE677A8E
:100360001CED016A96ED007A91ED001A76EE055AC1
:1003700036EE872A97ED00DA71EE24EA76EE453AFA
:1003800074EE252A31EE641A35EE466A3EEE825A44
:1003900074EE655A31EE664A72EE854A31EE471ABE
:1003A000B0EE67CA47ED014A34EE077AD1ED014A53
:1003B00031EE261AD0ED016A72EEC52A95ED014A9A
:1003C000A7EE6BCA74EEE60A96ED010AE7EE2B7A09
:1003D00092ED017A94ED015A74EEA64A3DEE473A49
:1003E000DCED006A70EEC4CA70EEC00AB0EE43EAFB
:1003F0007CEE80CA74EE001A70EE840AACEEEBEA72
:1004000036EEC54A3DEE077AB0EE63DA36EE850A7F
:10041000ACEEAB3AF0EE4EDAA1EE2BDAA1EE2B6A9F
:10042000E1EE6BDA75EE666AB0EE441AF0EE4CCA95
:1004300037EE405AA0EEAB1AE0EEEBCAE0EEAB6A44
:1004400037EE007A74EEA10A35EEE1FA75EEE45A61
:1004500075EE6EFA37EE600A71EEA55ADDED061AFA
:1004600035EE425A7FEE244A3FEE822A22EEE1FA2E
:1004700061EE80FADDED051A3EEE855A3EEE066A23
:1004800073EEAD3A21EE82EA73EE4DDA3DEE033AB9
:1004900024EEE1DADDED071A34EE2C4A7CEE266A12
:1004A00061EE85CA25EEE1CADDED041A77EE81EA38
:1004B00077EEC17AE9EEA2FADDED032AA9EE80FA21
:1004C0009DED030AAAEEA4EADDED014AAAEE82DA66
:1004D0009DED012AE8EEA5CADDED025AA8EE85CA17
:1004E0009DED025A21EEAD1A62EE832A6EEEE11AFC
:1004F00027EEC00A64EEA34A26EEC22A65EE865AAB
:1005000024EE455AABEE2E1AEBEE2D1AE8EE272A12
:10051000A8EE030AEAEE264AAAEE232AE9EE045AD6
:10052000A9EE065A37EE207A87ED007A1F44C2ED15
:1005300000FA82ED01FA1A440CED01EA8CED00DAC2
:100540009C44C4ED00CA84ED01CA1C4481ED001A2C
:10055000C1ED011A1944C6ED002A86ED010A1E44B8
:10056000C0ED005A80ED015A1844C5ED004A85EDF2
:10057000012A1D443FF6E4AE1099089A0831013271
:1005800010910F99089208310F910E9908310E9130
:100590000D9908310D910C9908310C910B99083186
:1005A0000B910A9908310A91099908310991139917
:1005B00091427FF468AE149B8A46DB009BB2149391
:1005C0002EE519B0BDEC108BBDE8F08F124B30B4A6
:1005D0001D686B6A28B943EA01430020AB6230BC56
:1005E0007047AC6A013803EB14440BD0002303F1CD
:1005F0004002013305EB8202DBB25268834204EB16
:100600001244F4D3403044EA014405EB80004460D6
:10061000002030BC704700BF88190024037870B4F4
:100620002BB30246C0F10105531912F8014FDBB29A
:10063000002CF9D101335B000E4C03220B8084F8AF
:10064000083484F80924017879B1022300265A1C61
:10065000E518023354FA82F285F80814DBB282F806
:10066000086410F8011F0029F1D170BC7047022303
:10067000E2E700BF8819002430B5EFF31181802331
:1006800083F312880A4AD2F80835D2F80C45D2F81A
:100690000805D2F80C55CAB282F31188013BA84272
:1006A00094BF4FF4006000201B1B184430BD00BFF6
:1006B00088190024012380F851307047014BD3F88A
:1006C000100570478819002401207047024BC3F8B9
:1006D0001425C3F81815704788190024024BC3F875
:1006E0001C25C3F8201570478819002470477047EF
:1006F000212870B505D0222829D0202810D000202C
:1007000070BD0029FBD0072AF9D1184B18791C6855
:100710005A799B79087100200C604A718B7170BD09
:100720000029ECD0072AEAD11148104B0C680E7949
:100730004D79D0F8182589791C601E715D71997109
:10074000002ADCD02146D0F814059047D7E70029CD
:10075000D5D0022AD3D1064AD2F82035002BCED0EC
:100760000988D2F81C059847C9E700BF000000249B
:10077000881900240020704703460A2201481A8085
:10078000704700BF080000240346642201481A8015
:10079000704700BF14000024012901D000207047D9
:1007A000014BD3F89030184700000024012901D0F4
:1007B00008F0FABD014BD3F88C3018470000002434
:1007C000014BD3F8883018470000002410B40B7890
:1007D0000A46044603F00303012B05D0022B0BD07D
:1007E00000205DF8044B70478B8843B920461146C2
:1007F0005DF8044B0CF07CBC8B88832BF6D0034B4C
:100800005DF8044BD3F88030184700BF0000002487
:1008100038B5054B04460D46DB6F98472946204600
:1008200009F036FB002038BD0000002438B5054B28
:1008300004460D469B6F9847294620460CF02EFE35
:10084000002038BD00000024F0B4002452004E1CEB
:100850002746030FB0F1204F4FEA001003F1300597
:1008600003F1370334BF0D550B5537550234A242FF
:10087000EFD1F0BC704700BF024808B5FFF7CEFECD
:10088000014808BDF8420A08901D0024024808B536
:10089000FFF7C4FE014808BD08430A08901D002464
:1008A0000B481A220B4B00681B680A80C01801D144
:1008B00009487047094B0822094910B51C68FFF721
:1008C000C3FF042207492046FFF7BEFF024810BDC0
:1008D00000E8F11F08E8F11FB000002404E8F11F50
:1008E000B2000024C2000024024808B5FFF796FEBB
:1008F000014808BD14430A08901D002408B520B91A
:100900000448FFF78BFE044808BD0448FFF786FE45
:10091000014808BD20430A08901D002444430A08EA
:10092000042301480B807047CC000024074A084B81
:1009300010B4122492F8240503F114020C8001284B
:100940000CBF184610465DF8044B70478819002408
:10095000D000002470B5574C00234FF4F0722021D2
:1009600004F22C5084F8283559F086FD04F20C70FE
:100970004FF4F072202159F07FFD94F8ED0810B18A
:1009800094F8EE380BB9002070BD43F029FEC4F88E
:10099000FC0828B183790BB1412BF4D12323C38008
:1009A0000D21454E3FF0F2FDD4F8FC0844F036F836
:1009B00094F8EE08013840B245F064FB02231021A0
:1009C000C4F8F40884F8F03850F094F9B6F8F6104A
:1009D000D4F8F40850F08EF9D4F8FC0844F018F874
:1009E000FF218C2051F0E6F90546D4F8FC0844F0CC
:1009F00015F80421D4F8F40850F07CF91B2D05D02B
:100A0000D4F8FC0820213FF0C1FDBCE70122D4F856
:100A1000FC3884F828250BB12322DA80B6F8F610CA
:100A2000D4F8F40850F066F9D4F8FC0843F0F0FF6D
:100A300040210A2051F0BEF9FF218A2051F0BAF975
:100A4000D4F8FC0843F0EAFFD4F8F408042150F08D
:100A500051F90821D4F8F408A6F8F61050F04AF934
:100A6000B6F8F610D4F8F40850F044F9D4F8FC08BD
:100A700043F0CEFF0221002051F09CF9D4F8FC088D
:100A800043F0CCFFD4F8F408042150F033F994F883
:100A9000052994F806390120C2F1200294F80419BE
:100AA000C3F1100384F8072984F8083984F8001981
:100AB00070BD00BF88190024000000240F4B07B54B
:100AC000D3F8F8205208B2FBF1F3B3F5803F02D31C
:100AD000012AF7D8F9E799B2019056F0FBFB0849D3
:100AE00041F27813074A0198CA5001F58B51002250
:100AF000183103B05DF804EB56F092BA0000002400
:100B000088190024DDF105082DE9F0478846002901
:100B100051D04618451EDFF8A4908024013EDFF82E
:100B2000A0A0EFF3118184F31288D9F80825C9B287
:100B3000D9F80C05D9F80835D9F80CC581F3118816
:100B4000634594BF4FF400630023121A1344012B32
:100B50001AD1012040F0C4F9EFF3118184F3128817
:100B6000D9F80825C9B2D9F80C05D9F80835D9F84B
:100B70000C7581F31188BB4294BF4FF400630023CE
:100B8000121A1344012BE4D0EFF3118284F312887C
:100B9000D9F80C35D2B215F8011F534483F88810E8
:100BA000D9F80C350133C3F30A03C9F80C3582F3C5
:100BB0001188B542B5D14046BDE8F08788190024B8
:100BC000802A0024F8B5002390F8505080F8503067
:100BD000CDB10F4E96F8242B032A16D1D6F85C7BA4
:100BE00000F13C0429462046FFF78EFFD6F85C3B17
:100BF0002D1A0444DB1B322B01D8002DF2D1B5FA9B
:100C000085F04009F8BD0120FCE71846FAE700BF6F
:100C1000802A0024002280F85120D3E790F8502049
:100C2000531C0244DBB280F8503082F83C1090F83C
:100C300051200AB1132B00D9C4E77047F8B50B4E09
:100C40000D46144696F8243B032B0ED1D6F85C7B58
:100C5000002C0ADD21462846FFF756FFD6F85C3BFC
:100C6000241A0544DB1B322BF2D9F8BD802A00245C
:100C70000F49D1F8403B10B5B3B191F89848D3F87B
:100C8000042244B100244023D1F8580B01210CF078
:100C9000B5FA204610BD4FF40073D1F8580B01216E
:100CA0000CF0ACFA204610BD0224204610BD00BF57
:100CB000802A002410B50C4CD4F8103563B10B49D0
:100CC000013BD1F8602BC4F8103512F8014BC1F884
:100CD000602B047013B10123184610BDFFF7C8FF45
:100CE0000123184610BD00BF88190024802A002463
:100CF00013B5074CD4F8603B03B9FEE701A8FFF732
:100D0000D9FF0028F6D09DF8040002B010BD00BF46
:100D1000802A002410B50B68064C074AC4F8103529
:100D2000C2F8600B0BB1002010BDFFF7A1FF00203F
:100D300010BD00BF88190024802A0024154BDB68F1
:100D4000C3F3022310B4C3F107041A1D042C28BFF7
:100D50000424062A4FF0FF328CBF033B0023A2403D
:100D6000002821EA020101FA03F108DB09010A4B1C
:100D7000C9B2034483F800135DF8044B704700F0D8
:100D80000F000901054BC9B2034419765DF8044B05
:100D9000704700BF00ED00E000E100E0FCEC00E087
:100DA0002A4B41F287302A490022D3F8F830A1FBC0
:100DB00003132849DB0C10B5274C013B82B0C4F863
:100DC000700B04F66430C4F8641BC4F8742BC4F8C8
:100DD0006C2BC4F8683B11F0FBFC204B062137203C
:100DE000D3F8E82042F02002C3F8E820D3F8E83036
:100DF00003F020030193019BFFF7A0FFD4F8643BAD
:100E00004FF400001649174A4860D96841F00101C3
:100E1000D96099680A40062A06D0B2F5803F03D00F
:100E20001A6842F001021A600F490020D4F8403BD2
:100E30000E4A01F61C34C3F81002C2F82005C2F8AD
:100E40001805C3E9814102B010BD00BF00000024B5
:100E500083DE1B4300140040802A00240044025813
:100E600000E100E007000100082B0024881900249D
:100E7000014BD860704700BF50400058012008B5B2
:100E8000FFF7F6FF72B656F017FB00BF03689B0A28
:100E9000A3F58013522B00D970470D4A70B5D45C6E
:100EA00084B00D2C12D800294FF0000309494FF0EF
:100EB000010514BF1E460226427901EB84106946E3
:100EC000CDE90065CDE9023311F070FB04B070BDCF
:100ED00048C30908243E00240D4B4FF6FF71D3F898
:100EE000F82010B50446520856F0F4F900212046C7
:100EF000FFF7CCFF0749084A41F27C132046CA504D
:100F000001F58B5100221C31BDE8104056F088B825
:100F10000000002488190024B5B405084309012203
:100F200000F01F008AB0023B02FA00F0082B11D833
:100F3000DFE803F0665A4E42362A1E120500364B91
:100F4000D3F8F4200243C3F8F420D3F8F42010407F
:100F50000190019B0AB070472F4BD3F8E020024369
:100F6000C3F8E020D3F8E02010400590059BF1E79E
:100F7000294BD3F8E4200243C3F8E420D3F8E4205B
:100F800010400290029BE5E7234BD3F8D4200243A4
:100F9000C3F8D420D3F8D42010400690069BD9E79C
:100FA0001D4BD3F8DC200243C3F8DC20D3F8DC204F
:100FB00010400890089BCDE7174BD3F8D820024388
:100FC000C3F8D820D3F8D82010400990099BC1E776
:100FD000114BD3F8EC200243C3F8EC20D3F8EC20FB
:100FE00010400390039BB5E70B4BD3F8E820024376
:100FF000C3F8E820D3F8E82010400490049BA9E748
:10100000054BD3F8F0200243C3F8F020D3F8F020CA
:1010100010400790079B9DE7004402582DE9F04FD0
:10102000DFF8DC802A4D44462DED068B8DB0CDE9EE
:101030000A0104920FCD0FC40FCD0FC4254B95E8C4
:10104000070093F86E3684E80700042B00F2A981AC
:10105000DFE813F0D801A701A2010500E6019FED2A
:101060001E8ADFED1E9A1E4A1E4B04981E49002858
:1010700018BF13461D4AC8E9062139EE887ADFED0C
:101080001C7AF5EE006ADFF87CB04FF0000928EE1C
:10109000278AB0EE679ADA4686EE87AAC8F8243027
:1010A000DFED148ACB46144B05930B9B5B4500F098
:1010B0006D81059A0BF1010312F8017BDEB20693F4
:1010C0000592002F00F0D88100230C4820E000BFDB
:1010D0009CC30908783B0024ACC5A737ACC5A7362C
:1010E0003DE60708651B07089D1F070849E6070836
:1010F0006F12833A00007A44EB410024004200243E
:1011000014000020480000200133152B00F0B481AA
:1011100003EB43024FEA4309815CB942F4D1C74B68
:101120001A4492F88916002900F0AE8138463FF043
:1011300011F9046805460390204656F04DF9697987
:101140003FF046F902780892002A40F095813D0967
:10115000BA4B07F00F02013D4B444FF00309062D37
:1011600083F8C96683F8C89600F24381B44B0293B2
:1011700003EB4503B3F8800040FA02F313F00103D8
:1011800000F03D810124AF4F04FA02F3013B184007
:101190005AF0E0F9029BAC4A1D4495F890100144C6
:1011A000039807EBC105EE7185F8069057F83130CA
:1011B000CAF814501A44029B007A920A079003EB73
:1011C0004202B2F89800FFF7A9FEAE8857F8311036
:1011D000002E39D0089BA646CDE908BADDF81CA040
:1011E0000EFA03F52E4229D0DC0803F007024FF077
:1011F0000F0C580001EB84044FF0020B9200276A99
:101200000CFA02FC0AFA02F227EA0C0C09FA00F7BF
:101210000BFA00F042EA0C0222620A6822EA070294
:10122000104308608A6822EA07028A604A6822EA54
:1012300005054D60CA6822EA0707CF60013336FA18
:1012400003F2CDD1DDE908BA039B1C68049B002B97
:1012500000F0BD80794BB3F86C3607EE903AF8EEAB
:10126000E77AFCEEE77A17EE905A784B9C420FD063
:1012700003F580639C420BD0754A03F580439C4282
:1012800018BF944204D003F580639C4240F0AA80CA
:1012900011F0D6FD6F4BD969C1F302216D4A4FF6AB
:1012A000FF731269C2F3C03241EAC201029A0A44D2
:1012B000049992F8AC2000FB02F0B0FBF5F21A445E
:1012C000120CB0FBF2F2002970D05C49B2FBF5F5CC
:1012D00091F86E16ABB204296ED007EE902AF8EEA4
:1012E000676A66EE887A28EEE77A544991F86F06C5
:1012F000A6EEA97A0A990190504600910399CAED89
:10130000027A8AED037A37F0ABFBBBF1000F65DDA3
:10131000DAF80430D8F83820934261D0BBF1010FDD
:101320005CD0D8F8502093425AD0BBF1020F55D070
:10133000D8F86820934253D0BBF1030F4ED0D8F8B1
:10134000802093424CD0BBF1040F47D0D8F89820AE
:10135000934245D0BBF1050F40D0D8F8B02093425E
:101360003ED0BBF1060F39D0D8F8C820D31A18BF29
:101370000123DDF818B001228AF810300AF1180AAA
:10138000BBF1080F0AF8072C7FF48FAE32480DB07E
:10139000BDEC068BBDE8F08F9FED308AF0EE489AE9
:1013A00061E69FED2F8AF0EE489A5CE623491D46E0
:1013B00091F86E16042990D107EE905A07EE102A84
:1013C000F8EE677AF8EE476A67EE897A8BE7FAFEFD
:1013D0004A7AFCEEE77A17EE905A46E70123C8E70F
:1013E0000023C6E711F044FD1A4BD969C1F302117D
:1013F00054E7089BCAF81430114B029326E7CAF849
:10140000143023E70023174A01219FED178A0A931E
:10141000164BF0EE489A0491C8E90632144B2CE6BC
:101420000023104A01219FED138A0A930F4BF0EE1F
:10143000489A0491C8E906320D4B1EE6783B002419
:1014400048C309086C4200240000FEA700000140C8
:101450000040014000440258140000202829303880
:101460006F1203399D1F07086F12833A49E6070878
:101470003DE6070800000000044A0020044BC8F8BD
:101480001C20C8F8243082E70B68FFDE511E0708D5
:101490003DE60708002850D0284A2DE9F84F0446B9
:1014A000274B006803449B0A02EB4303B3F8980000
:1014B000FFF734FDB4F804C02268BCF1000F3AD045
:1014C00000204FF0010B4FF00F0A4FF0030900F01E
:1014D00007030BFA00F645004FF0020EC7081CEA9E
:1014E000060F4FEA830309FA05F402EB87070EFAA9
:1014F00005F500F101000AFA03FE01FA03F317D023
:10150000D7F8208028EA0E0E43EA0E033B621368E8
:1015100023EA04032B431360956825EA04059560CC
:10152000536823EA06035360D36823EA0403D360B5
:101530003CFA00F3CBD1BDE8F88F704748C30908E7
:101540000000FEA700284FD0284A2DE9F84F044696
:10155000274B006803449B0A02EB4303B3F898004F
:10156000FFF7DCFCB4F804C02268BCF1000F39D0EE
:1015700000204FF0010B4FF00F0A4FF0030900F06D
:1015800007030BFA00F645004FF0020EC7081CEAED
:10159000060F4FEA830309FA05F402EB87070EFAF8
:1015A00005F500F101000AFA03FE01FA03F316D073
:1015B000D7F8208028EA0E0E43EA0E033B62136838
:1015C00023EA04032B431360956825439560536811
:1015D00023EA06035360D36823EA0403D3603CFA8A
:1015E00000F3CCD1BDE8F88F704700BF48C30908AD
:1015F0000000FEA700487047CC42002470B4204D84
:1016000006460468E36931EA030323D0D5F8743A47
:101610009B1AB3F1007F23681FD25807F2D5E36904
:101620001B05EFD54FF40062202300210320226226
:10163000226822F4D0722260A26822F00102A26025
:10164000C6F8803086F87C10C6F88430C6F888303A
:1016500070BC7047002070BC704723F4D073202208
:10166000002103202360A36823F00103A360C6F8D0
:10167000802086F87C10C6F8842070BC704700BFBC
:10168000783B0024F8B5044690F88000012800F06B
:10169000AB80B94E01272068D6F874CA94F88150FF
:1016A00084F88070012D5FFA85FE67680BD0B7F56E
:1016B000800F40F08F80A568002D40F08B80BEF138
:1016C000040F40F08780002B18BF002A00F08780AD
:1016D000002900F0848094F88150042D02D0052563
:1016E00084F881504FF0000E6266A44DB7F5800F6C
:1016F000C4F884E0A4F86A30A4F862304268A4F820
:10170000683005EA0205E165A4F8603045EA0305A2
:10171000C4E91CEE4560026842F00102026003D198
:10172000026842F400720260E2680F2A60D91A4629
:1017300048F20807416989070ED56BB1E16D51F890
:10174000043B0362B4F86230E165013B9BB2A4F84C
:101750006230B4F862309BB2416943EA0205394213
:10176000ADB211D0002A41D0056BB4F86A20616E89
:10177000013A41F8045B92B26166A4F86A20B4F8B9
:101780006A2092B242EA0305002DD3D1D6F8743A0A
:10179000A3EB0C03092B70D843691B070BD4D6F8B5
:1017A000743AA3EB0C03092BF6D9D4F8843043F038
:1017B0002003C4F8843020460CF0D8FA012200231C
:1017C00084F88120D4F8840084F88030C01A18BFCF
:1017D0000120F8BD0023022084F88030F8BD0023EA
:1017E000012084F88030F8BD0220F8BD1D46CBE70B
:1017F000072A52D8024619465569AD0715D5A3B137
:10180000032B40F2CC80E36B402B40F2DD80E56D92
:1018100055F8043B1362B4F86230E565043B9BB2B3
:10182000A4F86230B4F862309BB2556915F4604F89
:1018300012D089B15169090440F18980156BB4F85F
:101840006A20616E043A41F8045B92B26166A4F8C2
:101850006A20B4F86A1089B2D6F8742AA2EB0C0296
:10186000092A54D843EA010292B2002A00F0C78044
:1018700022685569AD07D8D5C1E720460CF076FA45
:10188000D4F88430012284F8805043F480731046E9
:10189000C4F8843084F88120F8BD19464269920763
:1018A00013D593B1012B43D9E36B002B40D0E26DEC
:1018B00052F8043B0362B4F86230E265023B9BB22B
:1018C000A4F86230B4F862309BB2426912F4604FFF
:1018D00011D081B14269170452D5056BB4F86A2062
:1018E000616E023A41F8045B92B26166A4F86A2024
:1018F000B4F86A1089B2D6F8742AA2EB0C02092A4D
:1019000005D843EA010292B2002AC7D144E7204633
:101910000CF02CFAD4F884300122002143F48073B7
:10192000104684F88010C4F8843084F88120F8BD13
:10193000E26D32F8023B0384B4F86230E265013BA9
:101940009BB2A4F86230B4F862309BB2BDE7516933
:1019500001F4C041B1F5005F47D9028E616E21F8F4
:10196000022BB4F86A206166023A92B2A4F86A20A7
:10197000B4F86A1089B26FE7783B00240000FFFFDB
:10198000028E616E21F8022BB4F86A206166013A7A
:1019900092B2A4F86A20B4F86A1089B2ABE7012BBE
:1019A00011D1E36D1B7882F82030B4F86230E56D18
:1019B000013B226801359BB2E565A4F86230B4F8BA
:1019C00062309BB231E7E36B002BEAD0E56D35F86E
:1019D000023B0384B4F86230E565023B9BB2A4F895
:1019E0006230B4F862309BB21FE792F83010626E3A
:1019F0001170B4F86A20616E013A013125E7206860
:101A0000CAE600BF034690F83C00012800F0AF8111
:101A10000220F0B5012483F83D0083F83C40142AED
:101A200054D8DFE812F05B005300530053009E00CF
:101A30005300530053006701530053005300DE006E
:101A40005300530053001D01530053005300150071
:101A50001A68D1F808C0156A0F6825F480159F4EE2
:101A60001562B242106AD2F804E0546D20F40010FE
:101A700024F4E04440EA0C5044EA07240ED0984D88
:101A8000AA420BD006F5804605F58045AA4218BF4C
:101A9000B24203D005F58065AA4204D12EF4003E7F
:101AA0004D694EEA852E4D68C2F804E05465D5654F
:101AB0001062506D0C6940F400605065506D20F468
:101AC00080605065516D41EA042151650022012179
:101AD000104683F83D1083F83C20F0BD1A688E68EC
:101AE000156A0F6825F001057E4C1562106A55686D
:101AF00020F00200D2F818C03043784E0CEA0404FB
:101B0000B24244EA07040ED006F58066B2420AD01B
:101B1000754F06F58046B24218BFBA4203D006F5AB
:101B20008066B2420BD1CE6820F008008F6925F4A0
:101B3000407530434E693E4320F0040035434E6803
:101B4000556094615663106290690C6940F008001A
:101B50009061906920F00400906191692143916146
:101B6000B4E71A688E68156A0F6825F010055F489B
:101B70001562146AD2F804C024F02004956944EA7E
:101B80000614564E2840B24240EA072000F0F18089
:101B9000534DAA4200F0ED80534E554DAA4218BF56
:101BA000B24203D005F58065AA4206D14E692CF4F5
:101BB000406C8D6935434CEA850C4E68C2F804C010
:101BC00090619663146290690C6940F400609061C2
:101BD000906920F480609061916941EA04219161EB
:101BE00074E71A68D1F808C0156A0F6825F48055A3
:101BF0003A4E1562B242106AD2F804E0D46920F479
:101C0000005024F4E64440EA0C3044EA07240ED0A5
:101C1000334DAA420BD006F5804605F58045AA4211
:101C200018BFB24203D005F58065AA4204D12EF454
:101C3000804E4D694EEA851E4D68C2F804E0D461BD
:101C400015641062D0690C6940F40060D061D069FD
:101C500020F48060D061D16941EA0421D16135E787
:101C60001A68D1F808C0156A0F6825F480351B4E34
:101C70001562B242106AD2F804E0546D20F40030CC
:101C800024F0700440EA0C4044EA07040ED0144DDE
:101C9000AA420BD006F5804605F58045AA4218BF3A
:101CA000B24203D005F58065AA4204D12EF4803EED
:101CB0004D694EEA052E4D68C2F804E054659565FD
:101CC0001062506D0C6940F008005065506D20F0B6
:101CD00004005065516D21435165F7E60000014055
:101CE000000401408CFFFEFF00400140FF8CFFFE1E
:101CF000004401401A68D1F808C0156A0F6825F43D
:101D00008075244E1562B242146A5568D06924F475
:101D1000007420F0730044EA0C2440EA070030D03D
:101D200006F58066B2422CD01B4F1C4EB24218BF43
:101D3000BA4203D006F58066B24206D125F4405778
:101D40004E698D69354347EA05154E685560D06187
:101D5000D6631462D0690C6940F00800D061D06984
:101D600020F00400D061D1692143D161AEE60220A8
:101D7000704724F08004CE6844EA061424F040043E
:101D800014E724F40064CE6844EA062424F4806452
:101D9000D4E700BF00000140004001400044014082
:101DA0002DE9F04FDFF89CB18BB0482200210BF6F3
:101DB000782058F061FB0BF52C604FF431725349D9
:101DC00058F0E0F99BF8843D1BB19BF8853D8BF8FA
:101DD000783A9BF8863D1BB19BF8873D8BF89C3A7F
:101DE0009BF88A3D1BB19BF88B3D8BF8903A9BF892
:101DF000883D1BB19BF8893D8BF8843A444B002603
:101E0000444A1B8812881B09434C4449C3EB1210F7
:101E10002288CBF89C3D1309414F424D424CCBF8F0
:101E2000983D91FBF0F1CBF8A01D03E001360C3793
:101E3000062E27D0042E00F0A081052E00F0C281CE
:101E400038780028F2D0394A002301331E2BEDD018
:101E500012F80C1F8842F8D103EB430C34480022DF
:101E600004EB8C0C0168EC3029B19CF88113114112
:101E7000C90700F1E1840132032AF3D101360C379E
:101E8000062ED7D12B4C0025DFF8BC90DFF8BC80A4
:101E9000294FDFF8BCA0294E54F8083C002B00F075
:101EA0000A81D4F8E020002A00F00581EC222360AA
:101EB00002FB05B2D2F81C1B41F00201C2F81C1B48
:101EC00099689A6801F0040102F008020A43DA688E
:101ED0004AD0920105D5A18A40F20112914200F048
:101EE000E5829A68510700F1CF829A68120708D5F7
:101EF0009A68910705D49968114A0A4042F0200275
:101F00009A600C21DBF8740A2AE000BF04C40908B7
:101F100020E8F11F40E8F11F60E8F11F8038010060
:101F2000F0450024000084CB48C30908C8C609084E
:101F30003846002440460024200882E00021024068
:101F4000C0FFFF7F783B00241CF800FC300882E0D3
:101F5000E03000FEDBF8742A121A052A00F25284DF
:101F60009A680A42F6D1DA6842F400122046DA6032
:101F70000BF010F8002800F06882236840F2FF7C24
:101F80009B490022D3F804E00EEA0101DFF878E271
:101F90005960C3F800C09968DFF870C221F0A04111
:101FA0009960996841F000519960D96801F08021E9
:101FB000D960D96841F00041D960196901EA090185
:101FC0001961596901F040415961996901F07841FD
:101FD0009961196A01F07C411962596A01F07C41EA
:101FE0005962D3F8B01001F07C41C3F8B010D3F8B7
:101FF000B41001F07C41C3F8B410D3F8B81001F06C
:102000007C41C3F8B810D3F8BC1001F07C41C3F890
:10201000BC10196B01EA08011963596B3940596307
:10202000996B39409963D96B01EA0E0E7149C3F877
:102030003CE08B42D3F860E01A66D3F864E05A665D
:10204000D3F868E09A66D3F86CE0DA66D3F8A0209B
:1020500002EA0C02C3F8A020D3F8A42002EA0C0282
:10206000C3F8A420D3F8C02002EA0C02C3F8C020B1
:10207000D3F8C42002F0F822C3F8C42000F06B812A
:10208000B34200F068815C4B9B68DB0704D45B4B78
:102090009A6802EA0A029A60EC22002302FB05B267
:1020A000C2F8203BC4E91733C2F81C3B84F8503017
:1020B000002840F04F810135EC34032D7FF4ECAE65
:1020C0004FF00009DFF848814F46454655F86C3C13
:1020D0001BB1EB6F002B40F049810137EC35032F2A
:1020E000F4D14FF00008464DDFF828914646DFF85E
:1020F00028A12B68002B00F02581D5F8E820002AC4
:1021000000F02081AC683B4B9C4200F02D814C4597
:1021100000F02A8139488368A16849072CD495F8D2
:102120005810012928D003F01F030121092B85F83D
:10213000581000F2B48140F22121D940CF0740F17C
:10214000AE81A16811F001017CD1D4F808C02D4FF7
:102150001CEA070F3DD0EC2303FB06B6D6F81C3B68
:1021600086F8181B43F01003C6F81C3BD6F8203B3A
:1021700043F00103C6F8203BFEE702214FF4002C98
:10218000AE460A46EC2007237970012100FB02B21B
:102190003878BB72D2F8A83BC7F804E043EA0C03D6
:1021A0007972C2F8A83B00283FF440AE42F018FA1A
:1021B000F31DDBB210B100228371C27103213EF026
:1021C000E5F933E602214FF4802CDFF850E00A46AF
:1021D000D8E7A16801EA0A0141F00101A160DBF83A
:1021E000747A8168C8062AD04C4528D12AE000BFFD
:1021F00000F8FFFF00200240006002580063025810
:10220000384600243F00008020F8FFFF0000F0FF68
:10221000A446002400210240C0FFFF7F0000B8CF89
:10222000A168C90705D4A16801EA0A0141F00101CA
:10223000A160DBF8741AC91B022900F243842168EB
:10224000C807EDD5EC20AF494C4500FB06B0D0F8EF
:102250001C7B01EA070141F48071C0F81C1B00D10E
:1022600043B9EC2303FB06B3D3F81C1B21F4801104
:10227000C3F81C1BEC2303FB06B3D3F81C1B11F49F
:10228000805140F04B83C3F8201B5308686D9708BA
:10229000DFF89CC203F07733D10807F03337C0F87A
:1022A0003CC0DFF890C201F011313B44964FC0F8BA
:1022B00040C04FF01C0CD31AC764C4F800C05B1AAE
:1022C0006268002142F0100203EB131385F85810E6
:1022D00004F14001626003F00F33FF22E768B3FBB3
:1022E000F2FC27F003076A6BCCEB0C2C1743874AF0
:1022F000A3EB0C0302EB4802E76009F0B7FFAA6802
:10230000936803EA0A0343F004039360002840F053
:10231000CD83D5F8E8305A08980802F07732D9080A
:1023200000F0333001F0113102449B1AFF225B1A96
:1023300003EB131303F00F33B3FBF2F2C2EB0222F1
:102340009B1A98440136EC35032E7FF4D2AE0BB0C5
:10235000BDE8F08FFEE76E4B9B68B2681343DA0767
:102360003FF59AAE6B4B93E66A48D4E635F8680CB5
:102370000426FEF7D3FDEB6FFF2245F8546C590895
:102380009C0801F07731D80804F0333400F01130A4
:10239000214403245B1AEC211B1A55F86C0C01FB39
:1023A00007B103EB131345F8640C4FF4403003F00E
:1023B0000F3345F8600C0820B3FBF2F2C2EB0222A7
:1023C00045F85C0C01209B1A002245F8580C45F892
:1023D0004C3C4FF4805305F84F0C45F8440C05F87D
:1023E000502C05F8482C05F82C2C049245E91022B5
:1023F00045E90E43D1F81C3B002B00F0188255F83C
:10240000646CB3689C0003D5B268434B1340B3605F
:10241000B36813F0805F414B1ED00193B368D800BE
:102420005FD50024B368590740F18680EC2303FB95
:1024300007B3D3F81C3BEC2303FB07B3D3F81C2BE7
:1024400042F01002C3F81C2BFEE7EC23012203FB31
:1024500005B3C3F81C2B90E5B1681A460193304BC5
:10246000D2F8F8200B402F49B2FBF1F243F0805331
:10247000B3600492049B002BD0D0049B013B0493D7
:10248000049B002BF9D1C9E79A6891073FF52DAD60
:102490009968254A0A4042F010029A6025E5EC222C
:1024A000002302FB06B686F8183B65E61A6850065C
:1024B00007D41E4A02E0013A00F0A48119684906D7
:1024C000F9D540221A609A68500708D59A68900793
:1024D00005D49968144A0A4042F010029A60042117
:1024E00010E5EC23012403FB07B3D3F81C2B42F0C7
:1024F0001002C3F81C2BD3F8202B2243C3F8202B47
:1025000090E700BFFEF0FFFFFD99040800000030D7
:102510000020024000230240C0FFFF5F00000024B3
:10252000C0FFFF6F400D0300C0FFFF7F00DC0C0009
:10253000159A0408119A0408EC2303FB07B3D3F897
:102540001C2BD2063FF577AFD3F81C2B22F48172F7
:1025500042F00202C3F81C2BB368DA0714D4BD4B57
:102560009E4200F0A58203F580739E4200F0A08297
:10257000B94B9B68D80707D4B8498B6855F8602CCD
:1025800023F47C1313438B60B54A41F203031268B2
:10259000B3EB124F55F85C2CC0F0C78155F8343CB2
:1025A00015F84F0C134315F8481C43EA403343EA2F
:1025B0000143012904D155F8442C013A43EA42432E
:1025C00055F8402C2AB102F4787255F83C1C0A43A5
:1025D0001343F168A34A0A401343F360B068B36839
:1025E00000F0040003F00803184300F0478155F899
:1025F000643C55F8582C012A00F0B8821A6B22F07E
:102600000F021A63EC2606FB07B6D6F81C3B06F64B
:102610001C3A23F0030343F00103C6F81C3B002CD3
:1026200040F00D8215F8143C0594012B00F0A281B6
:10263000A5F1640318460393012305F8143C0AF03E
:10264000A9FC002840F0E281D6F81C1B864A874B83
:102650000A40874942F00202C6F81C2B55F8642C48
:102660009068034043F0004393609368002BC0F2EE
:102670006C81EC220020DFF800C202FB07B20146A9
:102680000090D2F81C3B23F0030343F00103C2F88F
:102690001C3B05F8140C07E0009B0CF10C0C0133FB
:1026A000062B009300F067819CF80930002BF3D0D3
:1026B0009CF90130BB42EFD16E4B00224E1C8CF8CE
:1026C000089003EB810015F8143C09F10101069212
:1026D000012BD0F8E844DCF80420029100F0AE8130
:1026E00055F8643C0120996805F8140C490700F17D
:1026F0009681C2F31308B8F1000F40F0A181C2F334
:10270000846E910E00FA0EF0D3F81CA04FEA9419D3
:1027100003F1300E04F01F044AEA000A09F00C002D
:102720004FF01F09C3F81CA001EA090150F80EA0E0
:1027300009FA04F9A1402AEA090949EA010140F825
:102740000E109868996800F0040001F00801014338
:1027500045D1D10DC2F3045A03F114044FF0070917
:1027600001F004014FF0060E09FA0AF908590EFAB1
:102770000AFEDFF8ECA020EA090040EA0E0008514A
:10278000DAF8001001F07041B1F1805FD96800D033
:10279000D968196E900601F0F841B1EB826F03D150
:1027A000196E21F000411966596E01F0F841884216
:1027B00003D1596E21F000415966996E01F0F8413C
:1027C000884203D1996E21F000419966D96E01F0DB
:1027D000F841884203D1D96E21F00041D966996849
:1027E000C80708D4D3F8C010002A21EA0801C3F8AA
:1027F000C010C0F22F8100233146DDF8089005F8A3
:10280000143C49E7EC22012002FB05B2D2F81C1B64
:1028100041F01001C2F81C1BD2F8201B0143C2F882
:10282000201BDA6842F40012DA60FFF7A6BBC1F899
:10283000203B05F8143CE2E50C204FF0010C51B2AE
:1028400000FB034393F88803D3F884E30CFA00FCFD
:1028500098E400BF00200240006002580063025864
:102860000010005C03C0F0FFFDEEFFFFC0FFFE3F65
:1028700000F8C32548C30908F0450024F368C74A97
:1028800015F8501C1A4055F8383C42EA813215F8C8
:102890002C1C13430129F36000F09C81336923F061
:1028A00001033361326955F8303C22F07042BC4973
:1028B00013438E42336100F06981BA4B9E4200F0AF
:1028C0006581B94B9B6813F4403F14BF012300237B
:1028D000002B00F0B38110F0E3FA55F8603CB3F53B
:1028E000003F00F0A781B3F5403F00F09281B3F5BF
:1028F000803F00F09F81AD4A41F203031268B3EBC1
:10290000124FC0F07C81AA4B984240F2388155F8B2
:10291000643C9A6842F480729A606AE6D3F8201B9D
:1029200021F00601C3F8201BAFE4102A7FF436AE75
:1029300015F8481C15F84F0C0B0455F8342C43EAD5
:102940004033134343F01C0333E6059B01330593E7
:10295000059B8B42FFF489AEEC23002103FB07B3F8
:10296000D3F81C2B83F8181B22F0120242F010023D
:10297000C3F81C2BFEE78F4BFEB202203B443146CE
:1029800093F910203EF082FDD0F8048004464046C2
:102990003EF06CFD019A431E02EB431393F81421A1
:1029A000002A7FF4D4AC0136009983F8156183F8CE
:1029B000141100283FF4CBACD3F8FC004FF4005CBA
:1029C000A3684FF48071AA604FF480666B604FF487
:1029D00000644FF48033EA60774AC5F80080904283
:1029E0000CBFA020A1202E61C5E90713C5E9054C45
:1029F000FEF794FA284609F0E3FD284609F048FF5F
:102A0000039B45F8185CAB63FFF767BBDAF800304F
:102A100086F8184B43F01003CAF80030AAE7EC23FD
:102A200003FB07B3D3F81C2B42F02002C3F81C2B86
:102A3000EC23002203FB07B383F8182BFEE703E522
:102A400092FAA2FEBEFA8EFE910E0EF01F0E00FA52
:102A50000EF059E652498B4248D001F580718B4205
:102A600044D0564950488468896804F0E07EC943E0
:102A700001F001010029D2D051498A4257D0514971
:102A80008A4244D050498A427FF4B5AE64023FF591
:102A9000B2AE4A4A93427FF4AEAE836823F0E0734D
:102AA00043EA0E0343F480038360A4E6FFF764BBAC
:102AB0003B4B3C4A9B6892681343DB073FF564AD90
:102AC00042495AE5EC23002203FB06B6D6F81C3B2C
:102AD00086F8182B43F01003C6F81C3BD6F8203BB1
:102AE00043F00103C6F8203BFFF746BB37498C682B
:102AF0000846A1F5407104F0E07ED1F80890D1F8C5
:102B0000088149EA0801C94301F00101B2E7E20185
:102B10003FF571AE294A93427FF46DAE836823F08E
:102B2000E07343EA0E0343F08073836063E621029F
:102B30003FF561AE214A93427FF45DAE019B82680E
:102B4000D3F8F830224922F0E072B3FBF1F342EA05
:102B50000E0E5A004EF400038360069202E0069BBC
:102B6000013B0693069B002BF9D144E6196B55F8FF
:102B70004C2C21F00F01013A0A431A6342E555F843
:102B8000643C9A6822F480729A6032E50F4B9B682D
:102B900013F4403F14BF0123002399E6FCBFFFFF5D
:102BA0000020024000210240006302580010005C37
:102BB000002D3101FC480024000002400060025852
:102BC000000084CB000052C70000B8CF00230240B1
:102BD000400D030055E9093155F8282C0B43D6F870
:102BE00010C0013A55F81C1C43EA02434E4A0B43FD
:102BF00002EA0C02134343F00103336152E64B4BEC
:102C0000984208D855F8643C9A6822F440729A6059
:102C1000EFE480086FE6464B984242D9454B984214
:102C200055F8643C9A6825D822F4407242F4007248
:102C30009A60DEE41B0CB0FBF3F05CE63E4A936D59
:102C400003F44033B3F5803F5ED0B3F5003F4ED080
:102C5000002B62D055F8603CB3F5101F45D00DD85D
:102C6000B3F5E01F3FD025D9B3F5001F7FF443AE85
:102C7000400940E642F440729A60BAE4B3F5201F7E
:102C800050D0B3F5301F7FF436AE2C4A41F2030327
:102C90001268B3EB124FBFF472AF244BB3EB102F9B
:102CA000B0D255F8643C9A6822F4407242F48072C3
:102CB0009A609EE4B3F5801F07D00BD9B3F5A01F2F
:102CC00003D0B3F5C01F7FF416AE9B0C5B00B0FBC6
:102CD000F3F010E6B3F5002FF7D023F40022B2F59D
:102CE000802FF2D007E6000905E6800903E6D36CE1
:102CF00013F040530FD0B3F1805F0AD0104AB3F104
:102D0000005F08BF1046A5E707A80BF0DBFA09989B
:102D1000A0E70C489EE70C489CE707A80BF07EFB59
:102D2000079897E7C009E6E51EF800FC21BCBE0045
:102D300041787D0181F0FA02004402580010005CE5
:102D400000127A0000093D000090D0032DE9F04107
:102D5000D0F800E00C46DFF8588084B0DEF804506C
:102D60001746DFF850C0194605EA0805DDF8288047
:102D7000064603932C43424644EA0C0CCEF804C0AA
:102D800010F026FC78B931680246039B30468F620A
:102D90008021CDF8008010F04BFC003818BF0120D6
:102DA00004B0BDE8F081012004B0BDE8F08100BFAF
:102DB000009800FC00200181F8B5134F04460D4631
:102DC0000AE09B69DB0602D510F0C2FBD0B9D7F848
:102DD000743A5B1B0A2B08D823682A460A2120462E
:102DE0009E69B606EDD50020F8BD636C2021002257
:102DF00001200B4384F84020636484F8411084F878
:102E00004220F8BD0120F8BD783B00242DE9F041B7
:102E1000D0F800E00C46DFF8588084B0DEF80450AB
:102E20001746DFF850C0194605EA0805DDF8288086
:102E3000064603932C43424644EA0C0CCEF804C0E9
:102E400010F0C6FB78B931680246039B30468F62AA
:102E50004021CDF8008010F0EBFB003818BF0120B6
:102E600004B0BDE8F081012004B0BDE8F08100BFEE
:102E7000009800FC00200180F8B5474E96F8A44D5C
:102E800004EB4403650006EBC30393F8A83D032B52
:102E900077D8DFE803F0492A1F02254406EBC50571
:102EA000D5F8AC3D002B6ED196F8082E944268D030
:102EB000013404F003018A4286F8A41D61D001EBBD
:102EC00041040222184606EBC404C4F8AC3D84F861
:102ED000A82DF8BD2B1906EBC303D3F8AC2D72B1A6
:102EE000013A0020C3F8AC2DF8BD2B1906EBC30343
:102EF000D3F8AC2D002AF3D1022283F8A82D254463
:102F000006EBC50595F8B43D013BDBB285F8B43D51
:102F1000F3B1224B0120D3F8FC2202F2E733B3FBDA
:102F2000F2F3C5F8AC3DF8BD43F070F948B31B4A65
:102F300042F20F732C440121D2F8FC2206EBC404A8
:102F4000134484F8A81DB3FBF2F3C4F8AC3DF8BDFC
:102F5000124B601C0327D5F8B01DD3F8FC22384073
:102F600096F8084E531E85F8A87D001B0B4418BF29
:102F700001209A42B3FBF2F188BF0020C5F8AC1DD6
:102F800030B90120F8BD013B0020C5F8AC3DF8BDCB
:102F90000139C5F8AC1DF8BD783B002400000024C1
:102FA000F8B5364C05460821D4F80C0ED4F8746AEE
:102FB0000AF018FC00B1F8BDD4F8501ED4F80C0E7D
:102FC00009040AF0AFFB0028F5D1D4F80C3E4FF00D
:102FD000FF31082259629A6201301F28FCD9DA6A4F
:102FE0000020274941F2331722F0FF0242F033025A
:102FF000DA6298601846DA68114041F288320F436D
:103000003321DF600AF0F4FA0028D4D1D4F80C2E72
:103010008446074640F22A5104E0D4F8743A9B1BD8
:1030200001331ED0536B0B42536B09D11B03F4D4F5
:103030000028F2D1D2F880700120D2F880C0ECE7ED
:10304000190714D4536B9B070ED4506B10F020005B
:1030500010D19CFA8CF33FBA0A499163C5E9003755
:10306000F8BD4FF00040F8BD02209063F8BD082085
:103070009063F8BD20209063F8BD00BF783B00242A
:10308000C0E0FEFF3A0F001870B5114C41F20D136D
:10309000104D41F28832D4F8501ED4F80C0E0E04B4
:1030A0000D218660C66835402B43C3600AF0A0FA44
:1030B00038B1D4F8402E034600201343C4F8403EF4
:1030C00070BDD4F80C3E5869C0F3432070BD00BFFA
:1030D000783B0024C0E0FEFF134B30B4D3F8B80EA9
:1030E0000025D3F8C02ED3F8BC4E20F01F01C3F842
:1030F000A85E04FB0202521ABFF34F8FAA420DDDF5
:10310000013A01F12003094822F01F021A449342B8
:10311000C0F85C12194603F12003F8D1BFF34F8FBA
:10312000BFF36F8F30BC7047783B002400ED00E0A8
:103130000B4BD3F8A82E3AB1D3F8B02E00210132B0
:10314000C3F8A81EC3F8B02ED3F8AC2E3AB1D3F80A
:10315000B42E00210132C3F8AC1EC3F8B42E704760
:10316000783B002470B5037884B004461646012BE2
:1031700024D0022B1FD1C36841F080051BB19A886F
:10318000196812048A6101230DF10F020DF10E017D
:1031900060688DF80E504EF0FBFA01233246002194
:1031A00060684EF0F5FAE3688BB11A6801209B88DD
:1031B000936104B070BD002004B070BD00920A4657
:1031C000417990F9040052F05BF804B070BD012021
:1031D000F2E700BF38B5C36804461BB198881D6884
:1031E0000004A86163682348834217D0A0F57840A3
:1031F000834223D000F58060834217D000F57840E9
:10320000834232D107231C48FEF73CFAF0B9E36849
:1032100013B11A689B889361012038BD07231748B2
:10322000FEF730FA0028F2D0002210E007231448FD
:10323000FEF728FA0028EAD0022208E00723114806
:10324000FEF720FA0028E2D0012200E003220E4B14
:103250004FF48A7101FB0232B2F8D03E01339BB2C7
:10326000A2F8D03EB2F8D03ED1E707230748FEF7D8
:1032700009FACCE700300140884D00244C4A002474
:10328000744C0024604B0024783B0024384900240F
:103290002DE9F84FCB4C054694F84414D4F84C046F
:1032A000C1F3400141F0C0FB94F84414D4F8480441
:1032B000C94301F0010141F0B7FB002D00F0E780A8
:1032C00005F1FF39C04E4FF01008C04F5FFA89F981
:1032D000BF4DD4F84C3433B11A689B8851690B4206
:1032E00018BF1B049361D4F8483433B11A689B8823
:1032F00051690B4218BF1B049361B4F85434002B7E
:1033000040F0578194F85614D4F8580441F08CFBDF
:10331000FA204FF47A714FF0010C7B68C3F3080375
:10332000002B40F01981EFF31183002B40F0148142
:10333000D6F85C2BD5F808E0D6F85C3B9A42F7D17A
:10334000D4F87C349E45F3D8D4F878A401FB0AF372
:10335000A3EB0E03B3FBFAF301FB02327B68C3F36A
:103360000803002B40F0B680EFF31183002B40F0F0
:10337000B180D6F85C3BD5F808B0D6F85CEB734565
:10338000F7D1D4F87CE4F345F3D8D4F878A401FB62
:103390000AFEAEEB0B0EBEFBFAFE01FB03E39B1A2B
:1033A000B3F57A7FDAD30138B7D1D4F84C3433B1DE
:1033B0001A689B8851690B4218BF1B049361D4F8AB
:1033C000483433B11A689B8851690B4218BF1B04FB
:1033D0009361B4F85434002B40F0DF8094F8561415
:1033E000D4F8580481F0010141F01EFBFA204FF49B
:1033F0007A714FF0010C7B68C3F30803002B40F097
:103400008A80EFF31183002B40F08580D6F85C2B87
:10341000D5F808E0D6F85C3B9A42F7D1D4F87C3472
:103420009E45F3D8D4F878A401FB0AF3A3EB0E036E
:10343000B3FBFAF301FB02327B68C3F3080343BB1F
:10344000EFF311832BBBD6F85C3BD5F808B0D6F868
:103450005CEB7345F7D1D4F87CE4F345F3D8D4F8AA
:1034600078A401FB0AFEAEEB0B0EBEFBFAFE01FBDD
:1034700003E39B1AB3F57A7FDED30138BBD109F1A0
:10348000FF395FFA89F9B9F1FF0F7FF422AFBDE888
:10349000F88FEFF3118A88F31288D5F808B02B68FB
:1034A000DB0303D5C4F874C4D5F808B0D6F85C3B88
:1034B0005FFA8AFAD4F874E48AF31188D4F878A40D
:1034C000734401FB0AFEAEEB0B0EBEFBFAFE01FBE2
:1034D00003E3CEE7EFF3118A88F31288D5F808B03A
:1034E0002B68DB0303D5C4F874C4D5F808B0D6F84C
:1034F0005C3B5FFA8AFAD4F874E48AF31188D4F852
:1035000078A4734401FB0AFEAEEB0B0EBEFBFAFE81
:1035100001FB03E343E7EFF3118E88F31288D5F83C
:1035200008A02B68DA0303D5C4F874C4D5F808A042
:10353000D6F85C3B5FFA8EFED4F874248EF31188C3
:10354000D4F878E41A4401FB0EF3A3EB0A03B3FBAF
:10355000FEF301FB02326FE7EFF3118E88F312885E
:10356000D5F808A02B68DA0303D5C4F874C4D5F8DD
:1035700008A0D6F85C3B5FFA8EFED4F874248EF374
:103580001188D4F878E41A4401FB0EF3A3EB0A0384
:10359000B3FBFEF301FB0232E0E6D4F87034002BFB
:1035A0003FF424AF0023D4F85C24136084F86D3416
:1035B0001CE7D4F87034002B3FF4AAAE3DF056FD62
:1035C000A6E600BF704C0024802A002400ED00E035
:1035D00010E000E02DE9F04FCA4C83B00523CA4E3D
:1035E00094F844144FF01009D4F84C04C1F340018E
:1035F000019341F019FA94F84414D4F84804C943EB
:10360000DFF80C83C14D01F0010141F00DFAD4F84F
:103610004C3433B11A689B8851690B4218BF1B04A4
:103620009361D4F8483433B11A689B8851690B42CE
:1036300018BF1B049361B4F85434002B40F0598137
:1036400094F85614D4F8580441F0EEF932204FF4AF
:103650007A710127D8F80430C3F30803002B40F037
:103660001B81EFF31183002B40F01681D6F85C2B01
:10367000D5F808E0D6F85C3B9A42F7D1D4F87C3410
:103680009E45F3D8D4F878A401FB0AF3A3EB0E030C
:10369000B3FBFAF301FB0232D8F80430C3F308039A
:1036A000002B40F0B780EFF31183002B40F0B28085
:1036B000D6F85C3BD5F808B0D6F85CEB7345F7D18B
:1036C000D4F87CE4F345F3D8D4F878A401FB0AFEDF
:1036D000AEEB0B0EBEFBFAFE01FB03E39B1AB3F548
:1036E0007A7FD9D30138B5D1D4F84C3433B11A68C4
:1036F0009B8851690B4218BF1B049361D4F848346E
:1037000033B11A689B8851690B4218BF1B0493613F
:10371000B4F85434002B40F0E08094F85614D4F8F8
:10372000580481F0010141F07FF932204FF47A71A1
:103730000127D8F80430C3F30803002B40F08B8036
:10374000EFF31183002B40F08680D6F85C2BD5F880
:1037500008E0D6F85C3B9A42F7D1D4F87C349E4519
:10376000F3D8D4F878A401FB0AF3A3EB0E03B3FB60
:10377000FAF301FB0232D8F80430C3F3080343BB69
:10378000EFF311832BBBD6F85C3BD5F808B0D6F825
:103790005CEB7345F7D1D4F87CE4F345F3D8D4F867
:1037A00078A401FB0AFEAEEB0B0EBEFBFAFE01FB9A
:1037B00003E39B1AB3F57A7FDDD30138B9D1019BBE
:1037C0005F1E17F0FF0301937FF421AF03B0BDE844
:1037D000F08FEFF3118A89F31288D5F808B02B68BF
:1037E000DB0303D5C4F87474D5F808B0D6F85C3B95
:1037F0005FFA8AFAD4F874E48AF31188D4F878A4CA
:10380000734401FB0AFEAEEB0B0EBEFBFAFE01FB9E
:1038100003E3CEE7EFF3118A89F31288D5F808B0F5
:103820002B68DB0303D5C4F87474D5F808B0D6F858
:103830005C3B5FFA8AFAD4F874E48AF31188D4F80E
:1038400078A4734401FB0AFEAEEB0B0EBEFBFAFE3E
:1038500001FB03E342E7EFF3118E89F31288D5F8F9
:1038600008A02B68DA0303D5C4F87474D5F808A04F
:10387000D6F85C3B5FFA8EFED4F874248EF3118880
:10388000D4F878E41A4401FB0EF3A3EB0A03B3FB6C
:10389000FEF301FB02326EE7EFF3118E89F312881B
:1038A000D5F808A02B68DA0303D5C4F87474D5F8EA
:1038B00008A0D6F85C3B5FFA8EFED4F874248EF331
:1038C0001188D4F878E41A4401FB0EF3A3EB0A0341
:1038D000B3FBFEF301FB0232DEE6D4F87034002BBA
:1038E0003FF423AF0023D4F85C24136084F86D34D4
:1038F0001BE7D4F87034002B3FF4A8AE3DF0B6FBC4
:10390000A4E600BF704C0024802A002410E000E0F0
:1039100000ED00E010B4B8B10D4CD4F88034102B99
:1039200005D1052100205DF8044B3DF075B803EB8F
:103930004302224482F88514012182F884040B4456
:1039400082F88614C4F880345DF8044B704700BFD9
:10395000704C002430B5044683B00D4608480DF184
:1039600007022146FFF7FEFB9DF8072035EA020318
:1039700004D02A432146024842F0CCFB03B030BDBC
:10398000245100240378012B01D00020704790F9C6
:103990000420084902EB420201EB421292F84D1555
:1039A000202901D018467047D2F80C359869C0F329
:1039B000C0307047704C00242DE9F0411F4C84B09A
:1039C0000746884694F8B4541646022D11D0012DAE
:1039D0000BD113460091024694F8B91494F9B80437
:1039E00051F04EFC04B0BDE8F081002004B0BDE809
:1039F000F081D4F8C0341BB19A88196812048A6126
:103A000001230DF10F020DF10E01D4F8B8048DF869
:103A10000E704DF0BDFE334642460021D4F8B80486
:103A20004DF0B6FED4F8C03433B11A6801209B883B
:103A3000936104B0BDE8F0810120D3E7704C00240D
:103A40002DE9F04F037885B004460E46022B00F0B6
:103A50008E80012B04D00025284605B0BDE8F08FEC
:103A600090F904105C4F042987F87836D4BF0025FC
:103A70000125B1F1FF3F08BF45F00105002DEAD156
:103A800001EB4102480007EB4212D2F80CC5BCF131
:103A9000000FE0D092F84DE5BEF1200FDBD1DCF84D
:103AA000188018F40048D6D192F84CC5BCF1010F2B
:103AB000D1D04FF0400CDFF838E14FF0210BDFF8A8
:103AC000349194F805A0DEF874EA82F84DB582F8D6
:103AD0004EC507F5CF6CC2F85085A2F83635C2F84E
:103AE0003895B2F8364582F84C35A3B23B4CC2F853
:103AF00030C5FF2BC2F8404569D8B2F836C54FF043
:103B000000791FFA8CFC441835484FEA4A0ACDF870
:103B100000E000EB4410324607EB441451461430E9
:103B20001923A4F834C5FFF711F9002845D1D4F8BA
:103B30000C252C49536894F834650B402A4DD4F871
:103B4000401543EA0A03A94243EA064343EA09034C
:103B5000536084F84C0504D0244B994218BF4FF0B1
:103B6000F2081368012543EA0803136074E7C36889
:103B70001BB19A88196812048A6101250DF10F02A0
:103B80000DF10E0160682B468DF80E604DF000FEC1
:103B90002B460DF10F020DF10E0160688DF80E50ED
:103BA0004DF0F6FDE368002B3FF456AF1A68284647
:103BB0009B88936105B0BDE8F08FB7F87A36002294
:103BC000013384F84C259BB2A7F87A3644E74FF0CE
:103BD000FF0C4FF0807996E7704C0024753C050887
:103BE00068510024009C00FC193A0508313B050887
:103BF000783B00240000FFFF036870B55E6A26B1C1
:103C000033460522BDE87040184704460D464E1D58
:103C100000E023689B68204698470028F9D0236875
:103C2000204615F8011B1B689847B542F1D170BDBD
:103C30002DE9F0470023194D84B0074695F9819688
:103C400005F5D1664FF0B60A00EB010805F6281518
:103C50001C46D6F800C0304600226946E036BCF16A
:103C6000000F14D09CF838C0BCF1140F0FD019F11C
:103C7000020F01D0CC450AD1CDE90244CDE900784C
:103C8000ADF808A08DF80E4035F04CFA0346B54269
:103C9000DFD1184604B0BDE8F08700BF704C0024A7
:103CA000F0B500230E680DE0BCF1050F17D9BEF189
:103CB000050F18D80A2C16D103EB830316F8010B55
:103CC00004EB4303A0F13005A0F1610CA0F1410E1B
:103CD000A0F13704EFB2092FE6D82C46ECE7A0F1AB
:103CE00057040A2CE8D00E601360F0BD2DE9F743AD
:103CF000A0230124114E18255FFA84F8FF2B14DC51
:103D0000E9B2D6F828095F1CDBB2C1F11C02C1F18F
:103D10001B0180F80B808272C9B2026800930023F5
:103D2000D2F818904246C8473B46013DE6D10134DF
:103D3000052CE0D103B0BDE8F08300BF704C002437
:103D400008B5FCF707FE38B10449054841F05EFDAF
:103D5000034817F0E5FA024808BD00BF70C809081B
:103D60009C5500242DE9F04F884C16460B2287B055
:103D700094F8BA8B054694F8C5AB8946404611467F
:103D800002951D469DF840703CF050FBC2458346AD
:103D900040F0B0800390404640F022FC17F008034A
:103DA0000246019300F09980BBF1000F00F0918072
:103DB0009BF80710890700F18C80C4F884B9C4F817
:103DC0008009C4F87C09002800F0DC8040F60B3143
:103DD00005F0020AC1804FF48073DFF8C8810299B0
:103DE000584608EB030284F844590025C4F86C19BE
:103DF000C4F858293146664AC4F84C39C4F84029F9
:103E0000C4F85039C4F8486984F84579C4F8709901
:103E1000C4F85489C4F86059C4F85C59C4F86859A6
:103E2000C4F86459C4F89C5B84F8A05BA4F8945B64
:103E300034F06AF8D4F8840907F00101FDF726F898
:103E4000544A554BD4F88409C4F8A85BC4F8AC2B89
:103E5000C4F8A43BBAF1000F1CD0D4F88C79CFB1D0
:103E60003A6803689A4215D001233146384684F8EF
:103E7000A13B34F049F808F505722946D4F88C09BD
:103E800053F0CEF82A4608F50771D4F8840953F0A8
:103E9000C7F807E0414A002302F1080184F8A13B7A
:103EA00053F0BEF8D4F88439186853F081FA019BB6
:103EB000C4F888092BB33A4834F04EF8384807B0B4
:103EC000BDE8F08F039BCDE9040113B1D8798307D6
:103ED0001FD5002007B0BDE8F08F15F00101F1D12A
:103EE00005F0020C5FFA8CFABAF1000F2CD1D4F86D
:103EF00084B970E70B220C2150463CF097FA0390EE
:103F000049E7274834F01CF80121254834F04AF8E5
:103F1000D1E7504605F0020A40F062FB039AD4460E
:103F20000599C4F88429049AC4F87C09904202D106
:103F3000BAF1000F1CD10028D4D040F60C3EA0F8F6
:103F400006E0BAF1000FD2D0B8F1000FC1D0C4F82A
:103F5000802991B9BBF1000FBBD0C4F884B95FFAD6
:103F60008CFA002A3FF437AF40F60B31D18032E7AC
:103F7000B8F1000FADD0C4F88029C4F88CB9D4F8DA
:103F800084B9ECE705F0020A25E700BF704C002475
:103F9000C0C80908ED440708BD7F0708145800246D
:103FA000B0550024005600242DE9F04FB6480925ED
:103FB000B64C0023022200F6880665608BB0B44D33
:103FC00094F8BD13C0F8584BC4F80464256023630B
:103FD000636123616362A261E260C4E90733C4E9FB
:103FE0000A33002900F07B811F460321A84B84F887
:103FF000BD13DB6B13F48078AB6818BFD4F8108066
:1040000023F0010308BFC4F81080012AAB6040F020
:10401000DC80AA6B9F4B22F48032616BAA6301297A
:10402000EA6803EA0203EB60EB6823F44013EB60F9
:1040300000F09981284608F035FE0646B8F1010FD8
:1040400016D0FEB10222236884F8BD2394F824051B
:10405000012800F004818021012059625A6A42F44B
:1040600080029A62FCF7B2FA00200BB0BDE8F08F34
:10407000AB6843F00603AB60AB6843F02003AB6072
:10408000002EDFD123683220DA6822F0C042DA60E5
:10409000DA6842F08042DA6009F0AAFD606848B34D
:1040A000324601273146C2EBC203551C04EB8303A1
:1040B00083F83C20A3F84220EAB283F83D708242A4
:1040C00083F83F101965C3E91111ECD300221146A2
:1040D000C2EBC203551C04EB830383F8FC21EAB254
:1040E00083F8FD11824283F8FF11C3F81012C3E96F
:1040F0008111EDD300222368D4F80CC01546D4F802
:104100001080D4F82CE0D4E90671019102F140014D
:10411000013203EB81010F2A4D60F7D1BEF1000F90
:1041200040F01A81D3F8042803F5006542F002023A
:104130006A609A6B22F400129A631A6842F0400295
:104140001A601A6842F080021A600022012FC3F838
:10415000002E2A682A602A6800F0158142F00302C6
:104160002A604FF484614C4A196102E0013A00F080
:10417000128119698F06F9D41021474A196102E0AA
:10418000013A00F00A811969C906F9D400212961B0
:104190006961E96160B303F510624FF0904A4FF036
:1041A000006B0F464FF67F399C4607E017600131E0
:1041B0001761C2F808902032884271D01368002B32
:1041C000F4DA91B1C2F800A0F1E7EB68284643F0B9
:1041D0004003EB6008F066FDAB6B0646002F40F035
:1041E000B78043F48033AB6328E7C2F800B0DEE762
:1041F0002A6900206FF0804122F480722A61986160
:104200005961B8F1000F03D19A6942F010029A6126
:104210009969224A0A439A61019A1AB19A6942F04D
:1042200008029A61BEF1010F00F0A280002E40F05A
:10423000A6800121626A84F838608A4284F8BD133E
:1042400000F0AD806B68032043F002036B6009F05F
:10425000CFFC94F82405236801287FF4FCAE80226B
:1042600040215A625A6A42F400129A62FCF7AEF98F
:1042700020210220FCF7AAF940210320FCF7A6F92F
:1042800000200BB0BDE8F08F802A0024881900249C
:1042900000000840BFFFBDFF400D030000383C8018
:1042A000002163460CF530624FF0904A4FF0006BEE
:1042B0000F464FF67F39844607E0176001311761DA
:1042C000C2F8089020328C4592D010680028F4DAA9
:1042D00011B1C2F800A0F1E7C2F800B0EEE701F0BA
:1042E000FF073A4B03204FF4C05584F8BC73D3F852
:1042F000E01041F00101C3F8E01005A9D3F8E03067
:1043000006920A2203F00103089031480493049BAB
:1043100007970595099208F019FDE36A012B4BD028
:104320002A4B06216520D3F8D82042F00062C3F85A
:10433000D820D3F8D83003F000630393039BFCF735
:10434000FDFC244B2021A2692568D960A76A4CE6B0
:1043500023F48033AB6371E69A6B03F5006542F496
:1043600000129A63F1E6EB6843F48013EB6061E6B8
:104370009969194A0A439A61002E3FF45AAF022202
:1043800084F8BD2362E6BCF1000F3FF4E9AE42F0D1
:1043900001022A60E5E60126EEE60126F6E684F84B
:1043A000F4639969C4F8FC2341F000610B4A9961F8
:1043B000596D0A435A6545E74FF4007305A904484F
:1043C0000593CDE9067708F0C1FCA9E7004402583F
:1043D0000000025800E100E004000040030000106B
:1043E000094B93F86E36042B08D9053B032B08D8EC
:1043F00001231A4600B103701046704700230122C2
:10440000F8E700231A46F5E7783B00242DE9F0474A
:104410009AB004460D4617469846DDF89090DDE9BF
:10442000226A02E020683DF093F820683DF098F899
:104430000028F7D10146642201A856F01DF8264B4A
:104440008DF80450CDF85CA00293002D40D0AB1E37
:10445000012B3FD9042D14BF002303231F4A8DF8DD
:1044600005300123D2F85C2B039616448DF85B309F
:10447000CDE90594049637B14246394607A855F070
:1044800081FE8DF85A80164E002396F8169C1893DC
:10449000B9F1000F19D196F8150C642201A902FB9D
:1044A000006000F6184055F06DFE012386F8159C5B
:1044B00086F8163C236843B143463A4629462046CF
:1044C0001AB0BDE8F04719F07FBC1AB0BDE8F0871C
:1044D0000523C3E70223C1E744580024802A0024AF
:1044E000704C00249FED747A07EE901A20EE070AB4
:1044F000F8EE677A27EE800AFDEEC07A17EE903A62
:104500002033402B00F2C880DFED6C7AB4EEE70A6E
:10451000F0EE407AF1EE10FA0CDD9FED696ADFED06
:10452000696AB0EE677A77EEC67AB4EEE67AF1EEB3
:1045300010FAF6DC9FED647AF4EEC77AF1EE10FA29
:104540000CD59FED5F6ADFED616AB0EE677A77EEBA
:10455000867AB4EEE67AF1EE10FAF6D49FED5C7A44
:10456000F4EEC77AF1EE10FA40F386809FED537AAD
:1045700077EE677A67EEA75A9FED565A9FED566A17
:10458000B6EE007ADFED556AA5EE856A27EEA55AEC
:10459000E5EE866AE5EE267A27EE877ADFED4C6A4D
:1045A00070EE267ABDEEE76A16EE103A2033402B05
:1045B0006FD8B4EEE60AF1EE10FA0CDDDFED405AEA
:1045C0009FED406AF0EE676A77EEE57AF4EEC66A30
:1045D000F1EE10FAF6DCDFED3C6AF4EEE67AF1EE8D
:1045E00010FA0CD5DFED365A9FED386AF0EE676AA7
:1045F00077EEA57AF4EEC66AF1EE10FAF6D4DFEDA6
:10460000346AF4EEE67AF1EE10FA48DDDFED2B6A5B
:1046100076EEE77A67EEA75ADFED2E4A9FED2E6A17
:10462000B8EE005ADFED2D6AA5EEA46A67EEA54A42
:10463000E5EE866AE4EEA67A67EE857AC7EE206A32
:104640000023836143610362B7EE006AC36176EEC3
:10465000865A76EE666A86EE257A67EE277A80EDD0
:10466000007A66EE876A80ED027AC0ED017AC0EDCD
:10467000037AC0ED046A70479FED197AF4EEC77AA9
:10468000F1EE10FA7FF576AF9FED0F7A77EE677A4D
:1046900070E7DFED147AD1E79FED127A7EE7DFED68
:1046A000106AF4EEE67AF1EE10FAB3D5DFED066AA1
:1046B00076EEE77AAEE700BF27D4D236DB0F49406B
:1046C000DB0FC940E4CB1641DB0F49C0E4CB16C178
:1046D000DB0FC93F92E741B99730083C15A82ABEC5
:1046E000DB0FC9BF00000000F0B401282E4C2F4999
:1046F0004CF250372E4D08BF0421D4F8746A0429B7
:1047000011D0D5F8102121EA020212F0040F0CBFDB
:104710000123002363B1D4F8743A9B1BBB42EED94A
:104720000320F0BC70472B69C3F38003002BF2D148
:10473000012810D01E491F48D1F81021024224D16F
:10474000D1F81021D20313D54FF480321846F0BCB3
:10475000C1F814217047164A164C116921420AD13A
:104760001169C90304D54FF4803118465161D8E767
:104770001846F0BC7047104B104C1940D4F8983CC8
:104780000B43C4F8983C5161CBE70C4C01200A4B19
:104790001A40D4F8983C134343F00043C4F8983CC3
:1047A000C1F81421F0BC7047783B0024040000805D
:1047B000002000520000EE150000EE17704C00249F
:1047C000F8B5294E96F8943C012B4AD000F1784375
:1047D000012705460C46B3F5801F86F8947C4FF000
:1047E00000032CD30220C6F8983CFFF77DFF10BBD6
:1047F0001E4A0227D2F80C313B43C2F80C31214645
:10480000BFF36F8FBFF34F8F2A1B20340B688B5081
:104810000431A142FAD1BFF36F8FBFF34F8F3846F7
:10482000FFF762FF012F114A16D0D2F80C3123F0A6
:104830000203C2F80C31002386F8943CF8BD3846D8
:10484000C6F8983CFFF750FF0028F4D1074AD36818
:1048500043F00203D360D2E7D36823F00203D360AE
:10486000E9E70220F8BD00BF704C00240020005290
:104870000C480D4BD0F8B41C10B48A1E0B4C2231DE
:10488000C0F8A43CB0F8CE3C1B01A4FB03C3DB087A
:10489000A3F5B06322F8023F9142F3D15DF8044BD7
:1048A000704700BF704C0024D10A0608CDCCCCCC98
:1048B00070B5084C251D2E4614F8010B34F004FE8B
:1048C00028B10378B44205F8013BF5D170BDFF2350
:1048D000F8E700BF605900242DE9F0471C4F01267E
:1048E0004FF03C094FF0000807F10805B24617F8F1
:1048F000010B3FF075FE044690B180F80690C6713A
:10490000FB7803F07F02012A17D013F0800F2046B6
:104910000CD185F8048040F07BF885F805802C6088
:1049200001360835052EE2D1BDE8F08785F804A0F0
:1049300040F074F885F805A0F1E71B0605D40121C5
:1049400020463BF023FEFB78DFE740F067F8F6E710
:1049500068590024654B2DE9F04F4FF0010985B0EF
:1049600003F10C0ADFF8A0B1984618F8016B002E8D
:1049700000F0B080350906F00F02013D062D00F26F
:10498000AC800BEB4503B3F8800040FA02F414F05E
:10499000010400F0A68001235D44554C9340013B87
:1049A000184056F0D7FD95F890300422184404EBD7
:1049B000C004CAF8144084F80790A271002303E0F1
:1049C0000133152B00F0868003EB430249495D005B
:1049D000895CB142F4D1484B1A4492F889160029F7
:1049E00000F0828030463BF0B5FC0746006852F08C
:1049F000F3FC79793BF0ECFC017800296AD13E4B5D
:104A000004222B4483F8C99683F8C826002C44D08E
:104A100023683A4A387A1A440290920A0BEB42020F
:104A2000B2F89800FCF77AFAB4F804C02268BCF136
:104A3000000F32D00397012303FA01FE1CEA0E0F88
:104A400026D0CC0801F007030F25029F02EB840457
:104A50009B00266A48009D4007FA03F3022726EAD6
:104A6000050603253343854007FA00F023621368E7
:104A700023EA050318431060936823EA0503936053
:104A8000536823EA0E035360D36823EA0505D56013
:104A900001313CFA01F3CED1039F194C09F1010910
:104AA000184A0025B4F8223D5FFA89F9B4F8204D80
:104AB000504639460AF1180AB2FBF3F3CDE9004536
:104AC0009BB233F0CDFF0123B9F1090F0AF8073C7F
:104AD0007FF44BAF05B0BDE8F08F0024CAF8144056
:104AE0006CE7CAF8144069E70B68FFDE94590024AC
:104AF0006C42002400420024783B00240000FEA702
:104B0000704C002440420F0048C309088E4B2DE929
:104B1000F04193F8F02D82B00190002A40F00E8110
:104B200093F8142EB7EE007AB3F8187E012107EE41
:104B3000902AB3F8160EF0EE475ADFED846AB8EE0D
:104B4000E76A07FA01F507EE900AB3F8120E804CF7
:104B5000E6EE665A8542A6EE267AA4F80071F8EED3
:104B6000E77AB8BF054683F8F01DAEB267EEA67AC5
:104B7000A4F80461C4ED3D5A84ED3E7AC4ED3F7A59
:104B8000002A00F0D880DDED017AADB29FED710A08
:104B9000F8EE677A6D0080EE270A53F081F98046BF
:104BA000B0FBF5F5012DB8BF0125EDB2B0FBF5F373
:104BB0009BB284F8085100EE103ABBEEED0A84ED8A
:104BC000430A53F06DF9644A0023DFED646AA2FBE7
:104BD0000828DFED630A9FED636A4FEAD8089FED6E
:104BE000621ADFED625A07EE908A6149DFED611AC1
:104BF000F8EEE77A9FED602ADFED602A9FED603ADC
:104C000086EEA77ADFED5F3AB7FBF0F7022FB8BF69
:104C1000022784F8107184ED457A07EE903AB8EED9
:104C2000E77AF0EE467AE7EE207AFDEEE76A16EED6
:104C3000902A2032402A7BD8B4EEC17AF1EE10FAE5
:104C40000CDDDFED516A9FED517AB0EE675A77EED9
:104C5000E67AB4EEC75AF1EE10FAF6DCF4EEE57A35
:104C6000F1EE10FA0CD5DFED486A9FED497AB0EE0F
:104C7000675A77EEA67AB4EEC75AF1EE10FAF6D478
:104C8000F4EEC67AF1EE10FA4ADD73EEE77A67EEDB
:104C9000A76AB0EE424AB7EE007A67EEE64AA6EEA1
:104CA000A14A77EE677AB0EE627AB6EE005AA6EEC7
:104CB000847AE4EE877A67EE857A0133E1EC017A53
:104CC000202BAAD107EE905AB7EE006A314A102085
:104CD000F8EEE76A07EE906A2F4B02F12806F8EE2D
:104CE000677A202186EE267A84F81956C4F8BC2704
:104CF00002F1A8051422C4F8B867C4F8C857C3ED78
:104D0000AC7AC3EDAD7AC3EDAE7AA4F8B407A4F8DB
:104D1000C417A4F8C02783ED007A02B0BDE8F08183
:104D2000F4EEC37AF1EE10FA48BF75EEE77AAEE71B
:104D3000F6EE007AC1E7194B1A7024E7044C94F898
:104D40000851B4F80461BDE7704C00240AD7233C35
:104D50001400002000247449ABAAAAAADB0FC941A1
:104D60003C8C4F3EDB0FC93F0100F840DB0F49C0D0
:104D70002C01002092E741B99730083C15A82ABEC3
:104D8000DB0FC9BFDB0F4940DB0FC940E4CB164145
:104D9000E4CB16C1F0C8090830060020000000204E
:104DA000F0B5284C83B0B4F8205EA4F85454EDB9A3
:104DB00094F81C0E3FF014FC94F81D2EC4F858040F
:104DC000003A18BF012284F8562448B194F81E1EF8
:104DD0002B220029C28014BF112101213BF0D6FBF8
:104DE000002003B0BDE8F04040F08CBB94F81C7E7E
:104DF00000222B2138463BF019FB064638463FF08F
:104E0000EFFB00B10EB903B0F0BD2B22C4F8700463
:104E10000027C280317AFCF73DFB0B4AA4F8225EE2
:104E2000314604F25C400197B2FBF5F3C3F34F0542
:104E30009BB2009533F014FED4F85C341F6084F804
:104E40006D74E0E7704C002440420F002DE9F84FEC
:104E5000254B002693F8302E03F6276703F64464AB
:104E600083F8242E5FFA86FB4FF0010917F8010F33
:104E700001360BEB090A49464FF000085FFA8AFA3F
:104E800052463BF0D3FA054640B3387804F80E8C0E
:104E900004F80D8C04F80FBC04F8109C44F8045C72
:104EA0003FF09EFB18B180F8069080F807A0297AA1
:104EB000FCF7F0FA0D4A0021284652F00BFA0C4B91
:104EC000221D2146236028460A4BC4E9013852F0CE
:104ED000A7F842466979286833F048F9082E04F1AA
:104EE0001C04BFD1BDE8F88F704C002440420F0075
:104EF000218207084119070870B52C4C00222C4B61
:104F0000022194F85C0FC4F8543FC4F8142FC4F87D
:104F1000182FC4F81C2FC4F8502FA4F8582F3BF0BA
:104F200085FA002840D0234B0546066803F1C001EE
:104F30005A7C12B15A6896422BD018338B42F7D163
:104F4000002394F85C0FC4F8405E84F8343E3FF0D0
:104F500047FB08B10223C380297A0026FCF79AFA9E
:104F60002846154A002152F0B5F9144A1448154B49
:104F7000111FC4F8440E2846C4F8483EC4F84C6ECD
:104F800052F04EF8324669792868BDE8704033F037
:104F9000EDB8304651F046FEB36A0B4A0133B0FB20
:104FA000F3F082F80003CBE770BD00BF704C002423
:104FB00000FFFF004800002040420F00B85A0024C4
:104FC00069190708051B0708000000242DE9F04FA8
:104FD0005D4CC02283B006460D4604F1340000212A
:104FE00055F04AFA594B93F85D2F72B193F85E3F32
:104FF000DBB9574B3046294693F87026003A18BF64
:105000000122FCF70BF8C4F81C09D4F81C39002B5A
:105010007FD00022012183F82C5083F82D101A63D1
:1050200083F82E2003B0BDE8F08F4A4F04F6E8065F
:10503000DFF81C910FCF99F872C60FC60FCFBCF1E5
:10504000000E0FC699F86E3618BF4FF0010E97E8A4
:105050000700072B404F84F820E9C4F8007986E860
:10506000070043D9082B02D13C4BC4F824393C4BF0
:105070000027DFF808A101935FFA87FBBD424FF0DC
:1050800003010BF101082DDD019B5FFA88F813F88D
:10509000016B4246304601933BF0C8F90346304667
:1050A0001E46002B48D03FF09BFACAF8140020B1EE
:1050B0004FF0030380F80780837199F86F3699F8F1
:1050C0006E26002B34D1F3795946304601374FF024
:1050D000F1FA88B34FF00103082F0AF1180A0AF811
:1050E000073CC9D11F4BC4F81C398EE7042BBED92D
:1050F00099F871361C4A012BC4F8242906D0022BDA
:1051000008BFBCF1000F0CBF0123002384F828392D
:10511000ADE7164E164D0FCE0FC50FCE0FC596E854
:105120000700A5F1200385E80700C4F81C3979E7DA
:10513000F37983F00103C7E70E4900230E4AC4F850
:105140000419C4F80C29CEE714000020704C002488
:10515000783B002418CA0908FDFE0808C93300007E
:10516000EB410024FC080020FD33000044CA09087C
:10517000D05B002445E607083DE60708480000200C
:1051800070B5714C94F8C80C3FF02AFA94F8C96CC9
:1051900060B12D2305462021C3803BF0F7F90A209A
:1051A0003BF082FD284640F0E1F918B9D4F8943F6D
:1051B000DA0100D570BD013E092EFBD894F8C75C1A
:1051C000D5B9402035F02CFE0028F3D090F90430FA
:1051D00094F89D1C092BC8BF143B0A29234493F85B
:1051E000B05B00F0A28093F8BB3B94F8C62C002A79
:1051F00008BF1D46002DDDD028463FF0F1F90546D9
:10520000002800F08A802D230121C3803BF0BEF9E5
:10521000012108463FF010FC2B68AA889A613C20C7
:105220003BF05EFE002101203FF006FC94F8C93CF3
:10523000BBB3002694F84414D4F84804C94301F0E1
:1052400001013FF0F1FB94F84414D4F8500481F0CC
:105250000401C1F380013FF0E7FB7820002D38D036
:10526000AB8801362A681B0493613BF01DFD94F85E
:105270004414D4F8480401F001013FF0D5FB94F840
:105280004414D4F85004C1F380013FF0CDFB2B68E7
:10529000AA8878209A613BF007FD94F8C93C9E42A9
:1052A000C8DB94F8C73C83BB94F8C83C002B81D181
:1052B00094F8CA3C012B7FF47DAFD4F8943F13F0EF
:1052C00080737FF477AF84F8C93CBDE8704045F047
:1052D0000DB8782001363BF0E7FC94F84414D4F87C
:1052E000480401F001013FF09FFB94F84414D4F806
:1052F0005004C1F380013FF097FB78203BF0D4FCD1
:1053000094F8C93C9E4295DBCBE732203BF0E8FDA8
:10531000284600213BF03AF9C6E701213BF036F977
:10532000012108463FF088FB79E7D4F8983F5B05F8
:105330007FF540AF11F0AAF900287FF43BAF002DB4
:105340007FF45AAF36E700BF704C00242DE9F041DE
:10535000204C00234FF0050894F89F2F04F69C770B
:1053600004F5896584F8442417F8010B5E1C20BB02
:105370002860032E05F104053346F5D194F8441452
:10538000D4F84804C94301F001013FF04DFB94F803
:105390004414D4F84C0481F00201C1F340013FF001
:1053A00043FB94F84414D4F8500481F00401BDE8A0
:1053B000F041C1F380013FF037BB3FF011F901210B
:1053C000F3B2286010B180F80680C37128683BF002
:1053D000DDF8CEE7704C0024084B03F57A600DC869
:1053E000904202DC114602460846984204DD9A4289
:1053F000B8BF1A4610467047704700BF704C002473
:105400000B6810B414681B1B036054684B681B1BAB
:105410005DF8044B43608B6892689B1A8360704709
:105420002DE9F047041E0D4612DB092C26DC0B4645
:10543000814A82480021A0FB04605970C00800EB3B
:105440008000A4EB4000125C28461A70BDE8F0878B
:1054500064422D23092C01F8013B24D8764A774B6E
:105460000020A3FB046348702846DB0803EB83039A
:10547000A4EB4303D35C0B70BDE8F0876F4B632C48
:10548000A3FB04264FEAD60621DC0B466A4A6B4989
:10549000A1FB0601C90801EB8101A6EB4101515CAA
:1054A00003F8011BC5E7654A632CA2FB04364FEAEB
:1054B000D60637D8604A614BA3FB0603DB0803EB33
:1054C0008303A6EB4303D35C01F8013BC7E7A3FBCF
:1054D0000627B4F57A7F4FEAD7070DD20B46564A16
:1054E0005649A1FB0701C90801EB8101A7EB410166
:1054F000515C03F8011BCAE7A3FB072842F20F72B5
:1055000094424FEAD80836D80B464B4A4B49A1FB88
:105510000801C90801EB8101A8EB4101515C03F8C6
:10552000011BDDE7A2FB0637B4F57A7F4FEAD70708
:105530000CD2414A414BA3FB0703DB0803EB830377
:10554000A7EB4303D35C01F8013BB4E7A2FB0739A7
:1055500042F20F739C424FEAD90921D8364A374BA1
:10556000A3FB0903DB0803EB8303A9EB4303D35C31
:1055700001F8013BDEE7A3FB0829314A94424FEAD8
:10558000D90921D80B462C4A2C49A1FB0901C9088D
:1055900001EB8101A9EB4101515C03F8011BB5E767
:1055A000A2FB093A264B9C424FEADA0A21D8224A4A
:1055B000224BA3FB0A03DB0803EB8303AAEB4303A1
:1055C000D35C01F8013BCAE7A3FB09231D4A9442BF
:1055D0004FEAD30A21D80B461849174AA1FB0A0102
:1055E000C90801EB8101AAEB4101515C03F8011BE1
:1055F000CAE7A2FB0A38134B9C424FEAD80813D8DB
:105600000E4B0D4AA3FB0803DB0803EB8303A8EB57
:105610004303D35C01F8013BCAE70A22BAFBF2F06C
:1056200048F0B8FE0346D7E70A22B8FBF2F048F08C
:10563000B1FE0146E4E700BF68430A08CDCCCCCCFC
:105640009F8601003F420F00344870B490F8AC3F91
:10565000A3F13001092958D800F6AC7400F6BB70EC
:10566000224612F8015FA5F13001092904D88242CF
:10567000F7D1002070BC7047141B022C4BDD28486A
:10568000002101E010F8013B01EB8101161A0446EC
:1056900003EB4103022EA3F1300303F0FF01F1DC21
:1056A000204B03FB01F1A2424FF000030ED903EBA4
:1056B000830314F8016B5B00A242A3F1300333446F
:1056C00003F0FF03F3D1184800FB03F32E2D06D09F
:1056D0001648A0FB032370BC01EB93007047013216
:1056E0000425002404EB84041078013D3038640064
:1056F0000928A4B2204401D8013284B215F0FF0574
:10570000F0D1642202FB0433E2E700211D4600F6DB
:10571000AC720B46DAE70021054CC4E7704C00245C
:105720001D5C00248096980040420F00ABAAAAAAF4
:105730001C5C002438B50D460446FF2100682A464B
:1057400054F09AFE22682A44226038BD0C46164660
:10575000054683B533F00CFF204633F009FF0021E6
:10576000204B0846002E08BF1E463FF065F9002179
:1057700001203FF061F928463BF0F2FEB0B1012173
:1057800000203FF059F928463BF0E2FE074620464C
:105790003BF0E2FE0028FAD0394620463BF0E4FE1A
:1057A0003846B047002108463FF046F920463BF016
:1057B000D7FE0028DFD0012100203FF03DF9204630
:1057C0003BF0C6FE0146284601913BF0C5FE01991B
:1057D0000028F8D028463BF0C7FE002108463FF0DD
:1057E0002BF9C8E765830708F0B5002289B0DFF818
:1057F00098C004AF13460A604A603E468A60CA6099
:105800000A610268C2F3855040FA03F43546E407A2
:1058100004D513F80C4005F8014B2E460133062B36
:10582000F2D1174DC2F303240023C2F305302C44F8
:1058300005F5E76C33700DF1190694F830478DF8D3
:10584000184040FA03F43546E40704D513F80C4039
:1058500005F8014B2E460133062BF2D10023C2F38B
:10586000834506AC0846337002F00F030549C2F3C6
:1058700003120097CDE901454BF016F809B0F0BDD1
:1058800048C3090890430A0870CA090870B5094C52
:105890000546D4F8BC2F62B1002601362D21D4F87C
:1058A000BC0F40F081FCAE42F7DBBDE8704041F038
:1058B00001BE70BD704C00242DE9F04FCCB2002128
:1058C000164685B0804608463FF0B6F80021012014
:1058D0003FF0B2F83EF050FE022E09D0042E44F6FE
:1058E000C01518BF4FF49645072C06D900200CE0D0
:1058F000FF2C4FF41645F7D10326CB4B93F8C02F5E
:1059000099462AB90020C9F8C40F05B0BDE8F08F48
:10591000032E15D0C54900220C44032194F87306C8
:105920003AF084FD0028EDD0C14CC4F85009C37989
:105930009A07E7D4006851F03BFD41F25C13E05058
:10594000BB4C41F273130022032199F8C00FE654B7
:105950003AF06CFDC4F8540D0028D3D000684FF025
:10596000010A51F025FD41F258134FF4806204F60C
:105970005411E050032EAF4B04F60C17C4F818294D
:10598000C4F80C394FF00303C4F81C2941F2641227
:10599000A4F810394FF00003C4F8201904F6585148
:1059A000A35404F58B52C4F81459A2F800A041F294
:1059B0006C12C4F83839A35041F27012C4F82C3973
:1059C000A35241F27212C4F82839C4F82419C4F859
:1059D0003439C4F83039A3540ED0D4F850B99BF8F8
:1059E00004003EF0FDFDC4F84C09584619F00DFBCB
:1059F0005146384619F018FB32203BF071FA002E60
:105A000058D1D4F8540D22218B4A019051F062FCF8
:105A100041F27813894A07F66C010198E250324648
:105A200051F0FEFAD4F85009834A4FF6FF71019005
:105A300051F050FC31460198FBF728FA804A41F2B8
:105A40007C1307F507610198E250324651F0E8FAFD
:105A50007C4DC9F8C47F022E12D0D9F8C40F3BF098
:105A60007FFD68B1012100203EF0E6FFD9F8C40FA8
:105A70003BF076FD0146002840F09B803EF0DCFFC5
:105A800040463BF06DFD78B101214FF0060B084612
:105A90003EF0D2FF40463BF063FD0146002840F057
:105AA000918001203EF0C8FF042ED6D005203BF0A7
:105AB00017FAD0E7012E09D1D4F8540D2946FAF788
:105AC000FDFFD4F85009FBF707FAC1E7022E09D110
:105AD000D4F8500919F08DFA2946D4F8540DFAF784
:105AE000EDFFB5E7032E5CD14FF0000A41F27413CD
:105AF00040225548514604F803A054F0BDFCDFF89D
:105B000050B18DF80FA0DFF84CA19DF80F30072B96
:105B100009D901214D4819F087FA2946D4F8540DC6
:105B2000FAF7CCFF94E79DF80F3003EB43030BEB40
:105B3000C30393F845306BB39DF80F3003EB430379
:105B40000BEBC3039B6C2BB39DF80F20374B134417
:105B500093F87306F0B1002203213AF067FC01903C
:105B6000C0B119F046FA9DF80F309AF8001003EB17
:105B70004303019A09EBC1000BEBC3039B6CC0F814
:105B8000C83FD379DB0702D5012380F8CC3F013130
:105B90008AF800109DF80F300133DBB28DF80F301A
:105BA000B3E7042E7FF454AFD4F8500919F021FA6A
:105BB00082E7D9F8C40F3BF0CBFC014640463BF0EE
:105BC000D3FC53E740463BF0C3FC15F8E23C0746E4
:105BD00083B9242802D1012305F8E23C012E03D128
:105BE000394640463BF0C0FC3946D9F8C40F3BF07B
:105BF000BBFC4FE7012B06D14D280CBF022300232D
:105C000005F8E23CEAE7022B06D13C280CBF03234F
:105C1000002305F8E23CE1E7032B2AD10A281BD92F
:105C2000002305F8E23CD9E7704C0024783B0024BF
:105C30008819002488CA090840420F00B5F00508F9
:105C4000CDB30508685D0024385C0024942200244C
:105C500014000020FC2A0024002305F8EF0C05F8AE
:105C6000EE0C05F8F03C05F8ED3C042305F8E23CA9
:105C7000B4E7042B0AD115F8EE3C05F8E10C4340DB
:105C800005F8EE3C052305F8E23CA7E7052BA5D176
:105C900015F8F03C15F8EFAC15F8EE2C534509D289
:105CA000424005F8EE2C5A1C2B4405F8F02C03F862
:105CB000EC0C93E78242B3D115F8E13C05F8E2BC65
:105CC000F42B8BD1BAF1000F88D12421404605F87E
:105CD000E2AC3BF049FC4D2140463BF045FC3E2107
:105CE00040463BF041FC514640463BF03DFCF42130
:105CF00040463BF039FCF42140463BF035FC032E96
:105D000012D0D4F85059284651F04AF95146284645
:105D100051F060F92021287919F05AF9524651467C
:105D2000D4F8500951F07CF90022D4F8540D1146F2
:105D300051F076F90120E8E516490130002201EB27
:105D4000C000F0B4D0F874C7134E46F8E02C46F803
:105D5000D02C46F8C02C46F8B02C46F8A02C46F8BB
:105D6000902C46F8802C46F8702CBCF1000F0ED019
:105D700090F870775FB13F01E03E00240CEB040324
:105D8000351910340FCBA74285E80F00F6D1F0BCCF
:105D9000704700BF48C30908685D0024F0B5154D81
:105DA00083B00E4615F8603C022B0DD1070AC4B231
:105DB000D5F8D4010023012201A9384404F036FAB1
:105DC000012806D003B0F0BDC0F3D41700F07F0463
:105DD000EEE715F8603C022B019B04D133F8143038
:105DE000336003B0F0BD53F8243023F070433360C8
:105DF00003B0F0BD685D0024D0E9011310B48B42FC
:105E000090F91A2038BF0B46511C83600AD0144BFE
:105E1000FF2103EB021313F8352C6FF3000203F894
:105E2000352C817690F91B305A1C0FD00C49FF2479
:105E300001EB031111F8353CC3F34502013A22EAA4
:105E4000E27262F3460301F8353CC4760022436AED
:105E50005DF8044B114642614260036104F0CCB925
:105E6000685D002438B50F4C034694F8FF1104F523
:105E7000FC7084F8FB3101F03F0101F10A058B1C35
:105E8000083184F8FA51254484F8FD3121F016FDDB
:105E900085F8F60194F8FA31000A1C4484F8F701F9
:105EA00038BD00BF685D00242DE9F04FCD4C8DB0AA
:105EB0004FF00008DFF84093CB4D009054F80B0CE6
:105EC000002800F0FE803BF04BFB0646002800F067
:105ED000D781D9F85C3BE026A4F10B0BC34F44F803
:105EE000073C002306FB08F604F8033C54F80B0CAF
:105EF0003BF036FB002800F0E48054F80B0C3BF03C
:105F000027FB14F8023C82465A1E0B2A0DD8DFE804
:105F100012F01F003A004600530083009B00E2008D
:105F2000150134013F0175018C0124280CD0009A21
:105F30003AB995F88E22824240F07D81012204F820
:105F4000032C0D2BD2D186E0012304F8023CCDE7CF
:105F500000234D28C4F8C53084F8CD3084F8CE3005
:105F600004D0582808D004F8023CBFE7022284F885
:105F7000C43004F8022CB9E7032304F8023C0223DE
:105F800084F8C430B2E704233C2804F8023C0BD068
:105F9000BAF13E0F0CD0002304F8023CA6E70A2316
:105FA0003C2804F8023CF3D1002304F8013C9DE7AF
:105FB000012304F8013C99E7D4F8C500BB19421C41
:105FC0000344C4F8C520022A83F893A694F8CD00B0
:105FD0008AEA000184F8CD1088D12378C02BDAD862
:105FE0006278FF2A08D1052BD5D9012384F8C43063
:105FF000072304F8023C79E7A4F8C1200022C4F882
:10600000C930934284F8C320C4F8C52014BF0523C7
:10601000062304F8023C69E7D4F8C500BB19421C0A
:106020000344C4F8C52083F893A694F8CD00D4F8AF
:10603000C9308AEA00019A4284F8CD107FF456AF45
:10604000062304F8023C51E794F8CD308342A2D1F4
:106050000D2304F8023C14F8017C002F40F0F2807C
:10606000634B04AE0894ADF82C7003970FCB86E811
:106070000F00D4F8C930324608A9D4F8D10023441F
:106080000993B4F8C130ADF8283094F8C3308DF8D6
:106090002A3001238DF82E3003AB35F04FFB48B189
:1060A000049B314694F8C42058460593514B049301
:1060B00033F038F80023039E04F8023C002E40F031
:1060C000D78008F10108E034B8F1030F7FF4F6AE91
:1060D0000DB0BDE8F08FD4F8C500BA195146431C85
:1060E0000244C4F8C53082F893A694F8CD2094F801
:1060F000CE008AEA0202019384F8CD2048F0CCFC5D
:10610000019B84F8CE00072B7FF4F0AEB4F8053085
:10611000C02B3FF640AFB4F80320C4F8C930A4F850
:10612000C120A27884F8C32000229342C4F8C5207D
:1061300014BF0823092304F8023CD7E6014694F86B
:10614000CE0048F0A9FC94F8CD3084F8CE008AEA5D
:106150000303D4F8C50084F8CD30BB19421C0344B6
:10616000C4F8C52083F893A6D4F8C9309A427FF4C6
:10617000BDAE092304F8023CB8E694F8CD304340A4
:1061800084F8CD3094F8CE3083427FF404AF57E7E3
:10619000D4F8C500BA195146431C0244C4F8C530AE
:1061A00082F893A694F8CE00019348F075FC019B09
:1061B00084F8CE00052B7FF499AEB4F80120B4F832
:1061C0000330A4F8C1202278C4F8C93084F8C32071
:1061D00000229342C4F8C52014BF0B230C2304F8FB
:1061E000023C83E603530024685D0024704C0024C5
:1061F00090CB0908E0D00024802A0024014694F8BE
:10620000CE0048F049FCBB1984F8CE00D4F8C50094
:10621000421C0344C4F8C52083F893A6D4F8C930BF
:106220009A427FF463AE0C239DE694F8CE3083420D
:106230007FF4B1AE0CE723287FF483AE022204F88A
:10624000032C7EE6012F4FF0000602D004F8026C0A
:1062500037E7D4F8C93008A8089423440993B4F860
:10626000C130CDE90A66ADF8283032F0B7FBEDE772
:1062700054F80B0C33F07CF954F80B0CB04720E7C2
:1062800014F8033C002B3FF41CAFD9F85C2B54F8F6
:10629000071C521A632A7FF614AF012B30D0022B51
:1062A0007FF40FAF54F80B3C012285F8A50285F866
:1062B0009022C5F8A032134A1348C5F89C22134A0D
:1062C000C5E9A5334023C5F8E82285F8A432104B70
:1062D000C3F8BC2F95F8EF320E4A003B18BF0123DC
:1062E00082F82C3941F0EAF84FF4005035F0F2F81A
:1062F000094841F0D9F885F8FD6285F8FE62E0E6CC
:10630000FAF7BCFDE1E507089F430A080460002492
:10631000704C002414000020D5430A0838B51E4CE8
:106320000968D4F804530068491B1C4DDFED1C6A52
:1063300000EE901AD4F80013D5EDC17A1C46F8EEA1
:10634000E00A401A60EEA70A07EE900AF8EEE77A34
:1063500020EEA07AB1EE670AA7EEA77AF1EEC77A2F
:1063600067EEA67AFCEEE77AC2ED007A4AF080FB8F
:106370009FED0C7ADFED0C7AE0EE077AFDEEE77A1E
:1063800017EE902A002A02DBC4ED007A38BD48F6E9
:10639000A0431344236038BD685D0024000000243E
:1063A0002C7D8E3FA00CB34500A00C4638B50A4C9E
:1063B000002501228021204634F01EFD30B194F9E1
:1063C000040034F04DFD08B1006838BD01350C34CF
:1063D000092DEED10020F8E7885F002438B5041FAE
:1063E00000F1080554F8043FD81780EA43001EF076
:1063F000E1F8A542F6D138BD084B4FF6FF700021F9
:1064000003F5136210B40024C3F8DC09C2F8A41029
:10641000C3F8D8495DF8044B704700BF1400002052
:106420002DE9F041BB4CDFEDBC7AD4F8E42994F8B7
:10643000C53907EE102A2DED028BB8EE478A28EEFB
:10644000278A002B45D094F83079002F40F0B68091
:10645000B24E0025DFEDB28A4FF0000894F8E8391B
:106460002B41DB0712D594F8C4391BBBB4F8C639ED
:1064700007EE103A002F46D0B8EE477AC8EE877A7A
:1064800077EE887A88EE277A86ED027A013524360F
:10649000042DE3D194F8C959B4F8CC69B5BB2FB930
:1064A00094F8E03984F8F07984F8EC39BDEC028B8B
:1064B000BDE8F081B4F8C639301DD4F8E41900EE17
:1064C000103AB8EE400ACFB943F04CFF94F8307957
:1064D000DCE794F8C41994F8E129B1FA81F1D4F811
:1064E000D009B4F8C65949092BF07CF980B285422D
:1064F000A4F8C609A7D094F83079A9E755F018FF99
:1065000094F83079C2E7C6F80480B5E7854A94F874
:10651000CA39D2F8182392F8832013435ED1A5F12B
:10652000010194F8E129D4F8D009B1FA81F14909BF
:106530002BF058F980B2A4F8CC09002F61D194F85F
:10654000E03984F8F05984F8EC390028AED007EE31
:10655000900A0123B8EE678A9D42DFED717A84F8D4
:10656000F439C7EE888A00F08B80022D9ED1D4F8D2
:10657000E419B0EE480A6C4843F0F4FE94F8F039A0
:10658000012B00F0C180022B90D1B0EE480AD4F864
:10659000E419664843F0E6FE94F8F039012B00F068
:1065A000AE80022B82D1B0EE480AD4F8E4196048DC
:1065B000BDEC028BBDE8F04143F0D4BE94F8C9595C
:1065C000B4F8CC69002D3FF471AF564A94F8CA393B
:1065D000D2F8182392F88320134304D0002F7FF4BD
:1065E00065AF3046ABE7A5F1010194F8E129D4F895
:1065F000D009B1FA81F149092BF0F4F880B2A4F87E
:10660000CC09B0423FF452AF00283FF44FAF94F8AA
:10661000F039002B3FF44AAF07EE900A012BB8EE99
:10662000678ADFED3F7AC7EE888A47D0022B7FF476
:106630003DAFD4F8E419B0EE480A3B4855F078FE77
:1066400094F8F039012B52D0022B7FF42FAFB0EE2B
:10665000480AD4F8E419354855F06AFE94F8F03940
:10666000012B47D0022B7FF421AFB0EE480AD4F8BB
:10667000E4192F48BDEC028BBDE8F04155F058BE3F
:106680002C4A0021D2ED007A134678EEA76A43F82F
:10669000041F87EEA67A83ED017A78EEA76A0021BF
:1066A000996087EEA67A83ED037A77EEA88A0022B6
:1066B0001A6187EEA87A83ED057AF7E61D4A13463C
:1066C000F3EC017A78EEA76A87EEA67A83ED017A79
:1066D000D2ED007A78EEA76A87EEA67A83ED037A88
:1066E00077EEA88A87EEA87A83ED057ADEE6114A6E
:1066F000131DEDE70F4A131DD2ED007AF0E70D4AA6
:10670000131DD2ED007AD0E70A4A131DD2ED007AAC
:10671000C3E700BF14000020BD37863544090020C0
:1067200083F9223E685D00240C0A0020300A002014
:10673000540A0020780A0020012816D02E4B93F826
:10674000803A012B2AD02D4BF6EE006ABEEE007A7D
:10675000DFED2B7A03EB800090EDCD0A80FE660A18
:1067600080FE070A20EE270A7047244AF6EE006AE8
:10677000214BBEEE007A92EDCE0ADFED217A93F83E
:10678000843A80FE660A80FE070A20EE270A23B1BB
:10679000B5EEC00AF1EE10FA03DC70479FED190A5E
:1067A000704707EE903AB2F91E13B2F93233DFEDBB
:1067B000166AF8EEE77ACB1A07EE103AB8EEC77A07
:1067C00027EE267AB4EEE77AF1EE10FAE6DA77EE03
:1067D000C77AB2EE047AF4EEC77AF1EE10FADCD89A
:1067E000B1EE047A67EEA67A30EE470AA7EE807A19
:1067F000B0EE470A704700BF14000020685D002417
:106800000000484300000000CDCCCC3DF8B5774CEB
:1068100040F60302B4F8403313402DED048BB0EE84
:10682000408A04D0B0EE480ABDEC048BF8BD04EBFE
:106830004001B5EEC00ADFED6E6AF7EE007AB1F9FD
:106840003053BFEE007AB1F91C23F1EE10FA694E15
:106850004FEA800CA2EB050206EB8001C8BF0127BE
:1068600000EE102AD8BF4FF0FF37D1F8885AB8EEA3
:10687000C00A20EE260AB5EEC00AF1EE10FACCBF2F
:106880004FF0010E4FF0FF3E77FE877AEA1B18BFEC
:106890000122002D08BF0022002A48D106F52963F5
:1068A000F0EEC06A93ED007AF4EEC76AF1EE10FAEA
:1068B00007DD774508BF002D0CBF0122002200F044
:1068C0008480002D41D0B0EE408A4B4BDFED4B8AE7
:1068D000D3ED006A97EE278A9FED497ADFED497A7A
:1068E00028EE268A88FE478A88FE278A002A60D1F9
:1068F00096F8D83A984295D194F84233262B91D104
:10690000B2EE049A20EE090A51F0CAFAB0EE480A33
:10691000A4F84653A4F8440351F0C2FA28EE890AB9
:10692000A4F8480351F0BCFAA4F84A037AE706F544
:106930002962F0EEC06AC1F8883A92ED007AF4EE6E
:10694000C76AF1EE10FA3EDC1A4606EB80019FEDB5
:106950002E6AD1ED6D7AF0EEE76AF4EEC66AF1EEDA
:1069600010FA2DDC9FED296A66EE866A284BF0EE60
:10697000408AB7EE006A93ED005AFFEE005A67EEC8
:10698000857AE6EEA78AF5EEC08AF0EEE87AF1EEB7
:1069900010FAF4EE477ACCBF01214FF0FF3136FEFA
:1069A000256AF1EE10FA01DD8F4215D00025002A8C
:1069B0009ED08444174B002203EB8C035A6097E768
:1069C000F7EE006AD2E77745BED106EB0C037546B9
:1069D0000122C3F888EA74E7B0EE688A53ED017AC1
:1069E000002597EE068A28EE278AE2E7685D0024F4
:1069F000CDCCCC3D14000020A80A002000000000EF
:106A000000007A4400007AC4FFFFF9436F12033B91
:106A1000AC0A0020B00A002030B46B4C0A7804EBBA
:106A200080016A4D534207EE902AD1EDCD6A07EE00
:106A3000103AD1F84C33B8EEE76A85FB0315DB1743
:106A4000B8EEC77AC3EB651307EE903AF8EEE77A33
:106A5000E6EE267AF4EEC77AF1EE10FA05D407EEE8
:106A6000102AF8EE476A86FEE77A04EB400040F60B
:106A70000101B4F84023B0F91C33B0F930031142DE
:106A8000DFED536AA3EB000307EE903AF8EEE77AE6
:106A9000A7EEE67A06D04F4B93ED000A30BC27EE06
:106AA000000A7047B4F91C33B4F91E23002BD4ED4F
:106AB000D67A94EDD56AB8BF5B42002A87FE866A13
:106AC0004549B8BF52429BB291F8E00A92B2934254
:106AD000B8BF134607EE903AF8EEE77A67EEA67A6B
:106AE00060BB01F6EC23F7EE005AD3ED006AF4EE3A
:106AF000E56AF1EE10FA54D401F6E421D1ED007A02
:106B0000DFED365AF4EEE57AF1EE10FA46D9DFED14
:106B1000344AB7EE005AC4EEA76AF0EE457AE6EEC4
:106B2000667AC7FEC56AC6FEA56A2E4BD3ED007A0B
:106B300067EE277A30BCA7EEA60A704701F6E42379
:106B40009FED265AD3ED005AF4EEC55AF1EE10FA35
:106B500021DD01F6E821D1ED004AF4EEC54AF1EE5F
:106B600010FA18DDDFED206A74EEE77AB7EE004A1E
:106B700026EE266AC7EEA46AC6EE257AC6FEC46A69
:106B8000C6FE856A77EE847A66EEA76AC6FEC46A98
:106B9000C6FE856AC9E7F0EE456AC6E7F0EE656AAB
:106BA000C3E775EEE65ADFED114A9FED115A01F683
:106BB000E42165EEA45AD1ED004A75EE677AE5EE60
:106BC000A76A66EEA47A9BE7685D00241F85EB51F7
:106BD000CDCCCC3DF00A00201400002000000000C5
:106BE0000000C842040B00200000C8C2610BB63B85
:106BF000000034432DE9F04F0C4F97F84253102D0D
:106C00002DED048B83B000F06184094C002694F8CC
:106C1000B187B8F1060F00F24484DFE818F0D3041E
:106C2000940565040B00D800A8056903685D00247D
:106C300014000020E34B102D1A4693ED037AD3ED98
:106C4000057AB2EC011A27EE073A67EEA73A93ED00
:106C5000077A92ED006AD3ED097A27EE074AD3ED61
:106C60000B6A66EE062A93ED0D7A67EEA74AD3ED1E
:106C70000F7A26EEA65AD3ED021A67EE075A93ED65
:106C8000042A27EEA76AD3ED116AE1EE012A93EDFB
:106C9000137AA1EEA13AD3ED157AE2EE023AD3EDE2
:106CA000060A66EEA66A93ED081A27EE077AD3ED78
:106CB0000A1A67EEA77A93ED0C2AA0EEA04AE1EE3D
:106CC000014AD3ED0E0AA1EEA15A93ED101AE2EE9D
:106CD000025AD3ED121A93ED142AA0EEA06AE1EE47
:106CE000016AE2EE027AA1EEA17AB1EEE22AF1EEB9
:106CF000C32AB1EEE33AF1EEC43A03ED202AB1EE35
:106D0000E44A43ED1F2AF1EEC54A03ED1E3AB1EE07
:106D1000E55A43ED1D3AF1EEC65A03ED1C4AB1EEB9
:106D2000E66A43ED1B4AF1EEC76A03ED1A5AB1EE6B
:106D3000E77A43ED195A03ED186A43ED176A03ED3C
:106D4000167A93ED177AD3ED197A67EE075AD3EDD9
:106D50001B6A27EEA76A93ED1D7AD3ED1F7A66EEC4
:106D6000A66AD3ED164A27EE077A93ED185A67EE16
:106D7000A77AE4EEA45A93ED1A4AA5EE056AD3ED7C
:106D80001C4A93ED1E5AE4EE046AA4EEA47AE5EEE2
:106D9000057AB1EEE55AF1EEC65AB1EEE66AF1EEC9
:106DA000C76A03ED155AB1EEE77A43ED145A03EDC5
:106DB000136A43ED126A03ED117A00F0758794F8B7
:106DC000B18708F101085FFA88F884F8B18794F870
:106DD00010310F2B00F3B6877B490D2B03F1010C0B
:106DE00001EB830200F2C38701F2844A02F5C66216
:106DF0000AEB8301D2ED007A91ED6C7AB4EE677AFA
:106E0000F1EE10FA05DDB5EEC07AF1EE10FA00F3FE
:106E100046870020DFED6D7A0AEB8C02D2ED6C6ABA
:106E2000F4EE476AF1EE10FA08DDF4EE676AF1EE6F
:106E300010FA03DDF0EE667A5FFA8CF0D91C03F1EC
:106E4000020C0E29624600F3EE800AEB830292EDFB
:106E50006E7AB4EE667AF1EE10FA08DDB4EE677A77
:106E6000F1EE10FA03DDF0EE477A5FFA8CF00AEBF0
:106E70008302D2ED6F6AF4EE476AF1EE10FA07DD95
:106E8000F4EE676AF1EE10FA02DDF0EE667AC8B24F
:106E9000591D03F1040C0E29624600F3C4800AEB6D
:106EA000830292ED707AB4EE667AF1EE10FA08DDA4
:106EB000B4EE677AF1EE10FA03DDF0EE477A5FFA8E
:106EC0008CF00AEB8302D2ED716AF4EE476AF1EEC0
:106ED00010FA07DDF4EE676AF1EE10FA02DDF0EE6B
:106EE000667AC8B2D91D03F1060C0E29624600F37A
:106EF0009A800AEB830292ED727AB4EE667AF1EE32
:106F000010FA05DDB4EE677AF1EE10FA00F3E786C9
:106F10000AEB8302D2ED736AF4EE476AF1EE10FADF
:106F200005DDF4EE676AF1EE10FA00F3D38603F1A3
:106F3000090103F1080C0E29624674DC0AEB830296
:106F400092ED747AB4EE667AF1EE10FA05DDB4EEE5
:106F5000677AF1EE10FA00F3CD860AEB8302D2EDE8
:106F6000756AF4EE476AF1EE10FA05DDF4EE676A31
:106F7000F1EE10FA00F3B98603F10B0103F10A0CEC
:106F80000E2962464FDC0AEB830292ED767AB4EE6C
:106F9000667AF1EE10FA05DDB4EE677AF1EE10FADA
:106FA00000F3B3860AEB8302D2ED776AF4EE476A08
:106FB000F1EE10FA0CDDF4EE676AF1EE10FA00F370
:106FC0009F8605E060080020AC0100200000000062
:106FD00003F10C01012B0A4625DC0AEB830292ED3A
:106FE000787AB4EE667AF1EE10FA07DDB4EE677ADD
:106FF000F1EE10FA02DDF0EE477AC8B20AEB830236
:10700000D2ED796AF4EE476AF1EE10FA09DDF4EE9A
:10701000676AF1EE10FA04DD03F10D00F0EE667A16
:10702000C0B203F10E0202F16C030AEB82010AEB1B
:10703000830CD1ED6B6A9CED007AF4EE476AF1EEB9
:1070400010FA07D5B4EE677AF1EE10FA02DDF0EE31
:10705000477AD0B20F2A02F1010C00F0F3830AEB59
:1070600083030AEB8201D3ED006A91ED6D7AF4EEB1
:10707000476AF1EE10FA05D5B4EE677AF1EE10FA30
:1070800000F37D860E2A02F1020300F0DB830AEB97
:10709000830191ED6C7AD1ED6B6AF4EE476AF1EE03
:1070A00010FA05D5B4EE677AF1EE10FA00F37186A6
:1070B0000F2B03F1010200F0C5830AEB820191ED71
:1070C0006C7AD1ED6B6AF4EE476AF1EE10FA05D5F1
:1070D000B4EE677AF1EE10FA00F364860F2A02F13B
:1070E000010300F0AF830AEB830191ED6C7AD1EDDF
:1070F0006B6AF4EE476AF1EE10FA05D5B4EE677AE2
:10710000F1EE10FA00F357860F2B03F1010200F0A5
:1071100099830AEB820191ED6C7AD1ED6B6AF4EE02
:10712000476AF1EE10FA05D5B4EE677AF1EE10FA7F
:1071300000F34A860F2A02F1010300F083830AEB71
:10714000830191ED6C7AD1ED6B6AF4EE476AF1EE52
:1071500010FA05D5B4EE677AF1EE10FA00F3408626
:107160000F2B03F1010200F06D830AEB820191ED18
:107170006C7AD1ED6B6AF4EE476AF1EE10FA05D540
:10718000B4EE677AF1EE10FA00F336860F2A02F1B8
:10719000010300F057830AEB830191ED6C7AD1ED86
:1071A0006B6AF4EE476AF1EE10FA05D5B4EE677A31
:1071B000F1EE10FA00F329860F2B03F1010200F023
:1071C00041830AEB820191ED6C7AD1ED6B6AF4EEAA
:1071D000476AF1EE10FA05D5B4EE677AF1EE10FACF
:1071E00000F31C860F2A02F1010300F02B830AEB47
:1071F000830191ED6C7AD1ED6B6AF4EE476AF1EEA2
:1072000010FA05D5B4EE677AF1EE10FA00F31C8699
:107210000F2B03F1010200F015830AEB820191EDBF
:107220006C7AD1ED6B6AF4EE476AF1EE10FA05D58F
:10723000B4EE677AF1EE10FA00F30F860F2A02F12E
:10724000010300F0FF820AEB830191ED6C7AD1ED2E
:107250006B6AF4EE476AF1EE10FA05D5B4EE677A80
:10726000F1EE10FA00F302860F2B03F1010200F099
:10727000E9820AEB820191ED6C7AD1ED6B6AF4EE52
:10728000476AF1EE10FA05D5B4EE677AF1EE10FA1E
:1072900000F3F5850F2A02F1010300F0D3820AEB17
:1072A000830191ED6C7AD1ED6B6AF4EE476AF1EEF1
:1072B00010FA05D5B4EE677AF1EE10FA00F3E8851E
:1072C0000E2B40F0BF82B84B93ED007A53ED016A6C
:1072D000B4EE667AF1EE10FA40F3B482B4EEE77AD7
:1072E000F1EE10FA40F3AE82F0EE477A0F20ACE2F6
:1072F00094F8B22794F82C36DFF8C0E203F5937CBB
:10730000C3F120030CEB421C13F0FC0FC3F3850008
:107310005FFA83F80EEB8C0C00F00D8501300CF158
:107320001003AEF170010EF244624FEA00190CEB4B
:10733000001013ED026A103311ED027A103253ED92
:10734000076A103153ED057A26EE076A51ED074AB8
:1073500013ED087A834211ED085A66EEA46A51EDE6
:10736000055A27EE057A02ED066A67EEA57A42ED28
:10737000076A02ED087A42ED057ADAD18B49A9F164
:10738000100301F2B4629C44C818134418F00302BD
:107390001BD0DCED007A013A90ED007A67EE877A37
:1073A000C3ED007A11D0DCED017A012A90ED017A6B
:1073B00067EE877AC3ED017A07D0DCED027A90EDB3
:1073C000027A67EE877AC3ED027A94F82C060028D9
:1073D00063D094F8B2370EEB880C5FEA90090EEB9D
:1073E000C31E0CF2346C01EB88080EF5936E35D099
:1073F00009F101090EF1100308F110010CF110025E
:107400004FEA091A0EEB091913ED026A103311ED58
:10741000027A103253ED076A103153ED057A26EEE9
:10742000076A51ED074A13ED087A4B4511ED085AEA
:1074300066EEA46A51ED055A27EE057A02ED066A5A
:1074400067EEA57A42ED076A02ED087A42ED057A09
:10745000DAD1AAF110039E4498449C4410F0030032
:107460001BD0DEED007A013898ED007A67EE877A5E
:10747000CCED007A11D0DEED017A012898ED017A89
:1074800067EE877ACCED017A07D0DEED027A98EDCF
:10749000027A67EE877ACCED027A102D7BD094F8D1
:1074A000B18708F10108424BA3FB0823A8EB0302B4
:1074B00003EB52039B08C3EBC303A8EB030384F85D
:1074C000B13703B0BDEC048BBDE8F08F39F08AFC16
:1074D000384C97F84253064694F8B187102D08BFF0
:1074E000A7F84483FFF795BBDFF8CC80DFF8D0E046
:1074F000B0EE006AD8ED005AF6EE006ADEED007AD2
:107500000EF18C03B4F8B40777EEA77AD4F8C81755
:107510000138B0EE664A1031B0EE677A08EBC0026F
:10752000E5EE867A083A95EE867A67EEA67A27EE39
:10753000267ACEED1F7A8EED207AD2ED036A0138DD
:10754000D2ED027A01F1080153ED215AA2F10802AD
:1075500053ED224A03F1080335EEE67A11ED036A92
:1075600037EEE45A77EEA47A76EEA56A51ED045A26
:10757000A6EE057AE5EE857AA5EEE67AE6EE267ABF
:1075800027EE047A67EE847A03ED037A43ED047AFA
:10759000D3D1102D83D139F025FC801B94F8B1870D
:1075A000A7F846037DE700BF1C0800202C0100203F
:1075B0002549922414000020E0070020AC0100209F
:1075C000E4070020B4F8B4379A485908D4F8B8272B
:1075D00000EB8308DB084FEA810C00EB810A00F026
:1075E000A38003F1010E0CF1100C0AF1100310300E
:1075F0000AEB0E1AC44402F1100908F1100E5EEDF8
:10760000047A103310ED041A09F110095CED041A24
:10761000103013ED086A71EE278A5EED032A31EE11
:10762000671A1CED032A36EE218A5EED013A71EEEF
:10763000C61A13ED064A0EF1100E53ED054A0CF171
:10764000100C5EED066A53ED075A5CED067A1CEDF0
:10765000057A35EE820A10ED063A72EE655A10EDA3
:10766000075A74EE270A10ED056A77EEC47A40EDEA
:10767000088A35EE229A36EE232A35EE625A73EEE8
:10768000268A00ED079A74EE872A00ED052A37EE68
:10769000647A40ED068A73EE666A43ED052A36EE9B
:1076A000636A03ED088A03ED070A43ED060A5345B2
:1076B00059ED074A19ED084A24EEC12A24EE653A2D
:1076C00065EE242AA5EE042A61EE843AB0EE435A10
:1076D000E1EE042AE5EEA43AA1EEA45A0EED072A43
:1076E0004EED082A4CED073A0CED085A59ED055AB3
:1076F00019ED065A26EE253A65EEE63A27EE854A5A
:1077000065EE474AE6EE053AA6EE853AA7EE254A2B
:10771000E7EEA54A0EED063A4EED053A0CED054AA8
:107720004CED064A7FF46BAF89B242480191F8F7FD
:1077300067FC01994046D4F8B827F8F761FC102D92
:107740007FF4ADAE27E7DFF8EC80D4F8BC274046E5
:10775000B4F8C01750F0E2FA97F84253102D00F039
:10776000FE8294F8B137013384F8B137BEE6324B6C
:107770001B78002B00F06882304A94F8B23702F18F
:10778000DC08D4ED3D7A03EBC300D4F89C1108EB80
:107790008303D4ED3F0A02EB800093EDAC0AD0F8EE
:1077A0001CA0D0F8209020EE270A90ED054AD0F8D2
:1077B00018B0FCF797FE80ED054A6C32C0F818B09F
:1077C000C0F81CA0C0F8209094F8B237D4ED3E7AEF
:1077D00008EB8308D4F89C1103EBC30098EDAC0AC6
:1077E00002EB800020EE270AD0F814A0D0F8189001
:1077F000D0F81C80026AFCF775FE102DC0F814A0AA
:10780000C0F81890C0F81C80026200F0A08294F8C2
:10781000B2270B4B013294F8B107A3FB02130130DE
:1078200003F4FF7184F8B10701EB5303D21A84F813
:10783000B2275FE5E007002000000020540500208B
:10784000ABAAAAAA002800F04E81431E012B40F3E8
:10785000C4820AEB8002811E92ED6B7A1346D2ED50
:107860006A6AF4EEC76AF1EE10FA00F38280012929
:107870007FD093ED697AC21EB4EEE67AF1EE10FA8B
:1078800000F34982012A00F04682D3ED686A021FA4
:10789000F4EEC76AF1EE10FA6BDC012A69D093EDC1
:1078A000677A421FB4EEE67AF1EE10FA00F3338203
:1078B000012A00F03082D3ED666A821FF4EEC76AB7
:1078C000F1EE10FA55DC012A53D093ED657AC21F10
:1078D000B4EEE67AF1EE10FA00F31D82012A00F010
:1078E0001A82D3ED646AA0F10802F4EEC76AF1EEE1
:1078F00010FA3EDC012A3CD093ED637AA0F1090234
:10790000B4EEE67AF1EE10FA00F30582012A00F0F7
:107910000282D3ED626AA0F10A02F4EEC76AF1EEC8
:1079200010FA26DC012A24D093ED617AA0F10B0233
:10793000B4EEE67AF1EE10FA00F3ED81012A00F0E0
:10794000EA81D3ED606AA0F10C02F4EEC76AF1EEB1
:1079500010FA0EDC012A0CD093ED5F7AA0F10D0233
:10796000B4EEE67AF1EE10FA00F3D581022A07FEB2
:10797000267A431C0E2B00F33C820AEB800100F1B7
:10798000020CD1ED6D6A0A4691ED6E6AB4EEE66ABC
:10799000F1EE10FA00F36E81BCF10F0F00F08E8053
:1079A000D2ED6F6AC11CB4EEE66AF1EE10FA00F196
:1079B0005F810F2900F0B28192ED706A011DB4EE73
:1079C000E66AF1EE10FA00F355810F2976D0D2ED78
:1079D000716A411DF4EEC66AF1EE10FA00F34881B7
:1079E0000F2900F09B8192ED726A811DB4EEE66A68
:1079F000F1EE10FA00F33E810F295FD0D2ED736AE9
:107A0000C11DF4EEC66AF1EE10FA00F331810F29C0
:107A100000F0848192ED746A00F10801B4EEE66A28
:107A2000F1EE10FA00F326810F2947D0D2ED756AE6
:107A300000F10901F4EEC66AF1EE10FA00F31881C4
:107A40000F2900F06B8192ED766A00F10A01B4EE25
:107A5000E66AF1EE10FA00F30D810F292ED0D2ED77
:107A6000776A00F10B01F4EEC66AF1EE10FA00F34A
:107A7000FF800F2900F0528192ED786A00F10C012D
:107A8000B4EEE66AF1EE10FA00F3F4800F2915D097
:107A9000D2ED796A00F10D01F4EEC66AF1EE10FA4A
:107AA00000F3E6800E2940F03981E14A92ED006A48
:107AB000B4EEE66AF1EE10FA00F3DC8087FE667A37
:107AC000C7EE878A94F8B29709F1AC0BB2EE007A50
:107AD0000AEB8B02F7EE007A92ED008AC8FEC78AA5
:107AE000C8FEA78A17E0F2EE008AB7EE007AC7FE5A
:107AF000E88AC8FE878A94F8B29794ED430A09F1A0
:107B0000AC0B0AEB8B0393ED008A88EE000A50F071
:107B1000C7F9C0B2431C0AEB800207EE900ADBB241
:107B200092ED6C7AF8EEE76A0F2B27EE077A66EE95
:107B3000876A69D80AEB830207EE903A012892ED32
:107B40006C6AF8EEE77A26EE066AE6EE276A37EE0A
:107B5000067A59D8B5EEC07AB4F80431F1EE10FACD
:107B600069DD86EE879A94ED437A29EE077AB4F8B8
:107B7000002107EE902AF8EE677AF4EEC77AF1EE6C
:107B800010FA05DC07EE903AF8EE677AC7FEC77A7E
:107B900094ED457A77EEC87A0AEB8B0A28EE877A5D
:107BA000A7EE278A8AED008A2DF02AFB0028B8BFAD
:107BB0004042C0B214280DD9B4F8F43A07EE903A16
:107BC000F8EEE77A87FE888ABCEEC88A18EE103A8B
:107BD000A4F8F43AB9F1000F32D10F2D00F0A180D2
:107BE000112D6AD1934B9FED940AD3ED007A28EEC4
:107BF000800AFDEEE77A17EE903AA7F8443350F08A
:107C00004FF9A7F846034AE40138C0B20AEB8003F3
:107C100007EE900A93ED6C6AF8EEE77AB4F8043157
:107C200026EE066A37EE067AE6EE276AB5EEC07AE9
:107C3000F1EE10FA95DCB0EE487A9FED809A96E767
:107C4000102D7FF42EACA6E494F8B2377C4803EBF9
:107C5000C302D4ED3F0A00EB8303D4F89C1100EB80
:107C6000820093EDE30AD0F814A0D0F81890BFE595
:107C7000F0EE466A87FE667AC7EE878A94F8B29776
:107C800009F1AC0BB2EE007A0AEB8B02F7EE007A48
:107C900092ED008AC8FEC78AC8FEA78A3BE7F0EECD
:107CA000477A1846FFF7B8B839F09CF8801B97F868
:107CB0004253A7F84803FFF782B82B2DC0D15D4B84
:107CC000D3ED007AFDEEE77A17EE903AA7F8463347
:107CD000FFF7E5BBF0EE667AC8B2FFF728B9F0EE21
:107CE000477A5FFA8CF0FFF713B9F0EE667AC8B204
:107CF000FFF742B9F0EE477A5FFA8CF0FFF72DB943
:107D0000F0EE667AC8B2FFF763B9F0EE477A5FFA31
:107D10008CF0FFF747B9B0EE667A2AE6F0EE466AD5
:107D2000CCE69FED450A29EE000A50F0B9F8A7F815
:107D30004A03FFF7B6BBAEF180010EF2346308468A
:107D4000FFF724BBF7EE008ADFF8F8A0D3E639F09E
:107D500049F8801B97F84253A7F8460357E539F0D6
:107D600041F8801B97F84253A7F84603F9E41A46F6
:107D700001F2844A0020DFED317AFFF754B90E2A70
:107D8000F0EE477A5FFA8CF002F102037FF47FA9EC
:107D90005BE50F2BF0EE477AD8B203F101027FF4D6
:107DA0008CA952E50F2AF0EE477AD0B202F1010316
:107DB0007FF499A949E50F2BF0EE477AD8B203F189
:107DC00001027FF4A6A940E50F2AF0EE477AD0B26F
:107DD00002F101037FF4B3A937E5B7EE007AC8E5F5
:107DE0000F2BF0EE477AD8B203F101027FF4BDA960
:107DF0002BE5F7EE006A61E60F2AF0EE477AD0B283
:107E000002F101037FF4C7A91FE50F2BF0EE477ABB
:107E1000D8B203F101027FF4D4A916E50F2AF0EEDF
:107E2000477AD0B202F101037FF4E1A90DE500BF6A
:107E30001C080020E00800200000C84200000000EC
:107E400054050020300600200F2BF0EE477AD8B200
:107E500003F101027FF4E1A9F7E40F2AF0EE477A7B
:107E6000D0B202F101037FF4EEA9EEE40F2BF0EEA5
:107E7000477AD8B203F101027FF4FBA9E5E40F2AA7
:107E8000F0EE477AD0B202F101037FF408AADCE4F5
:107E90000E2BF0EE477AD8B23FF415AAD5E4F8B528
:107EA000214C1D270E46054684F8607320F054FDD2
:107EB000002020F0F7FC082020F0F4FC0E2020F039
:107EC000F1FC384620F0EEFC042020F0EBFC04200E
:107ED00020F0E8FC002020F0E5FC302020F0E2FC5F
:107EE000002020F0DFFC304620F0DCFC002020F0F9
:107EF000D9FC20F01DFD04F2613020F02CFC23465B
:107F000070B194F8612362B994F86223302A00D0EA
:107F10003AB993F8632322B993F8643301202B70A4
:107F2000F8BD0120FCE700BF685D0024104B03444E
:107F300010B5044693F8580816F0CCFA0D480A23F9
:107F400000EB44040920B4F97413B1F5FA6FA8BF2B
:107F50004FF4FA61B1F57A7FB8BF4FF47A71A1F5A9
:107F60007A71B1FBF3F1BDE81040C9B216F0E0BA86
:107F700048C30908685D00241C4991F8AC2F9AB3E6
:107F8000F0B4002605463346304637461BB991F813
:107F9000AC4F2D2C22D02E2A18D0CA1800EB80000E
:107FA00092F8AC4F4000A4F13002092A02D8A0F1A7
:107FB0003002A0180E2B14D80133CA1892F8AC2F37
:107FC000002AE3D106B14042F0BC70470133002DD6
:107FD000F8D0CA182A4482F8AC7FDEE701231E4697
:107FE000EBE70020F0BC704700207047704C002485
:107FF0001FB503AC8DF80C30002300948DF80D30C4
:1080000014F07CFB04B010BDF8B50546262025F021
:108010002BFA134C0146F8B9D4F8980390F838308D
:108020001E3B012B01D939F09FFA0E4F0026AE42BC
:108030000ADBB4F8BC330133A4F8BC330A4BD3F8E1
:108040005C3BC4F8CC33F8BD17F8011B0136D4F8FB
:10805000980339F089FAEAE7002384F8CA33EDE798
:10806000685D002404610024802A002410B5F9F71B
:10807000C1FA0446112138F089FA20463CF0C8FCC8
:10808000C82038F02DFF2046BDE810403CF0C6BCAB
:1080900008B552203CF0A4FA054BC3F8D00308B150
:1080A0002A23C3804021BDE8084038F06FBA00BFE2
:1080B000685D0024F8B5694CD4F8641B0B699E0711
:1080C00002D5CB689D074BD40B69580702D5CB6806
:1080D0005A073DD40B691B0702D5CB681F072FD465
:1080E0000B69DE0602D5CB68DD0621D40B69D80703
:1080F00002D5CB68DA073FD40B691B0603D5CB68E2
:108100001F0600F18F800B69DE0503D5CB681D06C5
:1081100000F18C800B695C0603D5CB68580600F132
:1081200089800B699A0602D5CB689B0620D4F8BDDE
:108130006FF0100200230A61CA6984F8803BD5E71A
:108140006FF0080200230A61CA6984F8803BC7E720
:108150006FF0040200230A618A6984F8803BB9E762
:108160006FF0020200230A618A6984F8803BABE762
:108170006FF020030B61F8BD394B6FF0010299429B
:108180000A61B9D1D4F8400BD0F81432002BB3D126
:10819000344E354AD6F8D45395B1D2F808C505F017
:1081A0003F076544C2F80855D2F80855B5F5006F89
:1081B00001D1C2F808350023C6F8D433002F43D0CC
:1081C000D2F80855D2F80C359D4295D0D2F8085512
:1081D000D2F80C359D4231D9D2F80855C5F5006565
:1081E000D2F80875B5F5007F204A28BF4FF4007516
:1081F000D0F814323A44C0F81052C0F80822002BCC
:108200007FF47AAF012781212B46C4F8B858C0F813
:108210001472D4F8580B04F0FBFED4F8641BC6F8B3
:10822000D45369E76FF080030B616CE76FF48073E0
:108230000B616FE76FF040030B6172E7D2F80C55EA
:10824000D2F80835ED1ACBE7D2F80825074BC0F86D
:1082500010721344C0F808324EE700BF802A002491
:1082600000140040685D002488190024082B0024B5
:1082700038B5D0F8D04201F00F03626893422BD892
:108280000A062BD41C25C1EBC102002005FB0141CD
:1082900004EB820201F5FE7182F8FD0101220B70F0
:1082A0008A7094F8BC03904216D084F8BC234A78B4
:1082B0002068012A09781DD000F5306202EB4112D6
:1082C0001568002D00DBF1B9116841F4001111604F
:1082D0001BB3002384F8BC33002038BD1C21C3EB42
:1082E000C302012001FB034104EB82023C3182F80E
:1082F0003D00D3E700F5106202EB4112156800293A
:10830000E2D0002DE0DB116821F08041116011689E
:1083100041F400111160002BDBD104F57172217C56
:1083200004F0DAFCD5E700BF10B504468021FFF762
:108330009FFF00212046BDE8104099E72DE9F04F4E
:108340009A4D89B02B685C6914F0010402D009B021
:10835000BDE8F08F59699A691142F8D05A69996954
:108360000A40900703D55A6902F002025A615A691D
:10837000996901930A40D10612D59A6922F0100238
:108380009A611A6AC2F3434102F00F07022900F012
:108390009D83062900F0FC829A6942F010029A61DE
:1083A0005A6999690A40120300F119825A69996958
:1083B0000A40510300F14E8159699A69114252D421
:1083C0005A6999690A4012050AD5019A02F50062B4
:1083D0009268D70700F1B2835A6902F400625A61C9
:1083E0005A6999690A40160110D55A6902F000626B
:1083F0005A6195F8F423002A40F03782012285F86B
:10840000F4235A6DC2F38302C5F8F8235A699969B7
:108410000A40D00400F1BC805A6999690A4092046C
:1084200058D45A6999690A40170747D45A69996913
:108430000A40D6023DD45A6999690A40940233D45D
:108440005A6999690A40500029D45A6999690A40C1
:1084500051077FF57CAF5C68620700F163835A685F
:1084600014435C6073E7019A02F50061D2F80428B6
:1084700022F001024A6095F8F423012A00F00F82ED
:10848000D5F8042492F89C12042903D192F89D1285
:1084900082F89C125A6902F000425A6190E75A69C8
:1084A00002F080425A61D0E75A6902F400125A6120
:1084B000C6E75A6902F480125A61BCE7D5F8040491
:1084C00090F89C22032A00F031825A6902F00802D7
:1084D0005A61ABE7D3F8000935490140C3F80019E8
:1084E000D3F8041841F48071C3F80418D3F80828AD
:1084F00012F0060140F0C3810193E9600AF0D0FC5C
:10850000EA68019BD1B2022900F0CD81D968B2F1AD
:10851000000821F4705118BF4FF00108D960DA68E3
:1085200042F41052DA60D5F80444402700230126B3
:108530003A46D4F8D002194604F036FF3A460023F2
:10854000D4F8D0028021C4F85861C4F8647104F0F2
:108550002BFF0023D4F8C822A661676284F89C62CE
:10856000C4F894326360C4F8A432002A00F0138384
:10857000D4F8B432204600215B689847D5F804242B
:108580002B6882F810805A6902F400525A6148E759
:10859000019A4FF48460D2F8041802F50066054A87
:1085A00021F001017160186108E000BF8819002402
:1085B00000F8FFFF400D0300013A02D01969890657
:1085C000FAD46F6817B3019A4FF67F3002F5106244
:1085D0009060013411682032BC4221F4001142F84D
:1085E000201C52F8201C41F0006142F8201CC2F807
:1085F000E801D2F8E01121F40011C2F8E011D2F83C
:10860000E01141F00061C2F8E011E1D1F269296B9B
:1086100042F00112F261002900F03781D6F884207F
:1086200042F00B02C6F88420726C42F00B027264B6
:10863000019C1846C24AD4F8001821F4FE63297C34
:10864000C4F8003804F048FB2B685A6902F48052E1
:108650005A61E1E6D3F81828D3F81C1802EA010899
:108660001FFA88F8B8F1000F3FF4A6AE019A4FF058
:10867000000AB44E02F51067029407E05FEA58085A
:108680000AF1010A06F11C0600F0988118F0010FAA
:10869000F4D05FFA8AF9D3F81018D3F8344803F508
:1086A000106209F00F0002EB4912C4409268E40125
:1086B000E4B20C431440E20727D54FF0010E019AB3
:1086C0000AF00F0C07EB4A10D2F834180EFA0CFC23
:1086D00021EA0C01D5F810C0F445C2F83418C0F8EE
:1086E00008E000F03582D5F804B4B9F1000F00F0CD
:1086F0005082DBF8B42252693AB19BF89C120329EC
:1087000003D15846494690472B68200703D507EB0D
:108710004A1208219160E10603D507EB4A121021A5
:108720009160620603D507EB4A1240219160A007D1
:1087300003D507EB4A120221916021069ED5D6E9A6
:10874000140484429AD8011B726C03EB4A1C8A42BF
:108750000CF5106C28BF0A46DCF81810033289B2F9
:10876000B1EB920F2CD309F101099E4603EB0939B5
:1087700028B3844223D2011B726C2B7C914228BF08
:108780001146B26C01F1030B4FEA9B0B73B98BB22C
:1087900003339B080AD002EB830352F8040B9A427E
:1087A000C9F80000F9D1B26CD6E91404DCF818302D
:1087B0000A440C449BB2B26474659B45D8D9734695
:1087C0008442FFF45BAF0AF00F000124D3F83418A1
:1087D00004FA00F021EA0001C3F834184EE7D3F898
:1087E0001828D3F81C180A405FEA124A3FF4DEAD9D
:1087F000DFF850B14FF00009DDF80480029407E083
:108800005FEA5A0A09F101090BF11C0B00F0D48050
:108810001AF0010FF4D05FFA89F603F5306101EB2D
:1088200046108468D3F814281440E70700F1298122
:10883000270700F1C580E70605D508F5306210214D
:1088400002EB49129160A60605D508F53062202199
:1088500002EB49129160A004D2D508F530624FF4C2
:10886000005102EB49129160CAE7D5F804240420B4
:1088700092F89C1282F89C0282F89D12C6E512F0D2
:10888000020F14BF02210F2136E6716942F22B025A
:108890000A437261326942F00B023261C8E600227B
:1088A00085F8F423F6E5284A284902448A4240F232
:1088B0002083274A274902448A4240F23383264ACA
:1088C000264902448A4240F2A083254A25490244AF
:1088D0008A42C0F0B583244A244902448A4240F2C5
:1088E0000F84234A234902448A42C0F01984224A51
:1088F000224902448A42C0F07684214A2149024436
:108900008A42C0F06C84204A204902448A4234BF23
:108910004FF4E0504FF4C050D9684FF0010821F4F3
:108920007051D960DA680243DA60FCE5D0F8B4220D
:10893000D269002A3FF4C9AD90472B68C5E500BF56
:108940004C1D002488190024405327FFFF340C00DD
:10895000401E1BFF3F420F0000DC0BFF7F4F120049
:10896000808CF9FE20D6130060B6E5FE5FE31600AA
:1089700000D3CEFE40771B00C05BB3FEC091210048
:1089800000CA91FE20753800E05459FEE09C410079
:10899000C7EBC70103F58050C2F30A1205EB810152
:1089A0000768D1F81462C5F8C47332440068C1F88E
:1089B0001422C5F8C803EFE4029CF7E4029CFBE430
:1089C00008F53062082003EB491102EB491201F56A
:1089D000306190601B6CD0481A4603938B688242CA
:1089E00004D91E0402D54FF400438B60D5F804640B
:1089F00095F8C4C306F52A7386F8A8C20CF01F07C1
:108A0000059395F8C533012F86F8A93295F8C70369
:108A100095F8C62302EB002291B2A6F8AA1295F8A7
:108A2000C92395F8C80300EB022080B2A6F8AC0277
:108A300095F8CA2395F8CBE304924FF00102C6F8EB
:108A40009422049A02EB0E2292B2A6F8AE22C6F845
:108A5000982200F0F580022F00F0DE80002F00F059
:108A600010810CF080013046FFF702FC039B1A4690
:108A7000A94B9A4203D92969012900F04E822B683B
:108A8000D9E6286908F53062012701EB491102EBAC
:108A90004912012897601F6C8A6800F087809F4800
:108AA000874200F01D82D5F8102259EA020100F039
:108AB0007882C6EBC6033146D5F8040405EB830380
:108AC000D3F8082204F032FC2B68B1E647F6F071C7
:108AD0000A423FF461ACC2F30A10C7EBC7014FEA88
:108AE000C70E0246033005EB81018008D1F80882E9
:108AF0000AD008EB800603F5805C4146DCF80000F4
:108B000041F8040B8E42F9D1AEEB070108EB0206E7
:108B100005EB8101D1F81402C1F808620244C1F8E2
:108B2000142239E4D5F804040122D0F8B43280F8D4
:108B30009C2201795B6898472B6890E4D5F804245F
:108B4000042092F89C1282F89C0282F89D1243E461
:108B5000D6E911120A44B264BAF1000F7FF4C3AD32
:108B60002A6D002A00F0E181D5F804B4AA6CDBF884
:108B70009432022B28D033F0040300F0C9819BF813
:108B8000A032012B7FF4C0AD00222B688BF8A0220D
:108B9000BBE5AA6CEBE7D4F8B832002B7FF4E8AC65
:108BA000D4F8C032002B7FF4E3ACE7E4100740F1C7
:108BB000A381594887427FF63BAE16047FF538AE55
:108BC0004FF400428A6033E6DBE90813994200F271
:108BD000B281DBF81C10B1FBF3F203FB121212B9E5
:108BE0008B4240F21582DBF8B432DB682BB19BF884
:108BF0009C22032A01D15846984780215846FFF706
:108C000037FB00230522DBF8D0021946CBF894226B
:108C10001A4604F0F3FAB2E70CF06007202F00F0D8
:108C20007081402F00F06D81002F00F0BF81802106
:108C30003046FFF71DFB30460021FFF719FB15E713
:108C40000CF06003402B02D01CF0400FEFD196F8DF
:108C50009C32013B022BEAD8C0B20328E7D8D6F8F1
:108C6000B432304605999B689847B6F8AE32002B6F
:108C70007FF4FCAE00287FF4F9AE304604F018FA19
:108C8000F4E60CF0600CBCF1200F00F03A81BCF16E
:108C9000400F00F03681BCF1000F08D08021304633
:108CA000FFF7E6FA39463046FFF7E2FADEE6092B2F
:108CB000BDD801A757F823F0158E04087D8D040850
:108CC0002F8C0408038E04082F8C04089D8D040843
:108CD000498D04082F8C0408258D0408E18C0408B4
:108CE000CFB20F4A012F82F8D873A0D896F89C32E1
:108CF000022B00F04982032B00F0318280213046A4
:108D0000FFF7B6FA00213046FFF7B2FA394630468F
:108D100002F018FDAAE600BF0A30544F0A31544F42
:108D2000685D0024012A82D196F89C32022B00F261
:108D30000E82002B3FF47BAF00233146304641F8D2
:108D4000083F04F0C5F991E60B0A0022013BADF89B
:108D50001E20062B3FF66BAF01A252F823F000BF96
:108D6000D18E0408B78E04089F8E04082F8C040847
:108D70002F8C0408898E0408438E040896F89C32D0
:108D8000013B022B3FF653AF01297FF46FAE002366
:108D90003046C6F8A43204F08BF967E650EA0203C5
:108DA0007FF445AF7F293FF642AF96F89C32032B04
:108DB0003FF43DAFCFB2D6F8D03286F89E7293F82A
:108DC000BC23012A11D01A68002083F83870D2F829
:108DD000007827F4FE67C2F80078D2F8007847EAF6
:108DE0000117C2F8007883F8BC033046049104F000
:108DF0005FF90499002900F00482022386F89C326E
:108E000034E601297FF432AE3046C6F8A41204F0ED
:108E10004FF92BE696F89C32013B022B3FF607AF49
:108E2000022A7FF404AF0122D6F8A432F2600BB11B
:108E30000323F360022206F10C01304604F048F9E6
:108E400014E6337C002B7FF4F2AED6F8B4320DF189
:108E50001E001B6B984707234370BDF81E206AB1A4
:108E6000B6F8AE32002B3FF408AF9A4201463046C6
:108E700028BF1A46ADF81E2004F02AF9B6F8AE3223
:108E8000002B7FF4F3ADF8E6337C002B7FF4CFAEFC
:108E9000D6F8B4320DF11E005B6B9847DDE7CBB21C
:108EA000052B3FF6C4AEDFE813F0F301ED01E70157
:108EB000E101D501CA01337C002B40F0AF81D6F827
:108EC000B4320DF11E009B6A984702234370C4E739
:108ED000D6F8B0320DF11E01307C1B689847BCE714
:108EE00010043FF56DAE93067FF5E3AD20238B6054
:108EF000DFE54FF470500FE590062FD520228A60F1
:108F000096E4D6F8B432304605999B689847ADE5AB
:108F100080215846FFF7ACF931E6D14A286803F0C2
:108F2000DBFEACE54FF46050F6E461461846CC4AEF
:108F300003F0D2FE18E6A1EB030CDBF8D00200210F
:108F40001FFA8CF3CBE9073C04F062F80023DBF84E
:108F5000D0021A46194604F051F910E612F0280F13
:108F60007FF466ACBF48874202D917043FF528AEAC
:108F70000A69DBF80402C2F31202DBF80812821A53
:108F80000144CBF81422D5F81022CBF8081259EA84
:108F900002027FF48EAD1846B14A012103F09CFE17
:108FA00087E51846AE4A03F097FE82E5012B5FFA8B
:108FB00080FC5CD0032B46D0002B7FF46FAE96F87C
:108FC0009C32022B00F0B080032B7FF430AE0306FE
:108FD00000F1E9800CF00F02142303FB0262D2F8C7
:108FE0005871002F3FF45AAE0CF07F0003FB006372
:108FF00003F5AA72002840F01A810023136011467D
:109000003046022204F064F830E54FF4505083E417
:10901000DBF898329942BFF4E6AD0023DBF8D002CA
:109020001A461946CBF81C3003F0F2FF0023DBF898
:10903000D0021A461946CBF8983204F0DFF89EE5C4
:109040004FF4405068E496F89C32022B5BD0032B1F
:109050007FF424AE51EA02037FF40FAE1CF07F0FC1
:109060003FF40BAE61463046FFF702F905E696F88D
:109070009C32022B47D0032B7FF410AE00297FF4E3
:10908000F5AC1CF07F0F3FF4F8ADD6F8D0220CF011
:109090000F01536899423FF6F0AD00064FF01C03F4
:1090A00000F1A58003FB01200027034600F5FE70B8
:1090B00083F8FD7100230170837092F8BC33012B9B
:1090C0003FF4DBAD0121136882F8BC1347780178C7
:1090D000012F0CBF03F5106303F5306303EB41135D
:1090E000196821F400111960C1780239012903D8E7
:1090F000196841F080511960002382F8BC33BCE547
:109100004FF4305008E41CF07F073FF4C7AD6146D0
:109110003046FFF7ADF830468021FFF7A9F8A5E407
:109120004FF42050FFF7F8BB1CF07F0F7FF47FADAA
:1091300002064FF0000330464FF002024CBF06F12A
:10914000140106F5AA710B6003F0C2FF8EE4032B35
:109150007FF46DAD311D304603F0BAFF86E4002F79
:1091600053D0716801293FF488ADC9B2304602F08E
:10917000E9FA3D4A304692F8D813716002F0EAFAF3
:1091800002287FF47AAD52E5002F3FF476AD01213D
:1091900003233046716086F89C3202F0DBFA022825
:1091A0007FF46BAD43E50CF00F03142202FB036365
:1091B0009F69002F3FF472AD0CF07F0303FB022286
:1091C0003244002B3FF419AFD6F8D0121C2000FB1C
:1091D000031393F83E3093B1012313600FE74FF46C
:1091E0000050FFF799BB4FF41050FFF795BB03FBFE
:1091F0000120012703463C3083F83D705AE7136095
:10920000FDE6012386F89C3230E4022339463046DD
:10921000776086F89C3202F095FA2EE5D6F8B432E3
:109220000DF11E00DB6A98470223437015E6D6F85D
:10923000D0321C2000FB0C3393F8FE31CBE7D6F87C
:10924000B0329F69002F3FF429AD0DF11E01307C33
:10925000B84702E6D6F8B0325F69002FF5D11DE5B8
:109260004C1D00240A30544F685D0024D6F8B032FB
:109270001F69002FE9D111E5D6F8B032DF68002F61
:10928000E3D10BE5D6F8B0329F68002FDDD105E5BC
:10929000D6F8B0325F68002FD7D1FFE4000000009D
:1092A00098B182680C4B12B107229A7070471878F7
:1092B0000421DA6003281A611A750CBF80224FF46A
:1092C00080729970C3E901227047034B012283F831
:1092D000E8215A70704700BF085D00240378022B14
:1092E0000FD0006908B9012070470E4B1B78032B83
:1092F00011D080B24FF6F773984294BF002001203E
:109300007047084A4368D2F85422B3EB422F2CBF6F
:10931000012000207047044B984294BF0020012098
:10932000704700BF085D0024F7FFFF0F0378022B92
:109330000FD00C4A4368D2F84C1200690B40D2F8A7
:1093400044120238D2F840225B0A01FB003010447C
:109350007047044B4268D3E98D0100EB410000EBFC
:1093600052207047085D002400487047C8630024FD
:10937000034B93F82400032894BF0020012070477A
:10938000A0630024034B93F82400003818BF012089
:10939000704700BFA063002403460A2201481A80D8
:1093A000704700BF080300240023D0F8C0221846ED
:1093B000137370470346222201481A80704700BF8A
:1093C000140300240346222201481A80704700BF7C
:1093D000380300240346222201481A80704700BF48
:1093E0005C03002403460A2201481A80704700BF2C
:1093F000800300240346432201481A80704700BFBF
:109400008C0300240346432201481A80704700BFA2
:10941000D00300240346432201481A80704700BF4E
:1094200014040024D0F8BC3283B110B5D0F8B8428F
:1094300094F80002FF2807D09B68214694F8012287
:109440009847FF2384F80032002010BD00207047A9
:1094500001F00F01D0F8D022C1EBC10102EB810273
:1094600038B5D0F8B832D0F8BC52D2F8144203F56F
:109470000371EA68D3F80402C3F80C429047002055
:1094800038BD00BF70B40479611E072930D8026866
:109490001B4B1C4E1C4DB24218BF9A4206F12806C7
:1094A0000CBF01230023AA4208BF43F00103283563
:1094B000B24208BF43F001032836AA4208BF43F076
:1094C00001032835B24208BF43F00103AA4208BF96
:1094D00043F0010313B90D4B9A420BD10C4B0D4DC8
:1094E00023449B00012202FA01F1C0E91B354167C8
:1094F00070BC7047084B094D23449B00F2E700BF46
:10950000085402581C5402583054025894540258BB
:109510003F960016405902583F8200104009024011
:109520000368294A294930B4294D2A4CAB4218BF57
:10953000934205F13C050CBF01220022A34208BF63
:1095400042F001023C348B4208BF42F001023C3140
:10955000AB4208BF42F00102A34208BF42F0010241
:109560008B4208BF42F0010212B91B4A934213D149
:10957000DBB21A4D1A4A0121083B1A4CA5FB0353D2
:10958000446602EB1312C3F30413920001FA03F3CF
:109590000266836630BC7047DAB21349134C194433
:1095A000103AA829A4FB02234FEA131300D808336A
:1095B0000F4A03F01F0501210E4C1A44A9404466CE
:1095C000920081660266E5E7085402584454025846
:1095D0001C5402583054025894540258CDCCCCCC70
:1095E0000096001680580258F0FBFDBFABAAAAAA4D
:1095F00000820010800802400268354B354930B4C3
:10960000354C364DA24218BF9A4204F148040CBFB3
:10961000012300238A4208BF43F001034831AA42D4
:1096200008BF43F001034835A24208BF43F00103DD
:1096300048348A4208BF43F0010301F56271AA422F
:1096400008BF43F0010305F56275A24208BF43F06D
:10965000010304F562748A4208BF43F001034831F4
:10966000AA4208BF43F001034835A24208BF43F0B5
:10967000010348348A4208BF43F001034831AA423B
:1096800008BF43F00103A24208BF43F001038A422E
:1096900008BF43F0010313B9114B9A4213D1D3B25F
:1096A0001049114C103BA1FB03515F2B0F4BC1F331
:1096B000021103EA0203615C88BF0433C16583655C
:1096C000184630BC704722F0FF038365F8E700BFFF
:1096D00010000240400002402800024058000240B2
:1096E000B8040240ABAAAAAACCD0090800FCFFFF2C
:1096F000F0B54B780D78012B26D000F530603B4C4F
:109700003B4B00EB45104D69066934400461046928
:10971000234003618B6805B14B610469C3F31203F5
:10972000012A44F400240461046943EA0403036148
:1097300005D0036843F0044303600020F0BDCB680C
:10974000002BF6D04361F4E74C6900F510638CB34D
:1097500003EB4513254FD1F808C0D3F810E0244E91
:1097600064450EEA07071F611F6906EA07061E61C6
:1097700002D96446C1F814C01E69C4F31204012A58
:1097800046F400261E611E6944EA06041C6124D0CA
:109790001A68496942F004421A600029CDD005F0E8
:1097A0000F020125D0F8343895401D43C0F83458D5
:1097B0000020F0BD03EB45130D4EA4F50024012A53
:1097C0001F6906EA07061E611E6946F400261E612F
:1097D0001E6904EA06041C61DAD10A6902B15A6101
:1097E0001A68002042F004421A60F0BD0000F8FF41
:1097F000FFFF07E02DE9F0434D780F78012D4DD0A4
:1098000000F530637A4E4C6903EB4713794D1F69BD
:109810003E401E611E6935401D616CB38D68012A92
:10982000754E2C441F6904F1FF34B4FBF5F41FFAA4
:1098300084FC06EAC44405FB0CF544EA0704C5F3BE
:1098400012051C611C6945EA04051D6121D0CA7816
:10985000012A0AD1D0F8082812F4807F1A680CBFB8
:1098600042F0005242F080521A601A6842F00442FC
:109870001A600020BDE8F0838C68012A1D69C4F3DA
:10988000120444EA05041C611C6944F400241C61B0
:10989000DDD1CA68002ADAD05A61D8E74B6900F5F1
:1098A0001064002B3CD004EB4714D1F808E0DFF83B
:1098B0004091C3F31206D4F8108003EB0E0C08EAB3
:1098C00009090CF1FF3CDFF82C81C4F81090D4F8A2
:1098D0001090BCFBFEFE09EA0808DFF81CC1C4F8C2
:1098E00010800CEACE4CD4F810E04CEA0E0CC4F810
:1098F00010C0D4F810C046EA0C062661CE78012EBE
:1099000047D0012A5FD0226807F00F0342F00442DB
:109910009D402260D0F834783D43C0F83458A8E721
:1099200004EB4714334E324D012AD4F810C00CEA30
:1099300006062661266946F400262661266905EAA0
:1099400006052561CE7833D02568012E45F0044503
:1099500025608ED1D0F8085815F4807F25680CBF9B
:1099600045F0005545F080552560002A81D19BB215
:1099700003339C083FF47DAFCA6800F5805302EBC7
:10998000840403EB073352F8041B94421960FAD1A4
:109990006FE72569012A25F0C0452561256945F055
:1099A0000055256114D0256845F004452560D1E7B0
:1099B0000B695BB9012E0ED02368002043F00443ED
:1099C0002360BDE8F0830B69002BF5D06361F1E7FC
:1099D0000B69002BFAD1D0F8083813F4807F236884
:1099E0000CBF43F0005343F080532360E4E700BF13
:1099F0000000F8FFFFFF07E00000F81F836B5A6DBF
:109A000042F040025A659A6D42F004029A6570472E
:109A1000704700BF836B5A6D12F0500F5A6D1AD108
:109A2000196842F400725A650A6812F0080FCA6891
:109A300016D012F4406F15D1CA68920412D45A6D30
:109A400022F480725A655A6DD1040BD45A6D42F0DB
:109A500001025A657047D20604D4DB6CDB6C1847F0
:109A60009007ECD0704700BF11F0800F4FF01C033F
:109A700001F00F0170B432D103FB0103C1EBC1024D
:109A8000002400EB820203F5FE7382F8FD41197099
:109A900090F8BC23012A31D00121026880F8BC1360
:109AA0005C781D7802F500638C422AD005F00F0423
:109AB000DE6B02F53062A1401C4C02EB451226EA37
:109AC0000146DE63DD6925EA0141D96113681C4066
:109AD0001460002380F8BC33184670BC704703FB49
:109AE0000103C1EBC102012400EB82023C3382F886
:109AF0003D40197090F8BC23012ACDD1022070BCE2
:109B0000704705F00F01DE6B02F510628C400849CA
:109B100002EB451226EA0406DE63DD6925EA040449
:109B2000DC61136819401160D3E700BF0078F3EFE0
:109B3000007833EC0022836BA3F85E20A3F8562054
:109B4000704700BF836B1A6830B4D3F88040D3F8F5
:109B5000840091680D0601D5212C1CD0916849061E
:109B600001D5222807D0D3F8882042F0100230BC5B
:109B7000C3F88820704700240E492025A3F85E40D2
:109B8000106820F490701060906801409160DC666D
:109B9000C3F88450E7E700212024A3F85610116889
:109BA00021F0C0011160916821F400019160C3F8B7
:109BB0008040D3E7FEFFFFEF704700BF704700BF54
:109BC000C369B3F5807F13D0826B00212020136816
:109BD000A2F85E10196821F480711960996821F06B
:109BE00001019960996821F040019960C2F88400F0
:109BF000704700BFC369B3F5807F0CD0826B002132
:109C00001368A2F856109A6822F080029A601A68C7
:109C100042F040021A607047836B00220121A3F8D2
:109C20006A20A3F8622083F881107047F0B43A4D9F
:109C3000AB6A03F00303032B66D02B682A46374C2C
:109C400023F080532B60256803E023685B1B022B05
:109C500057D813689E00F8D4936A056823F07C7384
:109C60002F4E43EA05539362D0E902356F1E013B44
:109C700045685B0205F1FF3C3F0405699BB207F4B0
:109C8000FE07CCF3080C013D3B432D0643EA0C03D1
:109C900005F0FE452B431364D36A456923F4406302
:109CA0002B43D362D36A856923F400732B43D362B9
:109CB000D36A23F48073D362556CC3692E4046EA9D
:109CC000C3065664D36A43F48073D362D36AF1B196
:109CD00001290CBF43F4000343F08073D3620E4BA1
:109CE00019681A4641F080511960216803E0236821
:109CF0005B1A022B05D813689B00F8D50020F0BC36
:109D000070470320F0BC70470120F0BC704743F45B
:109D10008003D362E3E700BF00440258EC4500240F
:109D20000700FFFFF0B43A4DAB6A03F00303032BC7
:109D300066D02B682A46374C23F080632B60256859
:109D400003E023685B1B022B57D813681E01F8D46D
:109D5000936A056823F47C332F4E43EA05339362FC
:109D6000D0E902356F1E013B45685B0205F1FF3CFF
:109D70003F0405699BB207F4FE07CCF3080C013DD4
:109D80003B432D0643EA0C0305F0FE452B4393634A
:109D9000D36A456923F0C0032B43D362D36A856934
:109DA00023F020032B43D362D36A23F01003D36242
:109DB000D56BC3692E4046EAC306D663D36A43F027
:109DC0001003D362D36AF1B101290CBF43F48013AD
:109DD00043F40013D3620E4B19681A4641F08061B8
:109DE0001960216803E023685B1A022B05D8136809
:109DF0001B01F8D50020F0BC70470320F0BC704771
:109E00000120F0BC704743F40023D362E3E700BFB6
:109E100000440258EC4500240700FFFF10B50B4C2E
:109E2000002394F85920236202B1E3654AF0D0FB85
:109E300020B10423022084F8243010BD044A0923F1
:109E4000126884F82430626110BD00BFA063002452
:109E5000DC35002470B50D4D04460E4695F82430CF
:109E6000042B0AD0082B06D1EB6983420CD0FFF7F4
:109E7000D5FF022801D0012070BD08230220C5E9CA
:109E8000074685F8243070BD022070BDA063002411
:109E900038B504468321D0F8D0020025FFF7E4FD51
:109EA000D4F8C002656518B150F046FAC4F8C05243
:109EB000002038BD38B5044600258121D0F8D002F5
:109EC000FFF7D2FD0121D4F8D002E562FFF7CCFD07
:109ED000D4F8D0028221C4F86C51FFF7C5FDD4F844
:109EE000B83225644BB1D4F8BC325B689847D4F8DB
:109EF000B80250F021FAC4F8B852002038BD00BFB3
:109F000038B5442200210F48032550F0B5FA0E4B16
:109F10004FF6FF7010211A78D3F85042022AA3F8A6
:109F2000060203F5F67083F8045218BF2A46C3F8F8
:109F3000104283F8051283F8EC21FBF75DFF012046
:109F400038BD00BFF45E0024085D00242DE9F04117
:109F50004FF0FF302F4C00232246054603E001332B
:109F600010320B2B14D092F82A100429F7D104EBED
:109F7000031191F82B10CF07F1D46E1C116A01D098
:109F80008142ECD21D460133084610320B2BEAD138
:109F90006B1C02D10120BDE8F081AF1C04EB07135C
:109FA0001989D9B92E01DFF87480A219A169D8F8EE
:109FB00060600023D06901EB45213669164AB0473D
:109FC000D0B1022815D1D4F8D03004EB0717012204
:109FD0000020013BBA72C4F8D030DCE7DFF83C80E7
:109FE00004EB05122E01D8F86030D069DB68984781
:109FF000DBE70020BDE8F081D4F8D03004EB071790
:10A0000003210122013BB972C4F8D03084F8D42076
:10A01000C1E700BF085D002439A00408A063002444
:10A02000044B93F8E82112B9012283F8E8210122B8
:10A030005A707047085D002438B5154B00241D4642
:10A04000204683F8D44003E0013010330B2813D0AE
:10A05000DC698C42F8D193F82A40032CF4D162B128
:10A06000AB6903EB40239A4201D0FFF7D9FF05EB20
:10A070000010012380F82A3038BDD5F8D03005EB28
:10A0800000100422013380F82A20C5F8D03038BDF2
:10A09000085D002408B50B46114602070FD50A4A91
:10A0A000581CD2F8C831834204D305D100230120C3
:10A0B0000B6008BDFFF7B4FF0860012008BD18461B
:10A0C000BDE80840FBF76ABE085D00242DE9F041B9
:10A0D0000D46416882B00446C1F308032B44B3F532
:10A0E000007F53D390F91A30591C09D02E4A0233FD
:10A0F000FF2102EB0313DA7A6FF30002DA72817642
:10A1000094F91B305A1C0ED0274A0233FF2002EB71
:10A110000313DA7AC2F34501013921EAE17161F3EF
:10A120004602DA72E0762378022B35D01E4AD2F846
:10A130004432B5EB432F4FEA432823DCD2F84C627C
:10A1400067683E407342AB421CDCAB19434511D3F8
:10A1500001AA2169207EFFF79DFF012812D16768BF
:10A16000A5EB080522694744019B35446261BF1B8A
:10A17000236167602046FFF7B1F820B93D44012014
:10A18000656000E0002002B0BDE8F08129440120B4
:10A19000616002B0BDE8F08161680120294461601E
:10A1A00002B0BDE8F08100BF085D002470B5114E1B
:10A1B0000020334693F82A4014B1DD698D4204D063
:10A1C000013010330B28F5D170BD72B1B36903EBC8
:10A1D00040239A4201D1022C01D0FFF721FF06EB68
:10A1E0000010012380F82A3070BD06EB001080F8C3
:10A1F0002A2070BD085D002470B5154604460E4641
:10A20000FFF764FF50B994F8280028B90223C4E985
:10A210000B5684F8283070BD022070BD1DB1204659
:10A22000A847012070BD012070BD00BF2DE9F84F87
:10A2300002F0020C9B4610B9BCF1000F53D1774DD0
:10A24000D5F83C72002F54D14FF0FF36734F0024E5
:10A25000B146B046B246FB69984200F0A88097F834
:10A260002AE0BEF1000F50D0BEF1010F13D105EB73
:10A27000041E9EF82BE01EF0010F0CD11EF07E0F85
:10A2800009D15FEADE1340F09A80D7F824E0F24566
:10A2900001D9F246A146013410370B2CDBD1741CD6
:10A2A00004D1B8F1FF3F00F091804646D5F8CC408C
:10A2B000B71C05EB061E4FF00009013405EB07182B
:10A2C000CEF81C00C5F8CC40CEF82040C8E90149C2
:10A2D00005EB0714A47A042C00F29B80DFE804F05D
:10A2E0001B3511354C000224FFF79AFE2046BDE8CD
:10A2F000F88FD5E9904606FB0744A042A4D3FFF7A8
:10A300008FFE00242046BDE8F88F26460134103722
:10A310000B2CA0D1C3E712F0010E67D105EB07109B
:10A32000BBF1030F4FEAE20490F80B8064F3C71807
:10A3300080F80B8058D94FF6FF705B46834528BFE5
:10A3400003469BB205EB07100381BCF1000F13D04D
:10A3500005EB061393F82A001C3304280CD0D5F81B
:10A36000CC0004240130C5F8CC0058609C73D5F8AB
:10A37000D0300133C5F8D030500705D505EB0710B4
:10A38000C37A43F00103C372D30608D505EB071760
:10A39000FB7AC3F34502013262F34603FB72AB69F9
:10A3A000012403EB462620460E60BDE8F88FA71C6B
:10A3B00005EB071E9EF80A606EB9264676E7A046B2
:10A3C000013410370B2C7FF446AF68E7B9F1FF3F3B
:10A3D00097D04E466AE7D5F8CC3026465C1CC5F8C7
:10A3E000CC40CEF8044073E77346ABE70C4A002339
:10A3F000A969D2F860C001EB46210A4ADCF808607E
:10A40000B04700283FF47DAF05EB07150223AB7280
:10A410006CE70224FFF704FE68E700BF085D002434
:10A42000A0630024ADA10408B1F904300F2BF0B5EE
:10A430000C4683B0164605462FD02846FEF776FF19
:10A4400095F91B7001467B1C31D02B4B03EB071297
:10A45000D26990420AD0FFF7E3FD2846FEF73EFF9F
:10A46000C0B100230120336003B0F0BD996901EB56
:10A4700047210029F1D0A388284601331BB201EB04
:10A480004311A3803160FEF751FF03460120236092
:10A4900003B0F0BD002003B0F0BD4FF40071FFF732
:10A4A00015FE0028F6D04FF6FF73A380C5E72846B7
:10A4B000FEF714FF0028D0D109B9FFF7B1FD084617
:10A4C0000023112201A9FFF7B1FE0128C5D10A4BD3
:10A4D00001999B69CB1A48BF03F2FF13B3F5B05F34
:10A4E0004FEA632202D257B2EF76C2E7FFF798FD38
:10A4F0000199EF76BDE700BF085D002430B5044642
:10A50000C06983B010B9012003B030BD0D460023EF
:10A51000032201A9FFF78AFE0128F5D1B4F9203002
:10A52000002B03DAFFF77CFD0220EDE7019A012DF5
:10A530004FEA431102EB431303D0022D12D1E5255C
:10A540005554A268DA612278032A04D100221A77CE
:10A550005A779A77DA77626AC2F30F415A839982FF
:10A5600003B030BDE268DA61EDE700BF70B5037893
:10A570000446023B012B037E02D913F0060F55D18E
:10A58000980636D494F91A30591C09D02B4A023354
:10A59000FF2102EB0313DA7A6FF30002DA72A1767D
:10A5A00094F91B305A1C0ED0244A0233FF2002EBD0
:10A5B0000313DA7AC2F34501013921EAE17161F34B
:10A5C0004602DA72E076237E1B0709D51B4D95F80B
:10A5D000CC31072B01D0FFF723FD002385F8CC31C8
:10A5E0000023E26A237084F82830F2B1BDE870409D
:10A5F0001047124D0023E0692A46D1691032884283
:10A6000006D001330B2BBDD0D16910328842F8D16E
:10A61000023305EB0313DA7AC2F34501013921EA6B
:10A62000E17161F34602DA72ACE770BD0121FFF718
:10A6300065FF0128F9D1237EA2E700BF085D002451
:10A64000B8B138B5027822B190F828201AB10020AC
:10A6500038BD012038BD826803244568C162AA4222
:10A6600080F8284038BF2A468260FFF77FFF01202C
:10A6700038BD0120704700BF2DE9F04FDFF844914D
:10A68000174683B08A4699F800300A68022B79D1C0
:10A69000D6B2D9F834524FF48074A6EB020805EB19
:10A6A0001225B844A044BA4208F1FF38B8FBF4F8C8
:10A6B00064D200F0010BA844032B06EB0704A8EBBF
:10A6C00005030CBF80214FF48071A41A8C4228BF6F
:10A6D0000C460EB98C4235D20B2201A92846FFF751
:10A6E000A5FD012802D003B0BDE8F08F99F8001055
:10A6F000DAF80020022902F1010325D0A64210D287
:10A70000019A6FF04040111F304401EB840102EBCD
:10A71000800242F8043F914203F10103F9D1DAF8D3
:10A720000020A61B3244BA42CAF8002002D1BBF175
:10A73000000F37D1BA4205F101051FD299F8003058
:10A740000026B9E70A22C8E7A642EAD201996FF0CB
:10A75000004C881EB44400EB440001EB4C0121F88E
:10A76000023F884203F10103F9D1DAE76FF00043B9
:10A77000019A4FF6FF71234422F81310012003B011
:10A78000BDE8F08F02F07F06032BC2F3D415D9F891
:10A790003412A6EB020814BF4FF4807480240D44D9
:10A7A000B8447FE799F80030022BDFD06FF04043C8
:10A7B000019A4FF0FF31234442F82310DAF80020C9
:10A7C000B8E700BF085D0024F8B590F838300446BB
:10A7D000032B49D8DFE803F0022B343F284BC06835
:10A7E0001A78D3F84412032AD3F8AC51D3F8C8210D
:10A7F0000CBF80264FF48076226101FB06F1971989
:10A8000000EB4120A5EB4125E060D3F8B001C3F88F
:10A81000AC51A0EB4121E06AC3F8C871C3F8B01194
:10A82000C4E90C2748BB6262012384F83830002158
:10A830001448FFF763FE012811D1022384F8383051
:10A84000626B04F130010120FFF716FF012806D1E9
:10A85000032384F8383000212046FFF74FFE431EC3
:10A86000DBB2012B01D9F8BD022094F82830062B69
:10A87000F9D1002384F82830F8BD921B2263D3E776
:10A88000085D0024AC5E00242DE9F04F3D4D012809
:10A8900083B00C462F788CBF4FF0000B4FF0010BAC
:10A8A0001646032F0B682ED0022F51D14FEA1328E2
:10A8B0004FF48079DFB20138012819D84FF0010A2E
:10A8C0009E425CD9D5F8AC211AB1D5F8C81199428D
:10A8D00041D0D5F834020023092201A94044FFF7F2
:10A8E000A5FC012818D0022809D028B12368E7E781
:10A8F00087B1FFF795FB022003B0BDE8F08F02207F
:10A9000003B0BDE8F08F4FF08009C3F3D41803F013
:10A910007F07D0E7CA46D3E7019A2B78022B14D0E1
:10A92000032BECD152F8273023F07043B3FA83F3B2
:10A9300057445B095B4523681FD053444F45236050
:10A94000EBD308F101080027BAE732F81730EDE73A
:10A950004FF48079D9E7D5F84412013A02EB41224D
:10A960004902B2FBF1F21344B3FBFAF20AFB1232D2
:10A970000AB153449B1A2360A2E7B342BCD303201D
:10A980002660B9E7085D0024F0B5104D83B00E468F
:10A990002B78022B15D1070AC4B2D5F83402002354
:10A9A000032201A93844FFF741FC012807D12B7885
:10A9B000022B019B0CBF23F8146043F8246003B002
:10A9C000F0BDC0F3D41700F07F04E6E7085D002473
:10A9D0002DE9F041002990F83C3082B0044614BFC4
:10A9E00002210021042B72D8DFE803F0030C384366
:10A9F0006000FFF783FD012867D1626B002A6CD1EC
:10AA000084F83C00DFF8F0804FF6F776394F1AE013
:10AA1000B54294BF0025012501A9002D43D1FBF7C4
:10AA2000BDF9012829464DD1206BFFF7ADFF012864
:10AA300048D1019AD8F84832511E22638B4228BF70
:10AA40000B46C8F8483298F80030206B032B85B2CB
:10AA5000DED1B84294BF00250125DDE7426B04F149
:10AA600030010020FFF708FE01282ED1032384F8CF
:10AA70003C30214B0021E56AD3F8C82103F5D270A0
:10AA8000C3F8C851551BD3F8442202FB05F2D3E9A1
:10AA90006B6506EB422605EB4222C3E96B62FFF7CA
:10AAA0002DFD012811D1042384F83C3094F828307E
:10AAB000042B02D1002384F82830A36B8BB12046ED
:10AAC0009847012002B0BDE8F0810228FAD194F83D
:10AAD0002830042B09D00220F4E7022384F83C300C
:10AAE000BDE7012002B0BDE8F0810023022084F818
:10AAF0002830E7E7F7FFFF0F085D002438B590F82E
:10AB000034300446052B40D8DFE803F01E03390F2C
:10AB10001863006B4FF0FF31FFF736FF012834D187
:10AB2000E06AA0BB032384F8343000212046FFF7FD
:10AB3000E5FC012829D1042384F8343094F8283026
:10AB4000082B28D0012038BD234D00F13001012011
:10AB5000D5F83C220232FFF797FE012828D00238B0
:10AB6000C0B2012811D8052384F8343094F8283075
:10AB7000082B15D00123022085F8E93138BDC06AC1
:10AB8000216BFFF701FF0128CCD0002038BD022344
:10AB900084F83430F4E70023012084F8283038BDED
:10ABA0000023022084F82830012385F8E931E5E705
:10ABB000D5F84422E368206B03EB4223E26AC5F830
:10ABC0004802C4E9033002B96062012384F83430DA
:10ABD000A0E7014DCAE700BF085D002443682DE9E6
:10ABE000F04F164683B0C3F30808002A00F0DD805A
:10ABF000054689464FF0000BDFF8B8A1C8F5007490
:10AC000095F91A702846B44228BF34467B1C2FD0D1
:10AC1000FEF78CFB0AEB0713DB69984205D0FFF7C0
:10AC2000FFF9584603B0BDE8F08FDAF8180000EBE2
:10AC300047200028F5D0224649464044A3444FF01F
:10AC4000A1FA002221462846FFF7D6FA0028E8D0CC
:10AC50002B7E1B0706D52A69DAF8C8319A4201D340
:10AC6000FFF7DEF9361BA1444FF00008C6D1D8E744
:10AC7000FEF734FB002845D12846FEF757FB6968EC
:10AC8000C1F3080313BB4A4AAB680A4002F50072DD
:10AC90009A422CBF062207222B7E03F00C030C2BBA
:10ACA0001AD0002301A9FFF7C1FA0128B9D10198F0
:10ACB000DAF81830C31A48BF03F2FF13B3F5B05FD8
:10ACC0004FEA63224AD257B2AF76B2E72B7E072211
:10ACD00003F00C030C2BE4D19AF800C0DAF84432EC
:10ACE000BCF1030F0CBF4FF0800C4FF4807C03FBD2
:10ACF0000CF34FEA432C0CF1FF3C0CEA0101A3EBEF
:10AD00005123CFE72B7E1A072DD59AF80020DAF8C9
:10AD10004432032A95F828200CBF80214FF480711B
:10AD2000062A03FB01F34FEA43233FF47AAFDAF834
:10AD3000AC118B4232D89AF8E931002B7FF471AF15
:10AD4000002A7FF46EAF06216B69284685F838200B
:10AD500085F82810EB62FFF737FD1BE0FFF760F97D
:10AD60000198AF7665E795F82830002B7FF459AF4E
:10AD70009AF8E931002B7FF454AF08216A6985F80D
:10AD80003430284685F82810DAF84832EA622B6316
:10AD9000FFF7B4FE01283FF46FAF42E701235846A6
:10ADA0008AF8E93103B0BDE8F08F934639E700BF78
:10ADB00000FEFFFF085D00242DE9F04790F83840C1
:10ADC00082B00546032C00F29A80DFE804F00218F6
:10ADD000610BFFF793FE01280FD0022809D103234E
:10ADE00085F8383000202B6C022485F8280003B148
:10ADF0009847204602B0BDE8F08785F838002B78E8
:10AE0000022B51D03F4A6B68D2F84C2203EA020869
:10AE1000C8F34F282846DFF8EC90FEF787FA06467D
:10AE2000A8EB0008022201A930460023FFF7FEF933
:10AE300008EB060701284FF40072BFB24FF0000183
:10AE4000044606F10106D4D101984FF015FBEB69D9
:10AE50004FF4007128460BB16B685BB3D9F84432EC
:10AE60005A1E974206D2FFF731F90028DAD1FFF7D0
:10AE7000D7F8D7E7C3EBC3532846590201F5007151
:10AE8000FFF724F908B9FFF7CBF8022385F838302B
:10AE900000222B6C85F8282053B1012428469847BE
:10AEA000204602B0BDE8F0876B68C3F34F28B1E7D6
:10AEB00001249EE7019B4FF020322E244FF0100C0E
:10AEC0001A605A601C70C3F80720D5F824E01A6293
:10AED0005A62CEF30F4A83F8204083F82140C3F82A
:10AEE000272083F80BC0EA6BA3F81AE0C2F30F44E3
:10AEF000A3F814A05A879C8683F82BC0AEE70024E1
:10AF000077E700BF085D00242DE9F04790F8303066
:10AF100088B00446042B00F2A280DFE813F0A300FF
:10AF2000AC0005008400E000B24D95F81432002B0F
:10AF300040F0958004F11C0901AEAF4F4FF00908B5
:10AF4000324649463846FFF76FFA012840F0138130
:10AF50000198002800F0F38003780BB1E52BEFD1C6
:10AF6000AA69821A48BF02F2FF12B2F5B05F4FEA37
:10AF7000622380F038811B01A04A13449A7B042A83
:10AF80000CD0D5F8CC2004210132C5F8CC205A6071
:10AF90009973D5F8D0300133C5F8D03095F9063221
:10AFA0005E1C09D00233FF2205EB031385F806224D
:10AFB000DA7A6FF30002DA7295F907325A1C0ED072
:10AFC0000233FF2105EB0313DA7A85F80712C2F387
:10AFD0004501013921EAE17161F34602DA7220226A
:10AFE00000214FF049FA2346019A05A853F8315F32
:10AFF00059681560516019899B7A11819372019B80
:10B00000627EDA7243F08CFABDF81430002B40F007
:10B01000278144F28172019903200A82CB810A833D
:10B02000CB8284F83000237E980600F1A78020466A
:10B03000FAF7E2FE2369002B00F0AC80237E03F0D8
:10B04000F70213F00403227640F0B280122A00F0D7
:10B05000B8800022E36A204684F82820984708B088
:10B06000BDE8F0876448FAF7C7FE4FF6FF72012388
:10B07000228484F8303004F11C0801AE5E4D04F1E6
:10B080003109324641462846FFF7CEF901282DD036
:10B090000228E4D1574D95F906325A1C09D00233E3
:10B0A000FF2205EB031385F80622DA7A6FF300021C
:10B0B000DA7295F907325F1C0ED00233FF2105EBDF
:10B0C0000313DA7A85F80712C2F34501013921EA40
:10B0D000E17161F34602DA72042384F83030002013
:10B0E000E36A2070984708B0BDE8F087019F0B2203
:10B0F00049463846002F00F083803B78002B7FD0F4
:10B1000097F80BA01AF0080FBBD14FF027FC0028CE
:10B11000B7D1637E8AEA0303DB0640F1C280354D76
:10B1200095F906325E1CC4D00233FF2205EB0313EF
:10B1300085F80622DA7A60F30002DA72B9E795F848
:10B14000EC313846022BC7D095F814120029C3D130
:10B15000D5F80022D5F8483285F8148285F82412F3
:10B1600085F82012C5E98A11C5E98623FFF724FE78
:10B1700001283FF4E5AE0228AED070E7002311228B
:10B1800005A9E069FFF752F801283FF450AF08B075
:10B19000BDE8F087237E19077FF55BAF154B93F869
:10B1A000CC21002A7FF45BAF072283F8CC2150E743
:10B1B0000023E26AA168204684F82830FFF71CF8D3
:10B1C0004DE7E56A0421626A204684F83C306363F7
:10B1D000A56384F828106362C4E90233C4E90B2232
:10B1E000FAF70AFE3BE7FEF71BFF01986FF00F032B
:10B1F000C2E600BF085D0024F45E0024245D002444
:10B20000454D95F90632581C09D00233FF2205EB53
:10B21000031385F80622DA7A6FF30002DA7295F9E1
:10B220000732591C0ED00233FF2105EB0313DA7AE3
:10B2300085F80712C2F34501013921EAE17161F392
:10B240004602DA72237EDA067FF546AF3348FAF714
:10B25000D3FD4FF6FF720223228484F8303064E677
:10B260002F4B05A902A8B3F9642043F0AFF99DF86C
:10B270000C309DF80D00DB029DF80A509DF80B2064
:10B28000BDF8081043EA401342EA45129DF80E004B
:10B29000A1F2BC7143EA500342EA41229BB292B24E
:10B2A000B9E6BB8A7A8B1C4D42EA0342D5F8443298
:10B2B00062625A02FB69B3FBF2F102FB1131A36037
:10B2C00009B113445B1AE36084F819A095F90632BA
:10B2D000581C09D00233FF2205EB031385F8062220
:10B2E000DA7A6FF30002DA7295F90732591C0ED040
:10B2F0000233FF2105EB0313DA7A85F80712C2F354
:10B300004501013921EAE17161F34602DA72032352
:10B3100084F8303087E600BF085D0024F45E002426
:10B32000A06300242DE9F04190F8283082B0044653
:10B33000013B082B43D8DFE803F04A054F545A6716
:10B34000426C45003A4BD0F80480D3F84C62016B54
:10B3500008EA0606D3F844328A195F02B2EB432F9B
:10B3600018D25BE02169207EFEF794FE012826D1E9
:10B37000216B6368C91B226907EB0308019B3144F9
:10B380006261A8EB060823618F422E46C4F8048050
:10B39000216343D82046FDF7A1FF01AA05460028F6
:10B3A000E0D0D4F80480A3680021E26A434584F821
:10B3B000281038BF4346A3600AB12046904702B028
:10B3C000BDE8F081FFF7F8FC02B0BDE8F081FFF7BF
:10B3D0009BFD02B0BDE8F081FFF7C8F802B0BDE800
:10B3E000F0810021FFF7F4FA02B0BDE8F0810121FD
:10B3F000FFF7EEFA0128E2D10023216C204684F801
:10B400002830FFF71DF9DAE7FFF7DEF902B0BDE8F3
:10B41000F081FFF773FB02B0BDE8F0812046FDF735
:10B420005DFF0028BFD18844C4F80480BBE700BF9B
:10B43000085D0024014B1B6E1B6A1847A0630024A3
:10B44000024B186E08B1836918477047A063002447
:10B4500010B5074C606D40B13AF088F894F851305F
:10B4600013B180F00100C0B210BD012010BD00BFBB
:10B47000A063002410B54379164C002B14BF0122A1
:10B48000002284F8502019D094F86930003B18BF8E
:10B49000012384F85930FFF7DBFF28B9237E84F8B5
:10B4A00024000133237610BD48F08CF948B1237E87
:10B4B0000022013384F82420237610BD84F8243040
:10B4C00010BD054B012220761B6884F8242063619F
:10B4D00010BD00BFA0630024DC35002410B548F087
:10B4E00071F948B10A4C237E0133DBB2072B237676
:10B4F00003D9002384F8243010BDFFF7A9FF0028EA
:10B50000F7D0044B01221B6884F82420636110BD2E
:10B51000A0630024DC3500242DE9F84F864C94F814
:10B520005050002D00F0ED8094F82420834E844F7D
:10B53000531E082B37D8DFE803F02C2F94365A42DD
:10B540001436050049F044F8002840F0EC806369A7
:10B550003268FA33934223D2FFF7C0FF94F82420D5
:10B56000E6E749F035F80028F1D0236A0022012BE4
:10B57000227640F2DC80E169013B94F859500131B8
:10B58000C4E9071305B1E2650823054684F82430B1
:10B5900012E0022384F8243049F01AF8002845D13B
:10B5A00094F82420531EDBB2022B35D9082A18BF89
:10B5B000042A0CBF012500252846BDE8F88F604B02
:10B5C0005B6A002B2ED15D4B0722E5681B6884F86F
:10B5D00024206361002DEFD023690120D4E90021EC
:10B5E000A847DDE763693268643393421AD2D7F81B
:10B5F0002080B8F1000FF5D148F0EAFF0028ADD067
:10B600000423E56884F8188084F82430002D00F0C5
:10B61000888040462369E1E7484B62691B689B1AB2
:10B62000C82B73D800252846BDE8F88F48F06EFE79
:10B630000028B5D194F86D30002BA3F10203B3FAC2
:10B6400083F314BF022201225B096276A37648F0DD
:10B650005DFE002880D1D4F8B8200323A26284F8CC
:10B66000243048F053FE8246002899D194F89C106B
:10B670004FF0040EB4F89EB00323D4F8A020C4F811
:10B6800020A0D4F8A0704FEA126CD4F8A06084F81F
:10B690002E103F0CD4F8A090360A94F8A48094F8A9
:10B6A000A55094F8A520D4F8A80025FA0EF5B4F812
:10B6B000AEA002F00F02B4F8AE1084F83160C1F30E
:10B6C0000B11B4F8AE6084F8385041EA1A2106F044
:10B6D0000F0584F83920724601F00F01A4F82CB050
:10B6E00084F82FC001F5FA6184F8307084F8329044
:10B6F00084F833806063618784F83C5084F824E0E8
:10B7000051E7284684F82450BDE8F88FFFF7E6FE9D
:10B7100094F82450082D18BF042D0CBF01250025D6
:10B720004AE7054648E7042384F8243044E7FAD181
:10B73000FEF774FB34E700BFA0630024DC3500246F
:10B74000004A002408B5D0F8B4325B68984700205E
:10B7500008BD00BF08B5D0F8B4321BB11B689847CC
:10B7600000B908BD022008BDF0B5D2E9023615695E
:10B7700033435669224C2B439569645C3343D66945
:10B78000204F2B43956A334306592B433740D66AE3
:10B7900005193B430351AEB16F69D2F838C027F0A9
:10B7A0000707D2E90C3E1E433E436E61065926F060
:10B7B000C07646EA0E060651035923F4C00343EA55
:10B7C0000C030351176A566AD2E900340E4AEC6042
:10B7D000AB6090426B684FF001000C4C04EA03042C
:10B7E0000B4B0B4444EA07044FEA83036C6018BF19
:10B7F00020331A6822F0FF0232431A60F0BD00BF06
:10B8000010D109081F80FCFF000002400000FFFF6C
:10B810000082001070B46A4C0D1E6A4A0346645CD4
:10B8200018BF0125821A005918BF012220F001001B
:10B83000185132BB2DBB6448644A002421250A44B8
:10B840000460446092008460C460046145611068D3
:10B8500020F0FF00106021B93F2201209A6070BCE7
:10B860007047012932D002292BD0032944D0042962
:10B8700047D0052934D006294BD0072955D00020C0
:10B88000EDE75348181A18BF01209DB990B95148E7
:10B890008D00514A002421262A44046044608460BB
:10B8A000C46004614661106820F0FF001060002948
:10B8B000D7D1D1E74C1E18BF01246AB964B94748F3
:10B8C000BAE74FF47C1201209A60C8E74FF4746223
:10B8D000084670BC9A60704738B934B94048D7E719
:10B8E0004FF474620120DA60B9E78C1E18BF01249E
:10B8F0005AB954B93B489FE74FF0746201209A60EF
:10B90000ADE73F220120DA60A9E738B934B93648FB
:10B91000BEE74FF47C120120DA60A0E7CC1E18BF0E
:10B9200001243AB934B9314886E74FF074620120F6
:10B93000DA6094E710B90CB92D48A9E70C1F18BFBD
:10B94000012412B90CB92B4876E710B90CB92A4872
:10B950009EE74C1F18BF012412B90CB927486BE7AA
:10B9600010B90CB9264893E78C1F18BF012412B9EF
:10B970000CB9244860E710B90CB9234888E7114A8C
:10B98000934203D1072901D1204855E70F4A0024EB
:10B990000C4D21260A441E48AB424FEA8202046045
:10B9A000446018BF20328460C4600461466110683E
:10B9B00020F0FF00106000297FF453AF4CE700BF78
:10B9C00010D109080000024010000240008200105F
:10B9D00000040240100402402008024028000240F7
:10B9E0002804024040000240400402405800024047
:10B9F0005804024070000240700402408800024077
:10BA000088040240A0000240A0040240B8000240A6
:10BA1000B80402402DE9F0479F4A00259F4E82B0AE
:10BA2000036882469E49846D934218BFB3420195D4
:10BA300008BF01260D68276818BF002621684AD074
:10BA40003032DFF86CE29748734518BF93420EF12D
:10BA5000480E0CBF01220022834208BF42F00102BF
:10BA60003030734508BF42F001020EF1300E8342C0
:10BA700008BF42F0010200F55C70734508BF42F058
:10BA800001020EF55C7E834208BF42F001023030B5
:10BA9000734508BF42F001020EF1300E834208BF29
:10BAA00042F001023030734508BF42F001020EF14E
:10BAB000300E834208BF42F001023030734508BFA8
:10BAC00042F00102834208BF42F001021AB9764AED
:10BAD000934240F00B82DAF85C10082201F01F0C50
:10BAE00002FA0CF2174240F08D8127FA0CF2D207CD
:10BAF0000CD55A69100609D5012202FA0CF2A2608F
:10BB0000DAF8542042F00202CAF854204FF0040E32
:10BB10000EFA0CF038425BD0002E4FD1634ADFF8AA
:10BB20009091DFF880814B4518BF934209F1480995
:10BB30000CBF01220022434508BF42F0010208F178
:10BB400030084B4508BF42F0010209F13009434576
:10BB500008BF42F0010208F55C784B4508BF42F08F
:10BB6000010209F55C79434508BF42F0010208F182
:10BB700030084B4508BF42F0010209F13009434546
:10BB800008BF42F0010208F130084B4508BF42F0FF
:10BB9000010209F13009434508BF42F0010208F1F2
:10BBA00030084B4508BF42F00102434508BF42F050
:10BBB00001021AB93C4A934240F02F821A68920758
:10BBC00006D5A060DAF8542042F00402CAF85420E6
:10BBD000102202FA0CFC1CEA070F6FD0002E46D18F
:10BBE000324A33482F4E834218BF934200F1480037
:10BBF0000CBF01220022B34208BF42F001023036DE
:10BC0000834208BF42F001023030B34208BF42F025
:10BC1000010206F55C76834208BF42F0010200F59E
:10BC20005C70B34208BF42F001023036834208BF65
:10BC300042F001023030B34208BF42F00102303618
:10BC4000834208BF42F001023030B34208BF42F0E5
:10BC500001023036834208BF42F00102B34208BFFE
:10BC600042F001021AB9104A934240F0DE811A688C
:10BC7000C2F3C00212B3C4F808C01A68520300F13C
:10BC80008B811A68D60503D41A6822F008021A605C
:10BC9000DAF8403093B10DE0280002401000024075
:10BCA000F800002470000240B8040240580002402E
:10BCB0004000024050469847DAF85C1001F01F013E
:10BCC00020268E403E426AD0DAF80020A74BA848D2
:10BCD000A84F824218BF9A4200F130000CBF0123E6
:10BCE0000023BA4208BF43F001033037824208BF45
:10BCF00043F001033030BA4208BF43F0010330374C
:10BD0000824208BF43F001033030BA4208BF43F01B
:10BD1000010307F55C77824208BF43F0010300F599
:10BD20005C70BA4208BF43F001033037824208BF5B
:10BD300043F001033030BA4208BF43F0010330370B
:10BD4000824208BF43F001033030BA4208BF43F0DB
:10BD500001033037824208BF43F00103BA4208BFF3
:10BD600043F001031BB9844B9A4240F0738113687E
:10BD7000C3F300139BB1A6609AF83530042B136807
:10BD800000F0148113F4802F136800F02D811C0340
:10BD900040F13881DAF83C300BB150469847DAF878
:10BDA0005430002B00F0DF80DAF85430D8071FD56C
:10BDB000DAF8002004248AF83540136823F00103E0
:10BDC00013606E4BA3FB0535AD0A02E01368D9077B
:10BDD00004D5019B0133AB420193F7D900238AF8C4
:10BDE00034301368DB074CBF032301238AF8353056
:10BDF000DAF84C30002B00F0B680504602B0BDE8B7
:10BE0000F0471847186840070AD5186820F0040062
:10BE10001860A260DAF8542042F00102CAF85420F7
:10BE200027FA0CF2D2077FF571AE554A5148DFF878
:10BE30006481834218BF934200F148000CBF012285
:10BE40000022434508BF42F0010208F13008834256
:10BE500008BF42F001023030434508BF42F0010202
:10BE600008F55C78834208BF42F0010200F55C707F
:10BE7000434508BF42F0010208F13008834208BF81
:10BE800042F001023030434508BF42F0010208F1A0
:10BE90003008834208BF42F001023030434508BFFA
:10BEA00042F0010208F13008834208BF42F001026B
:10BEB0003030434508BF42F00102834208BF42F0E0
:10BEC0000102002A7FF415AE002E7FF412AE042288
:10BED0001E6802FA0CF23A4240F09F80102202FAE9
:10BEE0000CFC17EA0C0F3FF4E9AE79E6254A264E22
:10BEF000264DB34218BF934206F128060CBF01221B
:10BF00000022AB4208BF42F001022835B34208BF0D
:10BF100042F001022836AB4208BF42F00102283548
:10BF2000B34208BF42F00102AB4208BF42F0010237
:10BF300012B9174A934216D1DAF85C5004261A68EF
:10BF400005F01F05AE400E4273D0570771D510049F
:10BF5000666040F19F80D10300F1A280DAF848309A
:10BF6000002B7FF44AAF02B0BDE8F087100002401A
:10BF70002800024040000240B8040240B5814E1B38
:10BF800058000240085402581C54025830540258B9
:10BF900094540258700002401B681B037FF578AE72
:10BFA000DAF84830002B7FF485AE87E623F01603DD
:10BFB000DAF840501360536923F0800353613DB3B6
:10BFC000136823F0080313603F230025012203FABE
:10BFD00001F1DAF85030A1608AF834508AF835203F
:10BFE000002B7FF40AAFBEE713F480737FF4D2AE68
:10BFF0001168012421F0100111608AF834308AF8A8
:10C000003540C7E6DAF84430002B7FF4C6AEC6E60A
:10C01000DAF84830002BD3D1D6E710221E6802FA96
:10C020000CFC17EA0C0F3FF449AE1A68C2F3800209
:10C0300020E60226AE400E4210D097070ED566606D
:10C04000140433D5D0033DD4DAF84430002B7FF408
:10C05000D4AE88E71368C3F340038BE60826AE40EE
:10C060000E4280D011077FF57EAF196801220026AD
:10C0700021F00E0102FA05F51960DAF84C3065601E
:10C08000CAF854208AF834608AF83520002B7FF4EF
:10C09000B4AE68E7920603D41A6822F004021A606C
:10C0A000DAF84030002B7FF4A8AE5CE712F02002F3
:10C0B00008D11968012421F00A0119608AF8342096
:10C0C0008AF83540DAF83C30002B7FF496AE4AE728
:10C0D000002860D038B590F835200346022A56D1A2
:10C0E0000168594A914249D01832914246D03032C3
:10C0F0005648574C814218BF914200F14800554DB7
:10C100000CBF01220022A14208BF42F001024834C4
:10C11000814208BF42F0010200F56270A94208BFE7
:10C1200042F0010205F56275A14208BF42F001022A
:10C1300004F56274814208BF42F001024830A9420E
:10C1400008BF42F001024835A14208BF42F0010297
:10C150004834814208BF42F001024830A94208BF7A
:10C1600042F00102A14208BF42F00102814208BF31
:10C1700042F0010212B9384A91420ED10422002045
:10C1800083F835200B6823F001030B6038BD802253
:10C1900001205A6538BD0120704704F1C0542F4A70
:10C1A0002F4804F59F442F4DA14218BF914204F13E
:10C1B00050040CBF01220022814208BF42F001025C
:10C1C0000868A94208BF42F0010220F00E0028359D
:10C1D000A14208BF42F00102086028340868A94261
:10C1E00008BF42F0010220F00100A14208BF42F066
:10C1F0000102086012B91C4A914217D11C6E01213C
:10C20000D86D226800F01F009D6D22F4807281407D
:10C21000586E2260D3E91A426960446032B11168F5
:10C22000186F5C6F21F4807111604460002401215B
:10C230001A6D83F8344083F835101AB118469047C8
:10C24000204638BD104638BD100002404000024074
:10C2500070000240A0000240B80402401C54025882
:10C26000305402584454025894540258002800F0A4
:10C270008A812DE9F047044690F83400012800F047
:10C280008481012094F83550854284F8340007D029
:10C2900000224FF4006384F834206365BDE8F08722
:10C2A00025684FF0020C58480027584E84F835C0D6
:10C2B000B54218BF8542DFF85CC106F130066765FC
:10C2C0000CBF01200020524F654508BF40F001001F
:10C2D0000CF1300CB54208BF40F0010006F5627663
:10C2E000654508BF40F001000CF5627CBD4208BF07
:10C2F00040F0010007F56277B54208BF40F0010049
:10C300004836654508BF40F001000CF1480CBD42BD
:10C3100008BF40F001004837B54208BF40F00100B7
:10C320004836654508BF40F001000CF1480CBD429D
:10C3300008BF40F00100A7F58F67B54208BF40F085
:10C340000100A6F58F66654514BF824640F0010ADC
:10C35000B54218BFBD420CBF0126002602D0BAF17B
:10C36000000F59D02F68D4F858C027F001072F606C
:10C37000002E00F08480676ED4E91A0E7860BEF15A
:10C38000000F02D0D4E91C707860E76D4FF03F09D0
:10C39000D4F8088007F01F07B8F1400F09FA07F733
:10C3A000CCF808702F6827F480272F606B6000F0AE
:10C3B000EF80A960EA601EB9BAF1000F00F0EE80CC
:10C3C0002B68226C23F01E0343F016032B601AB176
:10C3D0002B6843F008032B60236E1A68D20303D541
:10C3E0001A6842F480721A60BEF1000F05D0DEF8C0
:10C3F000003043F48073CEF800302B68002043F007
:10C4000001032B60BDE8F087400002405800024065
:10C41000B800024070000240654FDFF89CE1DFF891
:10C420009CC1754518BFBD420EF13C0E0CBF0127E3
:10C430000027654508BF47F001070CF1280C75453A
:10C4400008BF47F001070EF1280E654508BF47F009
:10C4500001070CF1280C754508BF47F00107D5F816
:10C4600000E0654508BF47F001072EF0010ED4F843
:10C4700058C0C5F800E017B94E4FBD420DD1676EE8
:10C48000D4E91A0E7860BEF1000F02D0D4E91C7016
:10C490007860BAF1000F7FF478AF474FDFF8108172
:10C4A000DFF818E1454518BFBD4208F128080CBF68
:10C4B00001270027754508BF47F001070EF1280E38
:10C4C000454508BF47F0010708F12808754508BF32
:10C4D00047F001070EF1280E454508BF47F0010758
:10C4E000754508BF47F0010717B9324FBD4255D116
:10C4F000E76D4FF0010ED4F8088007F01F07B8F180
:10C50000400F0EFA07F7CCF804706B6043D0A960B7
:10C51000EA602B68226C23F00E0343F00A032B60C1
:10C52000002A2DD02B6843F004032B60204B224AB5
:10C530002249954218BF9D4202F13C020CBF0123E3
:10C5400000238D4208BF43F001032831954208BF04
:10C5500043F0010328328D4208BF43F00103283124
:10C56000954208BF43F0010328328D4208BF43F0D3
:10C570000103954208BF43F00103002B3FF43DAF98
:10C58000D4F86CE028E7012070470220BDE8F0876E
:10C59000AA60E9600FE7AA60E960BAE72B68226C3D
:10C5A00023F00E0343F00A032B60002ABAD1BDE743
:10C5B0001C540258945402580854025830540258DB
:10C5C00038B50446864B87492268874D8A4218BF92
:10C5D0009A42864801F160010CBF01230023AA4260
:10C5E00008BF43F001034835824208BF43F001030E
:10C5F00000F562708A4208BF43F0010301F56271E1
:10C60000AA4208BF43F0010305F56275824208BFE4
:10C6100043F0010348308A4208BF43F00103483128
:10C62000AA4208BF43F001034835824208BF43F0E5
:10C63000010348308A4208BF43F001034831AA424F
:10C6400008BF43F00103824208BF43F001038A425E
:10C6500008BF43F001033BB9A1F59561644B9A42D1
:10C6600018BF8A4240F0CE80116800232125204661
:10C6700021F001011160136053609360D360136176
:10C680005561FCF7B9FFE26D3F2302F01F029340B2
:10C6900083602268574B5649524D8A4218BF9A42CE
:10C6A0004F4801F148010CBF01230023AA4208BFF3
:10C6B00043F001034835824208BF43F0010348308C
:10C6C0008A4208BF43F001034831AA4208BF43F041
:10C6D000010305F56275824208BF43F0010300F5CE
:10C6E00062708A4208BF43F0010301F56271AA42F9
:10C6F00008BF43F001034835824208BF43F00103FD
:10C7000048308A4208BF43F001034831AA4208BFBB
:10C7100043F001034835824208BF43F0010348302B
:10C720008A4208BF43F0010301F1C051AA4208BF89
:10C7300043F0010301F59F412F4D824208BF43F0B2
:10C7400001032E488A4208BF43F001033C31AA424C
:10C7500008BF43F001033C35824208BF43F00103A8
:10C760003C308A4208BF43F001033C31AA4208BF73
:10C7700043F00103824208BF43F001038A4208BF2D
:10C7800043F0010313B91E4B9A4211D12046FCF726
:10C79000C7FE236E23B10020D4E91921186051602F
:10C7A0006368013B072B11D90023C4E91B3363677E
:10C7B00000236365184684F8353084F83430C4E9C2
:10C7C0000F33C4E91133C4E9133338BD2046FCF7F5
:10C7D00059FEE16E0020D4E91C3208605A60E3E79C
:10C7E00058000240400002407000024088000240B1
:10C7F00028000240100002401C54025830540258D5
:10C80000945402581D4B1E491E4D8A4218BF9A422D
:10C810001D4801F13C010CBF01230023AA4208BFBF
:10C8200043F001033C35824208BF43F001033C3032
:10C830008A4208BF43F001031168AA4208BF43F0CF
:10C84000010321F00101824208BF43F0010311609E
:10C8500013B90E4B9A420FD1002320461360536048
:10C860009360D3601361FCF7C7FEE26D012302F011
:10C870001F02934043600CE7012038BD0854025862
:10C880001C540258305402584454025894540258CC
:10C89000A549F8B504460868002C00F065812268B7
:10C8A000A24B9A4249D018339A4246D03033A04E18
:10C8B000A04DB24218BF9A4206F148060CBF0123B0
:10C8C0000023AA4208BF43F001033035B24208BF3B
:10C8D00043F001033036AA4208BF43F0010305F5D7
:10C8E0005C75B24208BF43F0010306F55C76AA42CC
:10C8F00008BF43F001033035B24208BF43F00103E3
:10C900003036AA4208BF43F001033035B24208BFB7
:10C9100043F001033036AA4208BF43F0010330352B
:10C92000B24208BF43F00103AA4208BF43F001032B
:10C930001BB9814B9A4240F03C810223002584F8C8
:10C94000353084F83450136823F00103136004E099
:10C950000B681B1A052B00F2BF801368DD07F7D4A4
:10C96000D4E9023120690B431768D4E90516034363
:10C970000B437249D4E90705334339400343606AE6
:10C980002B43042841EA030100F0AD801160536994
:10C9900023F00703184350612046FCF72DFEE26D9B
:10C9A0003F2302F01F029340836022685F4B64497B
:10C9B0005F4D8A4218BF9A42624801F148010CBF9C
:10C9C00001230023AA4208BF43F0010348358242F5
:10C9D00008BF43F0010348308A4208BF43F0010317
:10C9E0004831AA4208BF43F0010305F5627582424F
:10C9F00008BF43F0010300F562708A4208BF43F0AC
:10CA0000010301F56271AA4208BF43F001034835F2
:10CA1000824208BF43F0010348308A4208BF43F016
:10CA200001034831AA4208BF43F00103483582425E
:10CA300008BF43F0010348308A4208BF43F00103B6
:10CA400001F1C051AA4208BF43F0010301F59F4123
:10CA50003D4D824208BF43F001033C488A4208BF73
:10CA600043F001033C31AA4208BF43F001033C35C7
:10CA7000824208BF43F001033C308A4208BF43F0C2
:10CA800001033C31AA4208BF43F00103824208BFC0
:10CA900043F001038A4208BF43F0010313B92C4B52
:10CAA0009A4213D12046FCF73BFDA368802B5DD052
:10CAB0006368206EDDB2013BD4E91921072B0560C4
:10CAC000516047D90023C4E91B3363670020012369
:10CAD000606584F83530F8BD2022032301206265AB
:10CAE00084F83530F8BDD4E90B50A36A28430143DC
:10CAF0001160506920F00700184340F00400002D39
:10CB00003FF449AF002E39D1012B4DD033F0020351
:10CB10007FF441AFEB017FF53EAF01234022184681
:10CB2000626584F83530F8BDEC4500241000024001
:10CB30004000024070000240B80402403F8010FEF6
:10CB400028000240580002401C5402583054025839
:10CB5000945402582046FCF795FCE16E0020D4E97D
:10CB60001C3208605A60B1E70120F8BD0023A16EB5
:10CB7000D4E91802636003605160A3E7B6F5005F73
:10CB800004D0022BC9D9032BC4D004E7032B3FF6F2
:10CB900002AF01A151F823F01BCB040815CB040808
:10CBA0001BCB0408A9CB0408B5F1C07F7FF4F3AE1A
:10CBB000B3E7344B344935488A4218BF9A4201F1F1
:10CBC0002801334D0CBF01230023824208BF43F0EC
:10CBD00001033C308A4208BF43F001033C31AA42C2
:10CBE00008BF43F00103824208BF43F001038A42B9
:10CBF00008BF43F0010313B9264B9A423AD10223EE
:10CC00000021254F84F83530A36884F83410402B78
:10CC1000116807EA01072BD0802B0CBF4FF480412D
:10CC2000002123692046E668DB086569DFF870C0EB
:10CC300043EAD603A66943EAD503E56943EAD60386
:10CC4000164E43EAD5031644256A43EA1513ACFB96
:10CC500006653B432D091943AD001160E565FCF7FE
:10CC6000CBFCE26D012302F01F02934043609CE67F
:10CC70001021D6E7402203230120626584F8353075
:10CC8000F8BD00BF085402581C54025830540258D2
:10CC900058540258945402580F00FEFFF8ABFDA7F9
:10CCA000CDCCCCCC0B4B01E0013B10D00269002A6B
:10CCB000FADA0369074A43F00103036101E0013A2C
:10CCC00005D0036913F00103F9D11846704703201A
:10CCD000704700BF400D0300144B10B4046C9C421D
:10CCE0001AD800F53060002301290361036943F479
:10CCF00000230361036943F018030361036943F0F0
:10CD0000C043036104D14261036843F080230360A0
:10CD100000205DF8044B7047D0F8003B00F5306010
:10CD2000002BE0DA00205DF8044B70470A30544FC6
:10CD3000002807DB00F01F0101234009024A8B4055
:10CD400042F82030704700BF00E100E02DE9F04FCD
:10CD50000D6883B0002D00F0C4800023DFF82C8222
:10CD6000DFF82CE201229A4012EA050C00F0B480B0
:10CD70004C6824F01007022F40F0B680DF0803F063
:10CD8000070A4FF00F0B0E6900EB87074FEA8A0A7C
:10CD9000D7F820900BFA0AFB06FA0AF64FEA430A84
:10CDA00029EA0B094FF0030B46EA09090BFA0AF6C8
:10CDB00004EA0B0BC7F820906FEA060907680BFA24
:10CDC0000AFB27EA06064BEA060606608768C4F3F4
:10CDD000001607EA090BCF689E4007FA0AF747EAF0
:10CDE0000B078760476827EA020216434660C66859
:10CDF000E7008A6806EA090902FA0AF242EA090229
:10CE0000C26069D5D8F8F47023F0030903F0030277
:10CE10000F2647F0020709F1B0499200C8F8F470F4
:10CE200009F58069D8F8F47006FA02FA07F00207EB
:10CE300001974D4F019EB842D9F8086026EA0A06CC
:10CE400020D007F58067B8426BD0484FB8426DD00C
:10CE5000474FB84260D0474FB84271D0464FB842B2
:10CE600073D0464FB84266D0454FB84272D0454F56
:10CE7000B84274D0444FB8420CBF09270A2707FABA
:10CE800002F21643C9F808606FEA0C07DEF80020CA
:10CE9000E60354BF3A404CEA0202CEF80020A20357
:10CEA000DEF804604FF0B04254BF3E404CEA060644
:10CEB000CEF804601668E2024FF0B04254BF3E4024
:10CEC0004CEA0606A4024FF0B0441660526854BF04
:10CED0003A404CEA02026260013335FA03F27FF411
:10CEE00041AF03B0BDE8F08F4FEA430A4FF00309AA
:10CEF000D0F800B0013F04EA090609FA0AF9012F47
:10CF00002BEA090B06FA0AF66FEA090946EA0B064C
:10CF100006603FF66CAF59E7032707FA02F21643A3
:10CF2000B0E7012707FA02F21643ABE7022707FA38
:10CF300002F21643A6E7062707FA02F21643A1E714
:10CF4000042707FA02F216439CE7052707FA02F2C4
:10CF5000164397E7072707FA02F2164392E70827D6
:10CF600007FA02F216438DE7000002580008025843
:10CF7000000C025800100258001402580018025801
:10CF8000001C025800200258002402580044025895
:10CF90008000005802689168890702D593680020D4
:10CFA00070479168CB070ED59168034601F00D01DB
:10CFB00001290AD0426D012042F010025A659A6D93
:10CFC00002439A6570470020704730B40E4903242D
:10CFD00095680E48294041F0020191601460046890
:10CFE00003E00168091B022905D89168C907F8D434
:10CFF000002030BC70475A6D012042F010025A6583
:10D000009A6D02439A65F4E7C0FFFF7FEC45002468
:10D01000F8B501F00F05012600271C21C5EBC5045A
:10D0200001FB050100EB84043C31A264236584F814
:10D030003C50676584F83D600369B34208BFE26411
:10D04000DAB200681DB9FCF753FB0020F8BDFCF70D
:10D05000D1FB0020F8BD00BFF8B5D0F8B8322BB333
:10D0600001EB8107064600EB8707FA695AB1D0F851
:10D07000D0C2C1EBC1040CEB8404606CB2FBF0F4D1
:10D0800000FB14241CB10020C3F81402F8BD01F009
:10D090007F05FC616046234605EB8505224606EBCD
:10D0A0008505EC61FFF7B4FF2046F8BD0220F8BD0E
:10D0B00010B504210024C0F894122346C46122460E
:10D0C0002146D0F8D002FFF7A3FF204610BD00BFD5
:10D0D00010B5134602240A460021C0F89442C0E964
:10D0E0000733D0F8D002FFF793FF002010BD00BF38
:10D0F00010B50C7882B00023D0F8C02214F0600480
:10D10000ADF8063016D0202C0ED14B78023B092BFF
:10D110000AD8DFE803F033390909090909093F2F63
:10D1200090F89C32032B5AD00224FBF7FDF82046DE
:10D1300002B010BD4B780B2BF6D80FF2080C5CF840
:10D1400023F000BFC9D1040829D1040829D104085B
:10D1500029D1040829D1040829D104089FD1040841
:10D1600029D1040829D1040829D1040821D10408AF
:10D17000BBD104088B7800241360D8E7111D01226D
:10D180000024FFF7A5FFD2E7114601220024FFF794
:10D190009FFFCCE74B8800241B0A5360C7E74B88EE
:10D1A0001B0A222B1FD0212BBED1CA881149092A64
:10D1B00028BF0922FFF78CFFB9E790F89C32032BB8
:10D1C000B2D18B789360B2E790F89C22032AABD15E
:10D1D00002220DF106011C46FFF77AFFA7E702F1D4
:10D1E00008010122E6E7CA880349362A28BF362209
:10D1F000E0E700BF900400245804002470B5C1EBA0
:10D20000C1040D4600261C2100EB840401FB05012E
:10D21000C4F80822C4F8103201F5FE7184F8FC51FC
:10D22000C4F8146284F8FD610369012B08BFC4F8D7
:10D230000C22DAB200681DB9FCF75AFA002070BD62
:10D24000FCF7D8FA002070BD2DE9F0410A7882B0D1
:10D2500000270D4612F060060446D0F8B8828DF81B
:10D260000570ADF8067013D0202E17D1CB88EBB126
:10D27000120641D5D0F8BC621A4641466878B368B8
:10D280003E469847EA8841462046FFF721FF09E0DD
:10D290004B780A2B21D00B2B29D093B120460226A4
:10D2A000FBF742F8304602B0BDE8F081D0F8BC424E
:10D2B0001E461A464878A3689847304602B0BDE833
:10D2C000F08190F89C32032B2AD002262046FBF7EF
:10D2D0002BF8304602B0BDE8F08190F89C32032B69
:10D2E000F3D101220DF10501FFF7F2FEDAE790F824
:10D2F0009C32032BD6D0E8E74A78032588F8013220
:10D30000394688F800224246C0F85C313E46C0F8F3
:10D310006031D0F8D002C4F89452FFF76FFFC1E734
:10D3200002220DF10601FFF7D3FEBBE770B50546FB
:10D3300041B9D0F894320C46032B10D0052B1FD0E6
:10D34000002070BDD0F8B4329B6933B190F89C22B4
:10D35000032A02D19847002070BD022070BDD0E999
:10D3600058639E4212D8D0F8B4321B6923B190F8AA
:10D370009C22032A00D198472846FFF799FEDFE751
:10D38000C5F89412FAF774FF204670BDF61AD0F86B
:10D39000D002B342C5F8606128BF33469BB2FFF7A5
:10D3A0002DFF204670BD00BF11F0800F01F00F016E
:10D3B000F0B44FF01C0442D1C1EBC10504FB0104E1
:10D3C000002600EB850504F5FE7485F8FD6165789F
:10D3D0002170A260E37005B1E180022B01D100232E
:10D3E000237190F8BC33012B53D00122036880F8DD
:10D3F000BC236178257891422CD003F5006605F0B6
:10D400000F0103F530638A40F16903EB451341EAEC
:10D410000242F2611A68120405D5002380F8BC3379
:10D420001846F0BC7047A2681D68C2F30A02E4788F
:10D4300019492A4342EA844211431960EDE7C1EBDE
:10D44000C105012604FB010400EB85053C3485F889
:10D450003D60BCE705F00F06D3F81CC803F5106269
:10D4600003F50067B14002EB451241EA0C01F96196
:10D4700013681904D1D4A3681668C3F30A03E478C7
:10D480000549334343EA844343EA85531943116012
:10D49000C3E70220F0BC70470080001010B50323E2
:10D4A000044608228321D0F8D002FFF77DFF012334
:10D4B000102063654CF038FFC4F8C00218B1002397
:10D4C0000373184610BD022010BD00BF2DE9F041C6
:10D4D000037C04460125002B3CD102234FF400724B
:10D4E0008121D0F8D002FFF75FFF294602234FF4D5
:10D4F0000072D4F8D002E562FFF756FFC4F86C5111
:10D500004FF00108032308228221D4F8D002FFF74C
:10D510004BFF4FF40770C4F840804CF005FF054600
:10D52000C4F8B80278B3D4F8BC3200271B68984717
:10D53000267CC5F814724146D5F80422D4F8D002EE
:10D54000C5F81872C6B140233E46FFF757FE304675
:10D55000BDE8F081022340228121D0F8D002FFF7FC
:10D5600023FF294602234022D4F8D002E562FFF7C8
:10D570001BFFC4F86C51C3E74FF40073FFF73EFE86
:10D580003046BDE8F0814646E1E700BF154B014655
:10D5900041F288321B6810B4134CA4FB03035B0AEE
:10D5A00002FB03F24AB1531E4A6B013B12F0450FD6
:10D5B00001D0920406D5581CF6D14FF000405DF81A
:10D5C000044B70474B6B5B0709D4486B5DF8044B09
:10D5D00010F0010014BF0123044B8B63704704203B
:10D5E0008863ECE7F8000024D34D6210C5002000EA
:10D5F000474B10B41B68474CA4FB03435B0A02FB78
:10D6000003F24AB1531E444C426B013B224201D00B
:10D61000920407D55A1CF7D14FF0004318465DF825
:10D62000044B7047436B5C073DD4436B13F001031D
:10D6300034D13A4B83630369DBB2994231D14269F9
:10D64000374B1340002BE9D0002A2FDB510030D498
:10D65000940030D4D00030D4110131D4540132D4EC
:10D66000D00133D4110234D4540235D490023FD4C3
:10D67000D1023AD4540335D4900330D4D10343D4E7
:10D6800014043ED4500439D4910434D412F0080F59
:10D6900014BF4FF400034FF48033BFE701228263CD
:10D6A000BCE70123BAE704238363B7E74FF00073B5
:10D6B000B4E74023B2E78023B0E74FF48073ADE7CF
:10D6C0004FF40073AAE74FF48063A7E74FF40063B9
:10D6D000A4E74FF48053A1E74FF400539EE74FF4C3
:10D6E00080239BE74FF4003398E74FF4004395E71E
:10D6F0004FF4804392E74FF480038FE74FF4001319
:10D700008CE74FF4801389E74FF4002386E700BFCE
:10D71000F8000024D34D621045002000C500200011
:10D7200008E0FFFD70B4816041F23714C66841F231
:10D730008832034D372135402C43C46070BC57E715
:10D74000C0E0FEFF114B0146114A186841F28833D0
:10D7500030B4104C0025A4FB00408D60CC68400A1A
:10D76000224003FB00F342F48052CA6002E04A6B9D
:10D77000120605D4013BFAD24FF0004030BC70478E
:10D78000054B002030BC8B63704700BFF8000024BD
:10D79000C0E0FEFFD34D6210C5002000C16841F219
:10D7A0000C130E4A41F0800170B5C1600026C168BB
:10D7B00004460B4D21F04001C1600C218660C66813
:10D7C00035402B43C360FFF713FFE368B0F1007FE0
:10D7D00008BF002023F08003E36070BD00E1F50581
:10D7E000C0E0FEFF70B4816041F21014C66841F2DF
:10D7F0008832034D102135402C43C46070BCF7E6DD
:10D80000C0E0FEFF2DE9F84F5B4D06460C46904602
:10D8100095F824C01F46BCF1040F09D0BCF1080FD5
:10D8200002D00020BDE8F88FFCF7F8FA0228F8D102
:10D830000122524B52484FF400719A600262C3E9D0
:10D840000041002C40D0DFF840B19BF83030012B74
:10D8500028D1731CDBF8502000209342CBF8340011
:10D860002BD80322DBF800308BF83020DBF838208F
:10D87000D8621846012ACBE909414FF4007114BF60
:10D880004FEA462AB246FFF7ADFFDBF8003008B397
:10D890003C4901229963DBF834301843CBF834005B
:10D8A0008BF83020FDF71AFEEC68002CB9D000226E
:10D8B0002B6969681046A047B3E7DBF8343043F0C2
:10D8C0000073CBF83430EDE72F4A536B43F000631D
:10D8D0005363E7E74FF0FF314FF4007259629A62E9
:10D8E00001301F28FCD9DA6A81204FF0010927494D
:10D8F00022F0FF0241F2111C42F09202DA62DA6871
:10D9000042F04002DA609C65C3F85090CBF82C00DE
:10D910001846C3F808A0DA68114041F2883241EA9B
:10D920000C0C1121C3F80CC0FFF762FE70B1DBF8DC
:10D930000030002213499963DBF834301843CBF8E8
:10D9400034008BF83090CBF82C20ABE7DBF80020CC
:10D950000521DFF83CC04846D36B2C6043F4957337
:10D960006E60C5F80C80D363DCF8003085F82410B5
:10D97000C5E90473BDE8F88FA0630024304A002491
:10D98000004A0024FF0FE01F84490024C0E0FEFF8E
:10D99000DC3500242DE9F047064682B00D4691465D
:10D9A0009A468C4C94F8241004290CD0082906D1EE
:10D9B000E369B34207D0FCF731FA0228F2D0012024
:10D9C00002B0BDE8F087D4F85C802560C8F34F272B
:10D9D0004FEA582266600F2F03D8236A0193002B69
:10D9E00068D101204FF4007807460123DFF8F8C121
:10D9F000062225F01F012372CCF8243005EB080322
:10DA0000C4F80C905B1AC4F810A084F82420BFF36B
:10DA10004F8F002B0EDD013B01F12002DFF8CCC15E
:10DA200023F01F0313449A42CCF86812114602F106
:10DA30002002F8D1BFF34F8FBFF36F8F002D6BD053
:10DA4000DFF89C9199F83030012B26D13044D9F879
:10DA5000503000229842C9F834204ED8D9F83830D6
:10DA60000321D9F80000012B89F830104FF4007120
:10DA7000C26218BF7602C9E90758FFF7B3FE002853
:10DA800050D0D9F80020012353499163D9F83420AC
:10DA90001043C9F8340089F83030FDF71FFDE56800
:10DAA000002D00F095800120236900226168A847BD
:10DAB000032085E794F85910002992D0B8F5005F4B
:10DAC00022D046484FF40072294608F500774044BA
:10DAD0004CF058FB019B7A0AE765012BC7F34F27EF
:10DAE00012D0102F10D0E269013B04210220013234
:10DAF000236284F82410E26162E7D9F8343043F0FD
:10DB00000073C9F83430C8E792B238464FEA472864
:10DB1000324D013AB61A68E7314A536B43F000635D
:10DB20005363BAE7D9F800304FF0FF325A62C3F8B6
:10DB3000288001301F28FCD9DA6A012122F0FF0277
:10DB40008F4242F09002DA62DA6842F04002DA6014
:10DB50009D65196521D9A022224941F2191518465F
:10DB6000C9F82C209E60DA68114041F288320D43DA
:10DB70001921DD60FFF73CFD08B3D9F80010012240
:10DB8000154D00238D63D9F834100843C9F83400CB
:10DB900089F83020C9F82C307FE79022114941F2F2
:10DBA00018151846C9F82C209E60DA68114041F219
:10DBB00088320D431821DD60FFF71AFDDCE7D9F844
:10DBC0000020D36B43F48D73D36302B0BDE8F087BC
:10DBD0000320F5E6A0630024FF0FE01F7464002417
:10DBE00084490024C0E0FEFF004A002400ED00E06C
:10DBF000034A0130116813685B1A8342FBD37047F4
:10DC0000EC45002438B5114B114A1B68A2FB0323D5
:10DC10009B09013BB3F1807F0CD20E4A05460E49A9
:10DC2000F0205360002407230F2D81F82300946017
:10DC3000136001D9012038BD29464FF0FF30F3F7BA
:10DC40007DF8064B2046C3F8945138BDF8000024F7
:10DC5000D34D621010E000E000ED00E00803002466
:10DC600038B50021144A03680446C0F888101568C6
:10DC700019680A070CD41B685B0713D42022002301
:10DC8000C4F880201846C4F8842084F87C3038BD5D
:10DC90002A464FF40011F3F7B1FC58B923681B680A
:10DCA0005B07EBD52A464FF480012046F3F7A6FC2C
:10DCB0000028E3D0032038BDEC450024836ADA074E
:10DCC00010B406D50168C46A4A6822F400322243BF
:10DCD0004A609C0706D50168046B4A6822F48032CA
:10DCE00022434A60590706D50168446B4A6822F40A
:10DCF000802222434A601A0706D50168846B4A686D
:10DD000022F4004222434A60DC0606D50168C46B57
:10DD10008A6822F4805222438A60990606D50168F7
:10DD2000046C8A6822F4005222438A605A060AD59B
:10DD30000168446C4A68B4F5801F22F4801242EAFC
:10DD400004024A600BD01B0606D50268C16C5368FA
:10DD500023F400230B4353605DF8044B70474A687B
:10DD6000846C22F4C00222434A60ECE70368344921
:10DD70005A6910B49C6944F008049C619C6944F0A1
:10DD800010049C611C6824F001041C601C69214083
:10DD90001961996821F44041996090F88110042933
:10DDA00001D0940633D490F8811003290FD0510686
:10DDB00009D5D0F8841041F00401C0F884109969A5
:10DDC00041F040019961816AB1F5800F2AD0910537
:10DDD00009D5D0F8841041F00101C0F88410996988
:10DDE00041F400719961D20509D5D0F8842042F040
:10DDF0000802C0F884209A6942F480729A61002374
:10DE00005DF8044BA0F86230A0F86A307047D0F893
:10DE1000841041F08001C0F88410996941F020011C
:10DE20009961C0E71406D2D5D0F8841041F0020100
:10DE3000C0F88410996941F080019961C7E700BF7B
:10DE400090FCFFFF036819695A69D3F808C02DE9EF
:10DE5000F04101EA0205044690F8817005F064067D
:10DE6000042E4AD005F0450001284FD005F02600C9
:10DE7000022800F0C88028075BD59A691CF4404F3F
:10DE800042F008029A619A6942F010029A619A6916
:10DE900042F400629A611A6922F008021A6108D0FD
:10DEA000FFB2042F00F0BF80A26FD269002A40F0B9
:10DEB000B7809A6812F4404F31D1B4F86A2092B218
:10DEC0006AB3616E0EE02268126B41F8042B616642
:10DED000B4F86A20013A92B2A4F86A20B4F86A2031
:10DEE00092B2E2B1E2680F2AEDD8072A40F29080A0
:10DEF0001A8E21F8022B6166EAE7436F9847236F79
:10DF00002046984705F04503012B02D1236F204698
:10DF1000984705F02605022D75D0BDE8F081204612
:10DF2000FFF724FF012384F88130D4F88430BDE862
:10DF3000F081120501D50F077BD415F4587FECD082
:10DF40006E0609D5D4F8842042F00402C4F8842077
:10DF50009A6942F040029A61A80509D5D4F8842054
:10DF600042F00102C4F884209A6942F400729A6176
:10DF7000E90509D5D4F8842042F00802C4F88420C9
:10DF80009A6942F480729A61AA0609D5D4F884206D
:10DF900042F08002C4F884209A6942F020029A611B
:10DFA000D4F88420002AB8D019680CF4404C254AD3
:10DFB00021F00101BCF5404F1960196902EA010224
:10DFC0001A613BD19A68E06F22F440429A6050B1E6
:10DFD0001D4B0365FEF77CF828B1D4F8843043F07C
:10DFE0004003C4F88430A06F002896D0164B036518
:10DFF000FEF76EF8002890D0D4F8843043F0400348
:10E00000C4F8843089E7636F2046BDE8F0411847C3
:10E01000226892F830200A70616E0131616657E71C
:10E02000032F3FF47AAFE26FD269002A3FF441AF89
:10E0300073E79A6942F400629A616EE7012384F8FB
:10E0400081306AE794FCFFFF199C04080346022113
:10E05000002210B41C68104683F88110216821F05A
:10E0600001012160C3F8842083F8802083F8812097
:10E070005DF8044B704700BF8449034602682DE9F0
:10E08000F04F834CA24218BF8A42C46814BF0121DA
:10E09000002129D07F48824226D00F2C21D8D3F8E6
:10E0A0003CC004F108004FEA5C15C00805FB000005
:10E0B000082816D89D6A4FF0000BB5F5800F33D1B4
:10E0C000744ED3F83080B24203D011B1B8F5702F3E
:10E0D00007D8B8F1000F01D14FEA0448B4EB184F4C
:10E0E00024D90120BDE8F08F694804F10805674E86
:10E0F000D3F83CC0ED08B24218BF8242654F4FEAE8
:10E100005C160CBF0120002006FB0555BA4214BF67
:10E11000834640F0010BBBF1000F01D0102DE0D879
:10E120009D6AB5F5800FCBD04FF0000893F8816061
:10E1300006F0FF07002E00F0A08002269F69D3F8AA
:10E1400004E083F88160B7F1806F1668D3F83890E7
:10E1500026F00106166000F083805E6BB5F5800F37
:10E16000986847EA060A5F6A1E694AEA070746EAAC
:10E1700007065F6946EA07061F6A46EA0706DF6C7C
:10E1800046EA07069F6C46EA0006D86947EA060792
:10E1900045EA000A9E6D4AEA0C0C46EA07064CEA7C
:10E1A000040446EA090644EA080446EA0E069460B6
:10E1B000D66029D0BEF1000F14D0116D1EF4800F6F
:10E1C00021F00101116505D0D168586D21F00041A1
:10E1D0000143D16000200122C3F8840083F881202C
:10E1E000BDE8F08F2DB9916821F4C05141F4006170
:10E1F0009160916821F4C06141F480619160116D7A
:10E2000021F001011165E5E71C6C012C14680CBFBD
:10E2100044F4004424F4004414605C6C012C146841
:10E220000CBF44F4804424F480441460194CA2428E
:10E230000CBF002101F0010111B1B8F5702F1FD002
:10E24000BBF1000F02D0B8F5F81F19D0116821F406
:10E2500000511160D96A1164BEF1000FC9D0ACE75A
:10E26000BEF5800F7FF479AFB9F1000F7FF475AF81
:10E27000166846F4805616606FE783F880705CE796
:10E28000116841F400511160E4E700BF003800401C
:10E2900000300140003C004008B504F013FE064B7E
:10E2A00006499B69064AC3F30323CB5C03F01F03B3
:10E2B000D840106008BD00BF00440258BCD0090817
:10E2C000F80000244F4B70B4996A9D6ADC6A15F01F
:10E2D0007C7FC5F305525E6C5CD0C6F3CC06C4F3FC
:10E2E000002401F0030104FB06F4012907EE904A23
:10E2F000B8EEE77A03D0022975D000294FD007EE97
:10E30000902ADFED416AF8EEE77A1B6C86EEA76A89
:10E31000DFED3E5AC3F3080306EE903AB7EE005A1B
:10E32000F8EEE66A76EE856AE7EE256A66EE266A1C
:10E33000344AB7EE006A136CC3F3462307EE103A73
:10E34000B8EEC77A70BC37EE067AC6EE877AFCEE76
:10E35000E77AC0ED007A136CC3F3064307EE103A78
:10E36000B8EEC77A37EE067AC6EE877AFCEEE77A21
:10E37000C0ED017A136CC3F3066307EE903AF8EE32
:10E38000E77A77EE867A86EEA77ABCEEC77A80EDDA
:10E39000027A704770BCC0E9002282607047196839
:10E3A000890627D5196807EE902A194AF7EE004A20
:10E3B000C1F3C101F8EEE77A1B6CCA409FED135A16
:10E3C000C3F3080306EE102A06EE903AF8EEC65A9A
:10E3D000F8EEE66A85EEA76A76EEA46AE7EE056ACD
:10E3E00066EE266AA4E707EE902ADFED0A6AF8EEE9
:10E3F000E77A8AE707EE902ADFED076AF8EEE77A18
:10E4000083E700BF004402580024744A000000392A
:10E410000090D0030024F44A0024744C4F4B70B495
:10E42000996A9D6ADC6A15F47C3FC5F30532DE6BA0
:10E430005CD0C6F3CC06C4F3001401F0030104FB66
:10E4400006F4012907EE904AB8EEE77A03D00229D4
:10E4500075D000294FD007EE902ADFED416AF8EE23
:10E46000E77A9B6B86EEA76ADFED3E5AC3F308039B
:10E4700006EE903AB7EE005AF8EEE66A76EE856A56
:10E48000E7EE256A66EE266A344AB7EE006A936BB9
:10E49000C3F3462307EE103AB8EEC77A70BC37EEE6
:10E4A000067AC6EE877AFCEEE77AC0ED007A936BC7
:10E4B000C3F3064307EE103AB8EEC77A37EE067A92
:10E4C000C6EE877AFCEEE77AC0ED017A936BC3F370
:10E4D000066307EE903AF8EEE77A77EE867A86EEF4
:10E4E000A77ABCEEC77A80ED027A704770BCC0E9AB
:10E4F0000022826070471968890627D5196807EEDF
:10E50000902A194AF7EE004AC1F3C101F8EEE77A02
:10E510009B6BCA409FED135AC3F3080306EE102A03
:10E5200006EE903AF8EEC65AF8EEE66A85EEA76A6D
:10E5300076EEA46AE7EE056A66EE266AA4E707EEC1
:10E54000902ADFED0A6AF8EEE77A8AE707EE902A6A
:10E55000DFED076AF8EEE77A83E700BF0044025870
:10E560000024744A000000390090D0030024F44ACB
:10E570000024744C08B504F093FC054B054A1B6A53
:10E58000C3F30213D35C03F01F03D84008BD00BFE0
:10E5900000440258BCD009082DE9F04383680446C2
:10E5A000B04D87B0E169B04ED0E904201A4323682A
:10E5B00002431F68606EB34242EA010205EA0705A2
:10E5C000A76942EA0002E06842EA05021A605A6856
:10E5D00022F4405242EA00025A6000F0A680986895
:10E5E00006F16846226AA14D06F582363A43054097
:10E5F000606AB34242EA05029A60DA6A22F00F02C8
:10E6000042EA0002DA6225D0994A934257D0994AE9
:10E61000934200F02D82984A934200F09982974AE3
:10E62000934200F0F181964A934200F09B82954A12
:10E63000934200F0D785944A934200F0B3850125B8
:10E6400000234FF0011228462367C4E91A2307B0BC
:10E65000BDE8F0838D4B5B6D03F03803282BEED8BB
:10E660008B4A13441D7AB1F5004F35D0202D00F2AE
:10E67000D581202D00F2BA80DFE815F09A016D01F6
:10E68000B800B8006401B800B800B8003B01B80099
:10E69000B800B800B800B800B800B8000E01B80063
:10E6A000B800B800B800B800B800B800B800B800AA
:10E6B000B800B800B800B800B800B800C400734B88
:10E6C0005B6D03F00703052BB9D8714AB1F5004F14
:10E6D000134493F83450C9D1202D00F20E82202D1E
:10E6E00000F2FA81DFE815F01204D403F801F80112
:10E6F000A403F801F801F8010204F801F801F80197
:10E70000F801F801F801F8016E03F801F801F801C9
:10E71000F801F801F801F801F801F801F801F80131
:10E72000F801F801F801F8013F0399684F4A57488A
:10E730000A403A439A60DA6A616A22F00F020A4399
:10E74000DA62836D03F00703052B3FF678AF504A7A
:10E75000134493F83C60202E00F29481012E7FF642
:10E760006EAFB31E1E2B3FF66AAF01A252F823F024
:10E7700053ED04083FE60408E7EC04083FE604080C
:10E780003FE604083FE604083DED04083FE60408C0
:10E790003FE604083FE604083FE604083FE60408B5
:10E7A0003FE604083FE6040889EC04083FE6040855
:10E7B0003FE604083FE604083FE604083FE6040895
:10E7C0003FE604083FE604083FE604083FE6040885
:10E7D0003FE604083FE604083FE604083FE6040875
:10E7E0003FE604083FE6040891EB040801250023F6
:10E7F000A3F110014FF6EF7291423FF620AF22686D
:10E80000D3601DE7002800F09F84012800F0B08548
:10E81000022800F0C385032800F0E885042800F0F2
:10E820000D86052800F07086062800F0AF860728C0
:10E8300000F0F486082800F08087092800F09C8703
:10E840000A2800F0F18743F60953124A0B2818BF33
:10E8500013466268002503EB5203B3FBF2F39BB24D
:10E86000C6E700BFF369FFCF000C0058FFF4FF11AB
:10E870000044004000480040004C00400050004070
:10E880000014014000780040007C00400044025821
:10E89000CCD0090800093D00B74B1A68920640F138
:10E8A0005A841A68B54BC2F3C102D3400028D0D0B5
:10E8B000012800F08584022800F0CC84032800F0B1
:10E8C000C684042800F04185052800F084860628C7
:10E8D00000F0EB86072800F00C86082800F03D8643
:10E8E000092800F081860A2800F0EE860B28B0D1B6
:10E8F00026E06846FFF7E6FC626A019B002AA8D082
:10E90000012A00F05D84022A00F0A484032A00F0AA
:10E910009E84042A00F01985052A00F01385062A32
:10E9200000F09D85072A00F0E485082A00F015868E
:10E93000092A00F059860A2A00F0C6860B2A88D1D7
:10E940001B0A86E703A8FFF769FD626A049B002A99
:10E950003FF47FAFD4E704F073FA636A03B3012B8B
:10E9600000F01285022B00F0EA84032B00F0E4840F
:10E97000042B00F02D85052B00F02785062B00F0D9
:10E98000F585072B00F03B86082B00F0BC86092B91
:10E9900000F0DA860A2B00F05D870B2B08BF000A17
:10E9A0006268002500EB5203B3FBF2F39BB21FE752
:10E9B00004F05EFA636A03B3012B00F0DE84022BDD
:10E9C00000F0C984032B00F0C384042B00F00685FB
:10E9D000052B00F00085062B00F0C285072B00F008
:10E9E0001A86082B00F09B86092B00F0C2860A2BA2
:10E9F00000F017870B2B08BF000A626800EB520378
:10EA0000B3FBF2F39BB2F3E65B4B5B6D03F00703E2
:10EA1000052B3FF614AE5A4AD55C24E6402D7FF410
:10EA20000EAE002800F09383012800F0A98402288C
:10EA300000F0B984032800F0DC84042800F001858C
:10EA4000052800F05D85062800F09C85072800F069
:10EA5000DE85082800F05F86092800F09C860A28D9
:10EA600000F014870B280CBF80234FF40043F0E61E
:10EA7000414B5B6D03F00703052B3FF6E0AD414AC8
:10EA8000D55CF0E5402E7FF4DAAD002900F09583E7
:10EA9000012900F08084022900F09484032900F009
:10EAA000C484042900F02185052900F04B8506293E
:10EAB00000F09685072900F01186082900F0558698
:10EAC000092900F08B860A2900F0C7860B290CBFA4
:10EAD00080254FF4004582E001250023A3F11001B9
:10EAE0004FF6EF7291423FF6AAAD23F00F02C3F347
:10EAF000420321681343CB60A2E5402D7FF49FAD14
:10EB0000002800F06083012800F05F83022800F0F5
:10EB10008284032800F0DB84042800F00D8505289A
:10EB200000F05085062800F0CC85072800F00F86FD
:10EB3000082800F03886092800F09D860A2800F091
:10EB400000870B280CBF4FF480714FF480313CE3F9
:10EB5000094B5B6D03F00703052B3FF670AD0A4AC6
:10EB6000D55C80E5044B5B6D03F03803282B3FF642
:10EB700066AD064AD55C76E5004402580090D003A5
:10EB800000D1090800D1090800D10908D4D009082A
:10EB9000002900F06F83012900F0F983022900F0B9
:10EBA0000C84032900F04584042900F09884052989
:10EBB00000F0CC84062900F00B85072900F08B8536
:10EBC000082900F0DF85092900F0E9850A2900F00D
:10EBD000378643F60955C94B0B2918BF1D46676890
:10EBE00007EB4703AB423FF62AADB5EB073F3FF6D5
:10EBF00026AD202E00F20183012E7FF620ADB31E3C
:10EC00001E2B3FF61CAD01A252F823F0DBF00408E6
:10EC10003FE60408C9F004083FE604083FE604089C
:10EC20003FE6040859F004083FE604083FE60408FC
:10EC30003FE604083FE604083FE604083FE6040810
:10EC40003FE60408D7EF04083FE604083FE604085F
:10EC50003FE604083FE604083FE604083FE60408F0
:10EC60003FE604083FE604083FE604083FE60408E0
:10EC70003FE604083FE604083FE604083FE60408D0
:10EC80003FE6040867EF04089D4B1A68950640F1BB
:10EC9000F3821B689B4DC3F3C103DD4000299ED066
:10ECA000012900F0B383022900F0AA83032900F0B0
:10ECB000A483042900F07F84052900F0B684062986
:10ECC00000F03685072900F08685082900F0BF8509
:10ECD000092900F0FC850A2900F0E6850B297FF45C
:10ECE0007EAF2D0A7BE703A8FFF798FB636A049DBC
:10ECF00003B3012B00F0B982022B00F0B182032B89
:10ED000000F0AB82042B00F02E83052B00F028834B
:10ED1000062B00F09A83072B00F0F983082B00F0F4
:10ED20002B84092B00F065840A2B00F0FB840B2B4D
:10ED300000F05382002D3FF483AC50E76846FFF7A4
:10ED4000C1FA636A019D002BD3D1002D3FF478AC4A
:10ED500045E7FFF70FFC636A0546002BC9D1002D7C
:10ED60003FF46EAC3BE7002800F0AA82012800F0D7
:10ED70001E83022800F04D83032800F0A683042898
:10ED800000F0D883052800F00D84062800F0928456
:10ED9000072800F0DF84082800F03785092800F0F4
:10EDA00049850A2800F0D08547F61223564A0B28D9
:10EDB00018BF13466268002503EB5203B3FBF2F35E
:10EDC0009BB28BE64E4B1A68910640F18F821A680F
:10EDD0004C4BC2F3C10223FA02F200B3012800F047
:10EDE0004483022800F09B83032800F0D483042886
:10EDF00000F05584052800F08184062800F0DD84A9
:10EE0000072800F04785082800F04785092800F00A
:10EE10007F850A2800F079850B2808BF120A6168EF
:10EE200000254B0803EB4203B3FBF1F39BB255E61D
:10EE300003A8FFF7F3FA626A049902B3012A00F00B
:10EE40009A82022A00F0AD82032A00F0CA82042AC4
:10EE500000F0F282052A00F04F83062A00F0798341
:10EE6000072A00F0D283082A00F03C84092A00F027
:10EE70008F840A2A00F002850B2A08BF090A6268FB
:10EE80000025530803EB4103B3FBF2F39BB225E6E5
:10EE900003F0D6FF636A03B3012B00F08C82022BD0
:10EEA00000F0BC82032B00F00B83042B00F03E83A8
:10EEB000052B00F08383062B00F00984072B00F05C
:10EEC0004F84082B00F09384092B00F0B6840A2BA2
:10EED00000F00C850B2B08BF000A616800254A086A
:10EEE00002EB4003B3FBF1F39BB2F7E56846FFF793
:10EEF000E9F9626A0199002AC1D09FE700093D0043
:10EF0000004402580090D00300127A0003F0B0FFD2
:10EF1000636A03B3012B00F04C82022B00F0808265
:10EF2000032B00F0D782042B00F00283052B00F0A6
:10EF30003E83062B00F0C183072B00F00E84082BC4
:10EF400000F05284092B00F07F840A2B00F0BC846F
:10EF50000B2B08BF000A61684A0802EB4003B3FBB1
:10EF6000F1F39BB2BAE5636A03B3012B00F04A8365
:10EF7000022B00F0BD83032B00F03C84042B00F037
:10EF80004C84052B00F09C84062B00F09484072B06
:10EF900000F08D84082B00F0E984092B00F0058532
:10EFA0000A2B00F0FE840B2B00F0F784C5480021EB
:10EFB0007D0800233A46401941F100014CF0B2FAB5
:10EFC000A0F54073C04A93423FF639AB2368002551
:10EFD000D860FFF735BBBD4B1A68900640F14A82F6
:10EFE0001A680021BA48C2F3C102636AD0400BB369
:10EFF000012B00F0C583022B00F0F483032B00F0FB
:10F000000784042B00F08D84052B00F08484062BEC
:10F0100000F0DA84072B00F0D484082B00F0CD84B4
:10F02000092B00F0C6840A2B00F0B3840B2B01D10E
:10F03000000A00214FEA012900237D083A464FEAE1
:10F04000002849EA106918EB050049F100014CF06D
:10F0500069FAA0F54073B5E76846FFF733F9636ACC
:10F06000019800210BB3012B00F05E82022B00F00F
:10F070009782032B00F00E83042B00F07483052B82
:10F0800000F0A483062B00F0F183072B00F03A84F4
:10F09000082B00F03484092B00F02D840A2B00F09B
:10F0A000A4840B2B01D1000A002162680F02060222
:10F0B0000023510847EA1067701847F100014CF02F
:10F0C00031FAA0F540737DE703A8FFF7A7F9636A5B
:10F0D00004980021002BE8D0C5E7FFF74BFA636ADC
:10F0E000002105460BB3012B00F08182022B00F0BA
:10F0F0001083032B00F08383042B00F09983052BEE
:10F1000000F0EE83062B00F0E583072B00F0F1837F
:10F11000082B00F06784092B00F060840A2B00F0B4
:10F1200059840B2B01D1050A002162680F022E02BF
:10F130000023500847EA1567301847F100014CF0EA
:10F14000F1F9A0F540733DE7624BFFF782BB4FF446
:10F150000043FFF77EBB002800F0EB80012800F0A1
:10F160002E81022800F05E81032800F0BB81042874
:10F1700000F0E581052800F02882062800F0B5821D
:10F180000728E1D0082800F0F380092800F0068164
:10F190000A2800F05381504B4D4A0B2818BF1346E4
:10F1A000FFF757BB494B5B6D03F00703052B3FF699
:10F1B00046AA4A4AD55CFFF756BA4FF400450EE519
:10F1C0005B08FFF746BB4FF480316268002501EB16
:10F1D0005203B3FBF2F39BB280E42D0A002D3FF4FF
:10F1E0002FAAFCE4394B5B6D03F00703052B3FF6B8
:10F1F00026AA3B4AD55CFFF736BA402E7FF41FAAF9
:10F20000636A03B3012B00F00C82022B00F098829A
:10F21000032B00F0D782042B00F02383052B00F092
:10F220008C83062B00F08583072B00F07D83082B51
:10F2300000F09283092B00F0A7830A2B00F09F8334
:10F240000B2B00F097834FF400000021B0E6254A15
:10F25000A2FB03239B08FFF7FCBA224BA3FB053557
:10F26000AD08002D3FF4ECA9B9E46D08002D3FF482
:10F27000E7A9B4E4174DB2E400296FD0012900F0EA
:10F28000C280022900F0F380032900F04A8104299A
:10F2900000F08A81052900F00582062900F03682F7
:10F2A0000729E7D0082972D0092900F086800A29A9
:10F2B00000F01581084D064B0B2918BF1D468EE442
:10F2C000094B77E50000093DFFFC0F0000440258A0
:10F2D0000090D00300093D0090D0030000D1090840
:10F2E00000D10908ABAAAAAA00127A00002850D0BF
:10F2F000012800F0B280022800F00F81032800F0FE
:10F300004881042800F09681052800F0F481062841
:10F3100000F050820728D3D0082848D0092878D098
:10F320000A2800F00781C54BC54A0B2818BF1346B1
:10F3300040E5C44BFFF78DBAC34BA3FB00308008F8
:10F34000FFF72EBBC14AA2FB0323DB08FFF781BAFC
:10F35000BD4BA3FB00308008FFF74FBBB94D3EE427
:10F36000BA4BA3FB0535ED08002D3FF469A936E43F
:10F37000B74BFFF76EBA490881E54008FFF73DBB80
:10F380004FF48043FFF765BA4008FFF709BBB04D63
:10F3900025E4AB4B0EE54FF4804520E4AD4BFFF781
:10F3A00058BA89086BE54FF40053FFF752BAAA4BDD
:10F3B00000E54008CFE540088FE5A64D0FE4A74BD8
:10F3C000FFF747BA4FF4005509E4A04BA3FB003008
:10F3D000C008FFF7E5BA9D4BA3FB0030C008FFF75C
:10F3E0000CBB994BA3FB0123990848E59C4BFFF705
:10F3F00030BA41F25553FFF72CBA934BA3FB0535B6
:10F40000AD08FFF7ECBB954DFFF7E9BB6D08FFF7C3
:10F41000E6BB8F4BCEE44FF48041D6E680085CE536
:10F42000800898E58F4BFFF714BA41F25555FFF766
:10F43000D6BB8B4DFFF7D3BBC90820E57F4BFFF749
:10F4400008BA4FF48053FFF704BA0C23B5FBF3F569
:10F45000002D3FF4F5A8FFF7C2BB7A4BAAE47A4A25
:10F46000A2FB0323DB08FFF7F4B95208D7E47D4D74
:10F47000FFF7B5BB636A03B3012B00F08681022B53
:10F4800000F09481032B00F0FC81042B00F0088233
:10F49000052B00F05D82062B00F06382072B3FF402
:10F4A00085AD082B00F0AE80092B00F021810A2BDE
:10F4B00000F0B3810B2B00F0FA816B48032177E554
:10F4C000614BA3FB0023980807E5684B72E442F602
:10F4D000AA217AE65C4BA3FB002398083BE5574D35
:10F4E000FFF77DBB624BFFF7B4B94FF48055FFF7D0
:10F4F00076BB1B09FFF7ADB90A23B1FBF3F1BEE4FC
:10F5000040F6CC43FFF7A5B95A4BFFF7A2B92D0936
:10F51000002D3FF495A8FFF762BB504B4AE49208D8
:10F520007DE4534DFFF75BBB4008BEE5C008D4E463
:10F53000C00810E5474B3DE44FF4005145E64E4B03
:10F54000FFF787B940F6CC45FFF749BB494DFFF7B8
:10F5500046BB0C23B1FBF3F191E45B09FFF779B9EA
:10F56000394BA3FB0030C008FFF747BA364BA3FB6B
:10F570000030C008FFF714BA6D09002D3FF460A8F1
:10F58000FFF72DBB40F6AA23FFF763B93B4BFFF70C
:10F5900060B93B4B0EE42C4BA3FB02239A083EE4DC
:10F5A000800882E5374B05E4334DFFF718BB0A238B
:10F5B000B0FBF3F0CFE4ED08FFF711BB0A23B0FB7B
:10F5C000F3F08AE441F69811FFE52F4BFFF741B9BC
:10F5D0002A4DFFF704BB0A22B3FBF2F3FFF739B958
:10F5E00040F6AA25FFF7FBBA9B09FFF732B9450899
:10F5F0009BE5AD09002D3FF423A8FFF7F0BA000901
:10F60000FFF7CEB921480021D2E4090937E44FF4CD
:10F610000063FFF71EB90009FFF7EFB91C4BFFF7B6
:10F6200018B94FF480000021C2E40A23B5FBF3F5BA
:10F63000FFF7D5BA0B4BFFF7BDBB00BF20A10700FA
:10F640000020A1070090D003ABAAAAAACDCCCCCCB5
:10F6500080841E0040420F0000093D000048E80180
:10F660002A2C0A000024F400000090D05458140002
:10F67000AAC2A200801A060000127A001516050020
:10F680005485450100350C0000A861000080841EEF
:10F6900090D00300062200234BF044FF05E5D2087A
:10F6A000FFF7BDBBDC4DFFF79ABA0C22B3FBF2F3B8
:10F6B000FFF7CFB8D94BFFF77DBB0C23B0FBF3F0BE
:10F6C00049E441F2545180E5DB09FFF7C2B80C234D
:10F6D000B0FBF3F001E4D24DFFF781BA4FF40065BF
:10F6E000FFF77DBA4909FFF7CABBCE4BFFF7B1B8A8
:10F6F000CD4800215CE4CD4BFFF75CBB0A23B2FB95
:10F70000F3F2FFF78CBB4009FFF74AB9C54DFFF78D
:10F7100066BA850809E54FF48063FFF79AB8400997
:10F72000FFF76BB9ED09002D3EF48AAFFFF757BA2A
:10F730000C23B5FBF3F5FFF752BABD4BFFF789B8C1
:10F740004FF40010002133E48009FFF729B94FF48A
:10F7500080513AE5B74BFFF72DBB0009FFF7FBBB24
:10F760000009FFF7BABBC0089FE44FF48065FFF7BC
:10F7700036BA8009FFF741B94FF22443FFF769B861
:10F78000400857E4AA4DFFF72ABAAB4801210FE41D
:10F790008909FFF774BB4FF40073FFF75AB84FF2B3
:10F7A0002445FFF71CBA4FF400610EE5A348002181
:10F7B000FFF7FEBBA24BFFF7FDBA0C23B2FBF3F23F
:10F7C000FFF72DBB9F480021FFF7F2BB0A22002361
:10F7D0004BF0A8FE69E42D09FFF701BA4FF400755C
:10F7E000FFF7FDB9800825E44009FFF7B4BB4009E5
:10F7F000FFF773BB80A1D1E90001FFF7D9BB062257
:10F8000000234BF08FFE05468FE4854BFFF7D2BAFD
:10F81000062200234BF086FE0CE48B480021FFF704
:10F82000C7BBC009FFF7E9B847F61223FFF711B8C5
:10F83000C5087AE47E4BFFF7BDBA8009FFF74DBBE0
:10F8400047F61225FFF7CBB98009FFF784BB6D0996
:10F85000FFF7C5B9C009FFF7A3B84FF48075FFF7EC
:10F86000BEB94FF480100021FFF7A2BB0C22002389
:10F870004BF058FE19E44FF48061A6E4C909FFF784
:10F88000FEBA5FA1D1E90001FFF792BB4FF480738C
:10F89000FEF7DFBF1209FFF7C2BA5209FFF7BFBA7E
:10F8A0006A480021FFF784BBED09FFF798B9684863
:10F8B0000021FFF77DBB54A1D1E90001FFF778BB20
:10F8C00064480021FFF774BBC009FFF744BBAD09D2
:10F8D000FFF785B90C2200234BF024FE054624E4F3
:10F8E0000A2200234BF01EFE05461EE4C009FFF766
:10F8F000F4BA050919E480090021FFF7D6BB4009D5
:10F90000FFF7D3BB0009FFF7D0BBD209FFF787BAD7
:10F910009209FFF784BA0A2200234BF003FEFFF797
:10F9200089BBC008FFF786BB4FF400200021FFF71A
:10F930003FBB49480021FFF73BBB48480021FFF788
:10F9400037BB4FF4007140E44FF22443FFF732BA63
:10F9500043480021FFF72CBB4FF480200021FFF724
:10F9600027BB2BA1D1E90001FFF722BB3D480021B5
:10F97000FFF71EBB4FF400400021FFF719BB4FF407
:10F9800080300021FFF714BB4FF400300021FFF757
:10F990000FBBC0090021FFF74DBB33480021FFF723
:10F9A00007BB32480021FFF703BB31480021FFF7B6
:10F9B000FFBA80090021FFF73DBB40090021FFF796
:10F9C00039BB0009FFF736BB0C2200234BF0AAFD20
:10F9D000FFF730BBC5090021FFF7A7BB8509002150
:10F9E000FFF7A3BB4509FFF7A0BBC0090021FFF744
:10F9F0005CBB00BFAFF30080002A2C0A00000000AF
:10FA000000AAC2A2000000000015160500000000B8
:10FA1000005561510000000000A861002A2C0A0076
:10FA200090D00300556151000040420F0050C300C8
:10FA300048E8010020A10700000048E8000024F485
:10FA4000AAC2A200005515000020A1070000127AEA
:10FA50000090D00300801A0600AA0A0000CC0C0017
:10FA60000000A8610048E80100093D0000127A008A
:10FA70000024F400F8B50368044613F000661CD0B7
:10FA8000426EB2F5001F00F0A68423D8002A00F0D1
:10FA9000E583B2F5801F20D102210430FAF742F944
:10FAA0000646002E40F09F84626E2368AB48002615
:10FAB000016D21F440110A430265DD0511D5626D27
:10FAC000042A00F20485DFE812F05E04650456049F
:10FAD000DD02DD02B2F5401FE8D0DD054FF0010682
:10FAE000EDD4354698051BD5A26D802A00F06A84B6
:10FAF00000F2EC80002A00F0AB83402A40F0ED8059
:10FB00000021201DFAF70EF923680546002D40F06C
:10FB100091839249A06D0A6D22F4E07202430A6556
:10FB200059051FD5D4F8A420B2F5800F00F01A842F
:10FB300000F2D680002A00F08583B2F5001F40F065
:10FB4000D7800021201DFAF7EDF823680546002D27
:10FB500040F06C838149D4F8A4008A6D22F46002DD
:10FB600002438A651A051FD5D4F8A820B2F1007F98
:10FB700000F0178400F2BF80002A00F07583B2F114
:10FB8000807F40F0C0800021201DFAF7CBF8236869
:10FB90000546002D40F048837049D4F8A8008A6DCE
:10FBA00022F0E06202438A659F0118D5A26C202AE8
:10FBB00000F0828300F2AA803AB1102A40F0A980B6
:10FBC0006649CA6A42F40032CA62002D40F05E8380
:10FBD0006249A06CCA6C22F030020243CA64D804A5
:10FBE0001DD5E26DB2F5005F00F0E48300F2948071
:10FBF000002A00F02183B2F5805F40F0958000215B
:10FC0000201DFAF78FF823680546002D40F00A837F
:10FC10005249E06D0A6D22F4E04202430A659904FC
:10FC20001AD5226EB2F5003F00F087837FD84AB123
:10FC3000B2F5803F40F083800121201DFAF772F871
:10FC400023680546002D40F01B834449206E0A6D51
:10FC500022F4E02202430A655A041BD5D4F8AC20F2
:10FC6000B2F1005F00F05F836CD842B1B2F1805F07
:10FC700070D10121201DFAF755F823680546002DA3
:10FC800040F002833549D4F8AC008A6D22F0E0429E
:10FC900002438A651F040DD5E26EB2F1805F00F069
:10FCA0003083B2F1005F00F0F981002A00F0FC819E
:10FCB00001263546D80163D5626C032A00F20A8416
:10FCC000DFE812F0540003034E005400C02A3FF452
:10FCD0001DAFB2F5807F3FF419AF012635461FE70F
:10FCE000B2F5C00F3FF433AFB2F5000F3FF42FAFC2
:10FCF0000126354636E7B2F1407F3FF44AAFB2F114
:10FD0000806F3FF446AF012635464DE7302A3FF479
:10FD10005CAF0126354662E7B2F5405F3FF475AF50
:10FD2000B2F5804F3FF471AF0126354677E722F4F4
:10FD30008031B1F5802F85D0B2F5403F82D00126C9
:10FD4000354689E722F08051B1F1804F97D0B2F16A
:10FD5000405F94D0012635469CE700BF004402581E
:10FD60000221201DF9F7DEFF23680546002D40F033
:10FD700081823D49606CCA6C22F003020243CA646E
:10FD8000590200F1FF81DF073FD5A26F282A00F258
:10FD90007681DFE812F0300074017401740174019F
:10FDA0007401740174013F037401740174017401DE
:10FDB00074017401740129007401740174017401E7
:10FDC00074017401740130007401740174017401D0
:10FDD00074017401740130007401740174017401C0
:10FDE0007401740174013000012104F12400F9F759
:10FDF0001DFF23680546002D40F05A821A49A06F66
:10FE00004A6D22F0380202434A6598071CD5626F9A
:10FE1000052A00F26583DFE812F00D00E902060012
:10FE20000D000D000D00012104F12400F9F7FEFE84
:10FE300023680546002D40F025820B49606F4A6D0E
:10FE400022F0070202434A65590721D5D4F89020D1
:10FE5000052A00F24283DFE812F01000D302090005
:10FE600010001000100000BF00440258012104F1EE
:10FE70002400F9F7DBFE23680546002D40F0FE81E3
:10FE8000B449D4F890008A6D22F0070202438A65D3
:10FE90009A061DD5D4F88C20B2F1005F00F03982AB
:10FEA00000F20D814AB1B2F1805F40F01281002171
:10FEB000201DF9F737FF23680546002D40F0EC813F
:10FEC000A449D4F88C004A6D22F0E04202434A650E
:10FED0005F061DD5D4F89820B2F5006F00F00782B8
:10FEE00000F207814AB1B2F5806F40F00C81002129
:10FEF000201DF9F717FF23680546002D40F0C88143
:10FF00009449D4F898008A6D22F4E05202438A653D
:10FF100018061DD5D4F89C20B2F5804F00F0DD8185
:10FF200000F2DA804AB1B2F5005F40F0DF800021D4
:10FF3000201DF9F7F7FE23680546002D40F0AA8141
:10FF40008449D4F89C008A6D22F4604202438A6599
:10FF500019070BD5D4F88010B1F5805F00F0F78158
:10FF60007C48426D22F440520A434265DA060BD5C2
:10FF7000D4F89410B1F5807F00F083827548826DCB
:10FF800022F440720A4382651F030ED5D4F8A010F4
:10FF9000B1F5803F00F0E080B1F5003F00F0E38074
:10FFA000002900F05C820126354658030FD5D4F8AD
:10FFB0008420B2F5001F00F0B780B2F5401F00F0BA
